:1000000000000320690200000D020000F92F00002B
:1000100015020000190200001D020000000000008F
:1000200000000000000000000000000021020000AD
:100030002502000000000000290200002D0200003F
:10004000110400001904000021040000290400002C
:10005000310400003904000041040000490400009C
:10006000510400005904000061040000690400000C
:10007000710400007904000081040000890400007C
:100080009104000099040000A1040000A9040000EC
:10009000B1040000B9040000C1040000C90400005C
:1000A000C1330000DD250000D1040000D9040000A8
:1000B000E1040000E9040000F1040000F90400007C
:1000C00001050000090500001105000019050000E8
:1000D0002105000029050000310500003905000058
:1000E00041050000490500005105000059050000C8
:1000F0006105000069050000710500007905000038
:1001000035380000CD37000075200000E54F0000B5
:100110008105000089050000910500009905000097
:10012000A1050000A9050000B1050000B905000007
:10013000C1050000C9050000554F00001520000052
:10014000D1050000D9050000E1050000E905000027
:10015000F1050000F9050000010600000906000095
:100160001106000019060000D1330000210600002E
:10017000290600002D0600003106000035060000AB
:10018000390600003D060000450600004D0600004F
:10019000550600005D060000650600006D060000C3
:1001A000750600007D060000850600008D06000033
:1001B000950600009D060000A5060000AD060000A3
:1001C000B1060000B5060000B9060000BD0600003B
:1001D000A0D700000000002050000000A0D70000C1
:1001E0000000FF1F00000000A0D700000000001466
:1001F000000000005000002060B001000000FF1F60
:10020000000000000000001400000000FEE700BF36
:10021000FEE700BFFEE700BFFEE700BFFEE700BF4E
:10022000FEE700BFFEE700BFFEE700BFFEE700BF3E
:10023000FEE700BF002393420AD210B450F8044BEB
:1002400041F8044B04339342F8D35DF8044B7047F4
:10025000704700BF002303E0002240F8042B043362
:100260008B42F9D3704700BF10B572B60AF0D0FDCB
:100270000E4B07E003F10C049A6859681868FFF701
:10028000D9FF23460A4A9342F4D30A4A934209D239
:100290001C46596854F8080BFFF7DCFF2346054A53
:1002A0009342F5D362B60BF085FCFEE7D001000067
:1002B000F40100000C020000FFFFFFFFFFFFFFFF43
:1002C000FFFFFFFFFFFFFFFFFFFFFFFFFFFFFFFF3E
:1002D000FFFFFFFFFFFFFFFFFFFFFFFFFFFFFFFF2E
:1002E000FFFFFFFFFFFFFFFFFFFFFFFFFFFFFFFF1E
:1002F000FFFFFFFFFFFFFFFFFFFFFFFFFFFFFFFF0E
:10030000FFFFFFFFFFFFFFFFFFFFFFFFFFFFFFFFFD
:10031000FFFFFFFFFFFFFFFFFFFFFFFFFFFFFFFFED
:10032000FFFFFFFFFFFFFFFFFFFFFFFFFFFFFFFFDD
:10033000FFFFFFFFFFFFFFFFFFFFFFFFFFFFFFFFCD
:10034000FFFFFFFFFFFFFFFFFFFFFFFFFFFFFFFFBD
:10035000FFFFFFFFFFFFFFFFFFFFFFFFFFFFFFFFAD
:10036000FFFFFFFFFFFFFFFFFFFFFFFFFFFFFFFF9D
:10037000FFFFFFFFFFFFFFFFFFFFFFFFFFFFFFFF8D
:10038000FFFFFFFFFFFFFFFFFFFFFFFFFFFFFFFF7D
:10039000FFFFFFFFFFFFFFFFFFFFFFFFFFFFFFFF6D
:1003A000FFFFFFFFFFFFFFFFFFFFFFFFFFFFFFFF5D
:1003B000FFFFFFFFFFFFFFFFFFFFFFFFFFFFFFFF4D
:1003C000FFFFFFFFFFFFFFFFFFFFFFFFFFFFFFFF3D
:1003D000FFFFFFFFFFFFFFFFFFFFFFFFFFFFFFFF2D
:1003E000FFFFFFFFFFFFFFFFFFFFFFFFFFFFFFFF1D
:1003F000FFFFFFFFFFFFFFFFFFFFFFFFFFFFFFFF0D
:10040000FFFFFFFFFFFFFFFFFFFFFFFFFEFFFFFFFD
:1004100008B508F0DBFE08BD08B508F0F7FE08BD1A
:1004200008B508F013FF08BD08B508F02FFF08BD98
:1004300008B508F04BFF08BD08B508F067FF08BD18
:1004400008B508F083FF08BD08B508F09FFF08BD98
:1004500008B508F0BBFF08BD08B508F0D7FF08BD18
:1004600008B508F0F3FF08BD08B509F00FF808BD9E
:1004700008B509F02BF808BD08B509F047F808BD24
:1004800008B509F063F808BD08B509F07FF808BDA4
:1004900008B5FFF7CDFE08BD08B5FFF7C9FE08BDDA
:1004A00008B5FFF7C5FE08BD08B5FFF7C1FE08BDDA
:1004B00008B5FFF7BDFE08BD08B5FFF7B9FE08BDDA
:1004C00008B5FFF7B5FE08BD08B5FFF7B1FE08BDDA
:1004D00008B5FFF7ADFE08BD08B5FFF7A9FE08BDDA
:1004E00008B5FFF7A5FE08BD08B5FFF7A1FE08BDDA
:1004F00008B5FFF79DFE08BD08B50AF02DFC08BD44
:1005000008B5FFF795FE08BD08B50AF037FC08BD31
:1005100008B5FFF78DFE08BD08B50AF041FC08BD1F
:1005200008B5FFF785FE08BD08B50AF04BFC08BD0D
:1005300008B5FFF77DFE08BD08B5FFF779FE08BDD9
:1005400008B5FFF775FE08BD08B5FFF771FE08BDD9
:1005500008B5FFF76DFE08BD08B5FFF769FE08BDD9
:1005600008B5FFF765FE08BD08B5FFF761FE08BDD9
:1005700008B5FFF75DFE08BD08B5FFF759FE08BDD9
:1005800008B5FFF755FE08BD08B5FFF751FE08BDD9
:1005900008B5FFF74DFE08BD08B5FFF749FE08BDD9
:1005A00008B5FFF745FE08BD08B5FFF741FE08BDD9
:1005B00008B5FFF73DFE08BD08B5FFF739FE08BDD9
:1005C00008B5FFF735FE08BD08B5FFF731FE08BDD9
:1005D00008B5FFF72DFE08BD08B5FFF729FE08BDD9
:1005E00008B50AF001FC08BD08B5FFF721FE08BDFB
:1005F00008B5FFF71DFE08BD08B5FFF719FE08BDD9
:1006000008B5FFF715FE08BD08B5FFF711FE08BDD8
:1006100008B5FFF70DFE08BD08B5FFF709FE08BDD8
:1006200008B5FFF705FE08BDFFF7FABFFFF7F8BFF3
:10063000FFF7F6BFFFF7F4BFFFF7F2BF08B50AF008
:1006400089FA08BD08B5FFF7F3FD08BD08B5FFF747
:10065000EFFD08BD08B5FFF7EBFD08BD08B5FFF7D6
:10066000E7FD08BD08B509F089FE08BD08B5FFF72C
:10067000DFFD08BD08B5FFF7DBFD08BD08B5FFF7D6
:10068000D7FD08BD08B5FFF7D3FD08BD08B509F0D3
:100690006BFE08BD08B5FFF7CBFD08BD08B5FFF739
:1006A000C7FD08BD08B5FFF7C3FD08BDFFF7FABFDA
:1006B000FFF7F8BFFFF7F6BFFFF7F4BFFFF7F2BF92
:1006C0002DE9F0470BF048F80AF048FC0AF0BCFDB1
:1006D00001F042FE4FF6FF7300BF013B9BB2002BBF
:1006E000FAD102F055FC04F061FD00F07BF800F057
:1006F00049FC4FF6FF7300BF013B9BB2002BFAD1C0
:1007000000F0AAFA002858D000F0B8FA0028FBD16F
:10071000012002F01FFA04F0B5FB02F0B5FF00283B
:100720004ED0284A284DD2F80831284EDFF8A8A02C
:10073000DFF8A890264FDFF8A88043F00103C2F845
:1007400008312C68013C2C608CB103F001FD78BBB2
:1007500000F04EF802F0FEFE00F07AFC02F0F4FA2F
:1007600001F024FE2C68013C2C60002CEDD102200D
:1007700008F07AFA49460246384609F003FA4FF083
:10078000400E4FF0010C1349A6F804E02346424600
:100790003846C6F810A0B460C6F814C0347334608C
:1007A00009F0CCFC00F0FEF803F0D2FC0028CFD01A
:1007B00000F00CFC01F0FAFDC3E702F0CBF9AAE768
:1007C000BDE8F0870070034000000020B4AE0120B7
:1007D00000700E408CAE012088AE0120F4D60000DF
:1007E000AD160000014B00221A7070479CB001202A
:1007F00038B5154A154D164B106929781B69154AED
:10080000C0F30040C3F3802301F00F0143EA40032B
:1008100002EB8102D45C2C7004F0F004102C02D0A6
:10082000202C00D038BD03F015FD40B903F002FDC7
:100830000028F7D02046BDE8384004F0F1B8204643
:10084000BDE8384003F05ABD00F00F409CB00120D5
:1008500040F00F40D8C1000070B50D46064601F0CB
:1008600071FF022D044613D0E8B107282DD00628C9
:1008700036D024F00203012B22D024F00403022BF3
:1008800033D1304601F0E6FFBDE8704003F078BC9C
:1008900018B903F0E7FC70B170BD841F012CFBD8C0
:1008A00003F06EFCF5E703F0DDFC0028F4D03046E1
:1008B00001F06CFFDDE73046BDE8704001F066BF37
:1008C0003046BDE8704001F047BF03F0CBFC002884
:1008D000EDD1304601F0DAFFBDE8704003F050BCC6
:1008E00003F0C0FC0028CCD0E1E7231F012B0AD87D
:1008F000304601F099FF03F0B5FC0028ECD03046FB
:1009000001F092FFE5E7072CE3D070BD10B51E4C57
:100910001E48214607220BF05CF920460722FF21E2
:100920000BF059F923786FF30413237063786FF396
:100930000003637023786FF34513237023796FF3FB
:10094000C303237123796FF382032371A3786FF3B9
:100950008203A370A3786FF34513A370A3786FF39A
:100960000413A370A3786FF30003A370E3786FF30D
:100970008613E370E3786FF34513E370E3786FF366
:100980008203E37010BD00BF481C0020501C0020F3
:100990000249034807220BF01CB900BF481C002085
:1009A000501C002030B4074A074C084B1461262421
:1009B00001251471022455711C7030BC044905488E
:1009C00009F006BCB4AE01204E1C0020A1B00120ED
:1009D0008CAE012000700E40082833D8DFE800F00C
:1009E0004933233E541D150D050003292AD8DFE89D
:1009F00011F00E010401FA002000032922D8DFE8DB
:100A000011F0E800DE00D400CA0003291AD8DFE89C
:100A100011F0B800AE00A4009A00032912D8DFE854
:100A200001F0887E746A03290CD8DFE801F05A507F
:100A3000463C884B5A796FF386125A715A796FF394
:100A4000C7125A717047002900F0FD80012926D194
:100A5000804A13786FF3C30313707047002900F0C6
:100A6000E68002291DD17B4A13796FF3410313718C
:100A70007047002900F0D580012913D1754A1378F9
:100A80006FF3000313707047002900F0D68002292D
:100A900006D1704A13796FF30003137170477047E2
:100AA0007047704770476B4B1A786FF382021A7069
:100AB0001A786FF341021A707047664B1A786FF319
:100AC00082021A701A7842F002021A707047614B63
:100AD0001A7842F004021A701A786FF341021A7001
:100AE00070475C4B1A7842F004021A701A7842F090
:100AF00002021A707047574B5A796FF300025A710D
:100B00005A796FF341025A717047524B5A7942F049
:100B100001025A715A796FF341025A7170474D4B75
:100B20005A796FF300025A715A7942F002025A71EF
:100B30007047484B5A7942F001025A715A7942F093
:100B400002025A717047434B5A796FF382025A710D
:100B50005A796FF3C3025A7170473E4B5A7942F08B
:100B600004025A715A796FF3C3025A717047394BB4
:100B70005A796FF382025A715A7942F008025A7117
:100B80007047344B5A7942F004025A715A7942F054
:100B900008025A7170472F4B5A796FF304125A7139
:100BA0005A796FF345125A7170472A4B5A7942F0BD
:100BB00010025A715A796FF345125A717047254BDA
:100BC0005A796FF304125A715A7942F020025A711D
:100BD0007047204B5A7942F010025A715A7942F00C
:100BE00020025A7170471B4B5A7942F040025A71E9
:100BF0005A796FF3C7125A717047164B5A796FF3CF
:100C000086125A715A7942F080025A717047114B1C
:100C10005A7942F040025A715A7942F080025A7170
:100C200070470C4A137843F0010313707047094A68
:100C3000137943F0020313717047064A137943F0A6
:100C4000010313717047034A137843F008031370CC
:100C5000704700BF481C0020074B1A88100709D4B2
:100C60001A88D10706D41A88520703D41888C0F30B
:100C7000400070470120704794B0012038B5124BF6
:100C800012491A78002008607AB1114B1A881007AF
:100C900009D41A88D10706D41A88520703D41888B1
:100CA000C0F3400038BD012038BD0A4A0A4C146127
:100CB00026240125147109490948557102241C7024
:100CC00009F086FAE1E700BFA1B00120241C002052
:100CD00094B00120B4AE01204E1C00208CAE012047
:100CE00000700E402DE9F04F012985B070D902291E
:100CF00007D06A4A136823F08043136005B0BDE84B
:100D0000F08F674A674B32F81020C2F3C011009190
:100D1000C2F380110191C2F340110291C2F300119C
:100D2000C2F3803BC2F3403AC2F30039C2F3C02899
:100D3000C2F3802EC2F3402CC2F30027C2F3C006D8
:100D4000C2F38005C2F34004039102F00102197856
:100D500000986BF3C711197019796AF3C3011971FF
:100D6000197969F382011971597868F38201597010
:100D700059786EF3C711597099786CF382019970A4
:100D8000997867F3C7119970D97860F30001D97029
:100D9000D978019860F3C711D970D978029860F3B7
:100DA0004101D970D978039860F30411D970D978CA
:100DB00066F38611D970D97865F3C301D970D978F3
:100DC00064F38201D970D97862F34511D97090E744
:100DD000334A344B32F810201878C2F3803B6BF35F
:100DE000041018701878C2F3403A6AF3451018706E
:100DF0001878C2F3003969F3861018705878C2F376
:100E0000C02868F3000058705878C2F3802E6EF343
:100E1000410058705878C2F3402C6CF3C3005870EE
:100E20005878C2F3002767F3451058705878C2F31A
:100E3000C01464F30410587058780094C2F38014FE
:100E400064F38610587098780194C2F3401464F3E8
:100E50000000987098780294C2F3001464F3410083
:100E6000987098780394C2F3C00666F3C300987034
:100E70009878C2F3800565F3451098709878C2F3AE
:100E8000400464F304109870987802F0010262F351
:100E90008610987000293FF45AAF2AE7601C0020A2
:100EA000FCC10000581C0020032842D8DFE800F0F5
:100EB00014262F02214B1A7942F010021A711A7966
:100EC00042F020021A711A7942F040021A711A791E
:100ED0006FF3C7121A717047184B1A796FF3041227
:100EE0001A711A7942F020021A711A7942F04002FE
:100EF0001A711A7942F080021A7170470F4B1A79F1
:100F000042F010021A711A796FF34512ECE70B4B9D
:100F10001A7942F010021A711A7942F020021A71FD
:100F20001A796FF386121A711A7942F080021A71D7
:100F30007047024B1A7942F01002D1E7481C00209A
:100F400030B4064B064D074C00394FF0010218BF74
:100F500001211A702980207030BC70479EB001209A
:100F600096B001209FB0012000380449044B18BFFF
:100F70000120002208801A70704700BF96B001203F
:100F80009EB0012038B50C4B0C4A0D4C0D4918464B
:100F90004FF6FF7500F8065F1061262001251071DD
:100FA0004FF0FF3055711860022598800648257073
:100FB00009F00EF9257038BD481C0020B4AE0120A0
:100FC000A1B001208CAE012000700E4038B5184C45
:100FD000184D23782A7843F00103237002B138BDFD
:100FE00003F0B6F870B1144A144B136101242623A0
:100FF0001371547102232B7011491248BDE8384017
:1010000009F0E6B8104B0C4A1870197850710C446E
:10101000146119780D4C481C645C1471C0B21870CE
:1010200001232B7006490748BDE8384009F0D0B8C5
:10103000481C0020A1B00120B4AE012048000020CF
:101040008CAE012000700E40A0B00120F4C1000061
:10105000F8B50524601EC0B201F074FB05460728F0
:1010600000F22281DFE810F02601080008000800E5
:101070001C011C0110002B0102F09CF9020600F17A
:101080001981012D00F00C81204601340321E4B2C6
:10109000FFF7A2FC092CDDD1B74C23883BB101330B
:1010A0009BB24CF25032934200F2E8812380B34D60
:1010B000B34E338843B12A78002A40F0058132804C
:1010C00002F078F90306FBD4AE4B1B68002B40F00E
:1010D0000D8103F0D5F8002840F01D81AA4F3B8810
:1010E0005A1CC3F30E033A80002B00F02A812B78A0
:1010F000012B06D13388228813439BB2002B00F0CA
:101100005381A24AA24B10781978C0F3001060F303
:101110000411197010781978C0F3401060F345116C
:10112000197010781978C0F3801060F38611197067
:101130005078597860F30001597050785978C0F3AD
:10114000400060F34101597050785978C0F3C000F5
:1011500060F3C301597050785978C0F3401060F3C0
:101160004511597050785978C0F3001060F304119C
:10117000597050785978C0F3801060F38611597017
:101180009078997860F30001997090789978C0F31D
:10119000400060F34101997090789978C0F3C000E5
:1011A00060F3C301997090789978C0F3401060F3B0
:1011B0004511997090789978C0F3001060F304118C
:1011C000997090789978C0F3801060F386119970C7
:1011D00010781978C00960F3C7111970107919795E
:1011E000C0F3C00060F3C301197110791979C0F31D
:1011F000800060F38201197150785978C0F3800043
:1012000060F38201597050785978C00960F3C711B2
:10121000597090789978C0F3800060F382019970DA
:1012200090789978C00960F3C7119970D078D9780F
:1012300060F30001D970D078D978C00960F3C71184
:10124000D970D078D978C0F3400060F34101D970EB
:10125000D078D978C0F3001060F30411D970D07839
:10126000D978C0F3801060F38611D970D078D9781E
:10127000C0F3C00060F3C301D970D078D978C0F34F
:10128000800060F38201D970D178DA78C1F340111F
:1012900061F34512DA703F4C2378002B59D0F8BD2A
:1012A00001212046FFF798FB0134E4B2092C7FF4BA
:1012B000D1AEF1E600212046FFF78EFBF4E70221D4
:1012C0002046FFF789FBEFE701339BB242F6E0626D
:1012D000934240F293810023338002F06BF80706BB
:1012E000FBD4284B1B68002B3FF4F3AE02F0A2FFA7
:1012F00000283FF4EEAE02F05DF8254B1A78C005E9
:101300004CBF6FF3C30242F008021A7002F0B8FF3C
:1013100000283FF4E3AE02F08DFF002800F08F803C
:1013200002F0A6FF00283FF4D9AE02F043F8184BB4
:101330001A78C1054CBF6FF3000242F001021A7027
:10134000CCE602F03FFE002800F0968001233B80AF
:10135000CDE602F0FDFE002877D00F4A0F4B136157
:10136000262301251371022355712370BDE8F8402F
:101370000B490C4808F02CBF98B001209EB001200A
:1013800096B0012014A601209AB00120581C00201C
:10139000481C0020A1B00120B4AE0120480000206C
:1013A0008CAE012000700E4002F004F803067FF5B9
:1013B000A8AEB44B1A78012A40F22281022A7FF4A7
:1013C0006AAFB14B1A7842F080021A701A7942F073
:1013D00008021A711A7942F004021A715A7842F01E
:1013E00004025A705A7842F080025A709A7842F099
:1013F00004029A709A7842F080029A70DA7842F089
:101400000102DA70DA7842F08002DA70DA7842F0BB
:101410000202DA70DA7842F01002DA70DA7842F01A
:101420004002DA70DA7842F00802DA70DA7842F0D4
:101430000402DA70DA7842F02002DA702BE702F068
:1014400001FF00287FF46CAF48E6904B8E4918707E
:101450001D788F4A29441161197850718D4D481CAF
:10146000C0B26D5C1870012315712370BDE8F8409F
:1014700089498A4808F0ACBE388038E688490A684D
:1014800000202080002A3FF412AE864B864D1E7845
:1014900062F304161E701E78C2F3400767F3451608
:1014A0001E701E78C2F3800767F386161E705E7882
:1014B000C2F3C00767F300065E705E78C2F30017E0
:1014C00067F341065E705E78C2F3401767F3C306A8
:1014D0005E705E78C2F3801767F345165E705E78C3
:1014E000C2F3C01767F304165E705E78C2F300277C
:1014F00067F386165E709E78C2F3402767F3000696
:101500009E709E78C2F3802767F341069E709E7896
:10151000C2F3C02767F3C3069E709E78C2F30037FC
:1015200067F345169E709E78C2F3403767F3041642
:101530009E709E78C2F3803767F386169E701E7881
:10154000C2F3C03767F3C7161E701E790860C2F376
:101550000040314660F3C30119711979C2F340406C
:1015600060F3820119715978C2F3804060F38201FF
:1015700059705978C2F3C04060F3C7115970997817
:10158000C2F3005060F3820199709978C2F3405021
:1015900060F3C7119970D978C2F3805060F30001ED
:1015A000D970D978C2F3C05060F3C711D970D97817
:1015B000C2F3006060F34101D970D978C2F3406092
:1015C00060F30411D970D978C2F3806060F386119A
:1015D000D970D978C2F3C06060F3C301D970D978EB
:1015E000C2F3007060F38201D970D978C2F3407001
:1015F00060F34511D20FD9702A7059E5338063E545
:10160000214B197841F010011970197841F020012F
:101610001970197841F040011970597841F00101B1
:101620005970597841F002015970597841F0080118
:101630005970597841F020015970597841F01001E2
:101640005970597841F040015970997841F0010181
:101650009970997841F002019970997841F00801E8
:101660009970997841F020019970997841F01001B2
:101670009970997841F040019970002A3FF4A2AE28
:1016800009E600BF9FB00120481C0020A0B0012047
:10169000B4AE0120F4C100008CAE012000700E40F9
:1016A000601C0020581C00209EB00120954B4FF676
:1016B000FF71196002B170472DE9F047924D2B7808
:1016C000013B1446032B12D8DFE813F0040022007C
:1016D000DC0013008D4B1A78052A40F2FE808C48FE
:1016E000027800241C70002A40F0E4802A70BDE8D3
:1016F000F087884A884B1361262301241371022343
:1017000054712B70BDE8F0478449854808F060BDEE
:1017100002F01EFD002840F0DD80824F824E4FF027
:10172000010801F047FE57F82430C01A062805D9F1
:10173000336808FA04F223EA020333600134082C08
:10174000EFD13368DFF8E881DC070ED498F8063073
:10175000D80700F10B82754C2388D90740F1048328
:1017600023889BB243F00103238033689C070ED487
:1017700098F806306D4CDB09238840F00F819807FC
:1017800040F1508223889BB243F0020323803368E8
:1017900059070ED498F806301A0700F12282634CDC
:1017A00023885B0740F1B28223889BB243F0040395
:1017B0002380346814F008040ED198F80630980796
:1017C00000F1F381594C2388190740F17E82238868
:1017D0009BB243F0080323803368DC060ED498F8EC
:1017E0000630580600F15C81504C2388D90640F140
:1017F000788223889BB243F01003238033689C06D1
:1018000015D498F80630980600F11E81474C2388BD
:10181000990640F1428223889BB243F02003238043
:1018200001F0C8FD7861336843F02003336033680A
:101830005C060ED498F80630D80600F164813B4C63
:101840002388590640F17B8223889BB243F04003F2
:10185000238033681C060DD498F8063058076BD4E3
:10186000324C2388190640F1988223889BB243F0BA
:1018700080032380254B274A002018701978507167
:10188000414407E0214B2A49224A002018701C7865
:101890005071214411611978264C481CC0B2645C17
:1018A0001870012314712B70BDE8F0471B491C48C8
:1018B00008F08EBC174A184B0470136101242620CF
:1018C0000223107154712B70BDE8F047134914487E
:1018D00008F07EBCDFF85880CCE71C7814480D4A2D
:1018E000144D0E49204410611C780D482D5D157172
:1018F00001340025E4B255711C70BDE8F04708F0D2
:1019000067BC00BF00000020A1B00120A0B00120F2
:101910009DB00120B4AE01204E1C00208CAE0120F1
:1019200000700E40281C0020241C002094B00120D0
:10193000481C0020F4C10000B84B1A88120699D543
:101940001A8822F080021204120C1A8001F032FD73
:10195000B34B0720DB6900F0F5FE0446002800F0D9
:101960009282072800F0B382062800F0D08224F08B
:101970000203012B00F0618224F00403022B40F0EB
:101980000783072000F066FF02F0FAFB01F012FD6A
:10199000F861336843F0800333606BE79A077FF5A3
:1019A000F6AE238823F002031B041B0C238001F0F6
:1019B00001FD9B4B5B68C01AB0F5FA7F4FF004093C
:1019C00021D902F04FFC5FFA89FA03465046002BFA
:1019D00000F0258200F094FE30B923889BB223FAF0
:1019E00009F3DB0700F1F08209F10109B9F1080FF1
:1019F000E7D102F0C5FB01F0DDFC7860336843F00D
:101A000002033360C3E602F02DFC5FFA89FA034655
:101A10005046002B00F0FA8100F072FE30B92388A6
:101A20009BB223FA09F3D80700F1CE8209F101092C
:101A3000B9F1080FE7D102F033FC002840F07A82B8
:101A4000012002F079FED4E7744B1A8892067FF5E4
:101A5000EEAE1A8822F020021204120C1A8001F055
:101A6000A9FC6F4B05205B6900F06CFE0446002862
:101A700000F0F781072800F01682062800F0548253
:101A800024F00203012B00F0DC8124F00403022B7C
:101A900040F05482052000F0DDFE02F071FBBFE64D
:101AA0005E4B1A88D2067FF5A9AE1A8822F0100282
:101AB0001204120C1A8001F07DFC594B04201B69A2
:101AC00000F040FE0446002800F0BF81072800F027
:101AD0000882062800F0158224F00203012B00F092
:101AE000A88124F00403022B40F03682042000F089
:101AF000B1FE02F045FB01F05DFC3861336843F054
:101B0000100333607AE6454B1A8852067FF5A1AE82
:101B10001A8822F040021204120C1A8001F04AFCCA
:101B20003F4B06209B6900F00DFE0446002800F0A4
:101B3000A181072800F0C181062800F0DC8124F093
:101B40000203012B00F0718124F00403022B40F00A
:101B50001182062000F07EFE02F012FB01F02AFC4A
:101B6000B861336843F04003336072E62B4B1A8848
:101B7000D2077FF5FAAD1A8822F001021204120C86
:101B80001A8001F017FC264B1B6802F063FB044629
:101B9000002800F0348102F097FB01F00BFC386064
:101BA000336843F001033360DFE51C4B1A881207EA
:101BB0007FF512AE1A8822F008021204120C1A8065
:101BC00001F0F8FB164BDB6802F034FB002840F014
:101BD000638101F0EFFBF860336843F00803336082
:101BE000FAE50E4B1A8854077FF5E3AD1A8822F008
:101BF00004021204120C1A8001F0DCFB084B9B68F3
:101C0000C01AB0F5FA7F40F2298101F0D3FBB86029
:101C1000336843F004033360CBE500BF94B0012088
:101C2000041C002001F0C6FBBC4B4FF004095860B7
:101C300002F018FB5FFA89FA0346504653B300F0EE
:101C40005FFD30B923889BB223FA09F3D90700F16D
:101C5000AD8109F10109B9F1080FE9D1B04B1A883A
:101C60000AB101221A80AF4BD3F8282122F00102D9
:101C7000C3F82821D3F8282142F00102C3F8282113
:101C800002F07EFA01F096FB7860336843F00203BD
:101C9000336077E500F024FDDBE701F08BFB9F4A22
:101CA00003460520536100F04DFD28B10638012898
:101CB0003FF6B1AD02F064FA02F0D4FA00287FF4E6
:101CC000AAAD052000F062FDA5E501F073FB934B82
:101CD000D86001F06FFBF860336843F008033360AD
:101CE00075E501F067FB8D4A03460420136100F09F
:101CF00029FD002871D0063801286CD901F05AFB63
:101D00003861336843F01003336072E501F052FB31
:101D1000824A844B9060D3F8282122F00102C3F854
:101D20002821D3F8282142F00102C3F8282101F02C
:101D300041FBB860336843F00403336034E501F0DD
:101D400039FB764A03460620936100F0FBFC00282D
:101D500039D00638012834D901F02CFBB86133683A
:101D600043F0400333606FE501F024FB6B4A6D4B99
:101D70001060D3F8282122F00102C3F82821D3F8FB
:101D8000282142F00102C3F8282101F013FB38603A
:101D9000336843F001033360E2E401F00BFB5F4A78
:101DA00003460720D36100F0CDFC00B306380128BC
:101DB0001BD901F0FFFAF861336843F08003336008
:101DC00053E502F0DDF902F04DFA0028C4D10620F7
:101DD00000F0DCFCC0E702F0D3F902F043FA00287F
:101DE0008CD1042000F0D2FC88E702F0C9F902F09F
:101DF00039FA0028DDD1072000F0C8FCD9E702F04D
:101E000047FA2246012103F005F8C6E600F068FC17
:101E100000283FF40BAE504600F04AFDE9E500F023
:101E20005FFC00283FF4E0ADF5E7062000F094FCED
:101E300094E6042000F090FC5DE6072000F08CFCA6
:101E4000A4E5052000F088FCEAE402F00BFA002883
:101E50003FF451AE042000F099FC3DE602F038FE5C
:101E6000D3E602F0FFF900283FF4DAAC052000F0D9
:101E70008DFC05E602F0F6F900283FF46FAE06206F
:101E800000F084FC5BE602F0EDF900283FF47EAD43
:101E9000072000F07BFC6AE502F0FAF922460121F6
:101EA00002F064FE95E602F0DDF90028DED105209F
:101EB00000F0ECFC02F064F9B2E402F0D3F900287F
:101EC000DDD1062000F0E2FC02F05AF946E602F00D
:101ED000C9F90028DCD1072000F0D8FC02F050F945
:101EE00054E502F0BFF90028B4D1042000F0CEFC84
:101EF00002F046F9FFE502F0B5F900283FF429AEFB
:101F0000BDE702F0AFF900283FF4F0ADA2E702F020
:101F1000A9F900283FF435ADBAE700BF041C002042
:101F200098B001200070034002F09CF900283FF4B3
:101F3000B1AD9BE7002002F0FFFB5AE5231F012B08
:101F400054D8052000F070FC02F08CF90028B1D0C4
:101F5000052000F069FCAAE7231F012B52D80420BA
:101F600000F062FC02F07EF90028C1D0042000F0ED
:101F70005BFCBAE7231F012B3CD8062000F054FC81
:101F800002F070F900289FD0062000F04DFC98E781
:101F9000231F012B32D8072000F046FC02F062F923
:101FA00000289BD0072000F03FFC94E7504600F04B
:101FB00097FBB8B1504600F07BFC50460021FEF77D
:101FC0004BFC02F0DDF85DE6504600F089FBE8B11D
:101FD000504600F06DFC50460021FEF73DFC02F03B
:101FE000CFF808E5504600F0D1FBE3E7072C7FF47B
:101FF00017AC5CE7072C7FF4B1AD62E7072C3FF428
:102000006AAFC3E4072C7FF476AD6EE7504600F06C
:10201000BDFBDDE738B51048104C07F0F9FC014670
:102020000D4807F023FD237843B1013B022B02D872
:102030000B4B01221A70BFF34F8F38BD094A0A4B70
:10204000136126230125137108490948557102239C
:10205000237008F0BDF8EBE700F10F40A1B00120BC
:102060009DB00120B4AE01204E1C00208CAE01209A
:1020700000700E40224AD2F82C3103F0010310B553
:10208000C2F82C3102F064F890B91E4C2388D907AD
:102090001CD423889A0711D423885B0709D4184AD3
:1020A000D2F8283123F00103C2F82831BFF34F8F53
:1020B00010BD0021022002F063FBF0E701210220A5
:1020C00002F05EFB23885B07E9D5F2E7238823F063
:1020D00001031B041B0C238002F0ACF830B102207A
:1020E00002F0C2FC23889A07D6D5E7E702F0AAF8E7
:1020F0000028F4D1014601221E2002F037FDC8E776
:102100000070034094B00120F8B53D4C3D4E0123D2
:1021100002253370E570A37803F0BF03A370204657
:1021200007F050FF830659D4A37843F03003A3701F
:102130004FF4967300BF013BFCD1334D304A4AF255
:1021400002034FF49674EB5A03EB830315F8133034
:102150005B00DBB2137100BF013CFCD14AF2020309
:10216000274FEB5A03EB830305EB430213465278E8
:10217000591C01322346384607F032FF234B1860C2
:10218000E8B9384607F00AFF48B1BC7000BF022327
:102190008022BA70FB70BB7843F04003BB70184AD2
:1021A0004AF2020402202B5BD07091780133C3F312
:1021B0000B0341F040012B5391703070F8BD38464D
:1021C00007F0ECFEBC7000BF80230222BB70FA70E7
:1021D000BB7843F04003BB703270F8BD204607F077
:1021E000DDFE0023A37000BF8023A3702046E570AE
:1021F00007F0E8FEA37843F04003A3703570F8BD04
:1022000000700640A4B0012088BC00208C5C012036
:10221000172870B50C4611D878B3013816282CD879
:10222000DFE800F0585B5E2B2B2B2B2B2B2B2B2B63
:102230002B2B2B2B2B2B2B612B644500E22858D00A
:10224000E4281BD13A4C3B4904F520450622288856
:1022500000EB800004EB400009F0BBFC2B88364A01
:1022600003EB8301127804EB41040133C3F30B0346
:10227000AD21D2432B806171E27170BDE128FCD1A8
:102280002B4D2E4905F520460622308800EB8000B4
:1022900005EB400009F09DFC338803EB830205EB5E
:1022A00042050133C3F30B0333806C7170BD2048CA
:1022B000234900F52044062223885D1C03EB830399
:1022C00000EB4300258009F084FC2388C3F30B0353
:1022D000238070BD164D1B49D4E7154D1A49D1E72F
:1022E00013481A49E5E712481949E2E71048194925
:1022F000DFE70F4D0F4905F520460622308800EB39
:10230000800005EB400009F064FC328802EB820398
:10231000013205EB4303C2F30B02AC25200E210C66
:102320003280220A1C725D71D87199715A7270BD27
:1023300088BC002080C200004800002098C2000035
:1023400068C2000090C20000A0C2000078C2000075
:1023500088C2000070C2000008B54AF204020021E1
:102360000E4809F038FC4AF2040200210C4809F03A
:1023700032FC0C4B0C492220002218709A709A787B
:1023800042F0C0029A705A7942F080025A719A79EA
:10239000022002F0DF029A71087008BD641C002060
:1023A00088BC002000700640A4B00120F8B5854C20
:1023B000854D4AF2020704F52046E25B338829780E
:1023C000934201D002297CD09B1A322B15DD0329C0
:1023D00013D17E4B7E489978002201F0BF0199709D
:1023E000326002709A7000BF022280219970DA7008
:1023F0002A709A7842F040029A7076484AF20204B3
:1024000000F52042035B12889A420CD003EB830153
:1024100000EB410101334D780A794E79C3F30B0388
:10242000042D035300D0F8BD172A35D8002AFAD05E
:10243000531E162BF7D801A252F823F0E124000016
:10244000FB2400002725000027240000272400008B
:102450002724000027240000272400002724000050
:102460002724000027240000272400002724000040
:102470002724000027240000272400002724000030
:1024800027240000272400001F2500002724000027
:102490002F250000CF240000E02A52D0E32AC2D129
:1024A00001F056FE0028BED0FEF772FA01F0F8FEE9
:1024B00002F042F9002001F045FE474BFF221A705E
:1024C000F8BDFFF721FEE25B338829787CE701F055
:1024D0003FFE002862D1BDE8F840012002F0C4BAF6
:1024E00001F036FE00284FD11E2E9CD80022304627
:1024F0001146BDE8F84002F08DBC01F029FEC8BBD2
:1025000001F0B6FE00288ED01E2E8CD80022304658
:10251000114602F02BFBBDE8F84001F04BBEBDE8D0
:10252000F84001F0C9BEBDE8F84001F017BE01F067
:102530000FFEE8BB01F0C0FEBDE8F840002002F04D
:1025400093BA01F005FE78B972B602F0E1FD02F02F
:102550002DFEFEF7DBF9304601F0F4FD3146E120B7
:10256000FFF756FE62B6F8BD3146E120BDE8F840FF
:10257000FFF74EBEFEF70CFA01F092FE02F0DCF817
:10258000002001F0DFFDBBE7FEF702FA01F088FE54
:1025900002F0D2F8002001F0D5FDA5E7FEF7F8F92A
:1025A00001F07EFE02F0C8F8002001F0CBFD92E7BA
:1025B000FEF7EEF901F074FE02F0BEF8002001F023
:1025C000C1FDB7E788BC0020A4B001200070064020
:1025D000A2B00120641C00204800002070B53B4CD4
:1025E0002378012B3A4B66D0DA78D006D1B21CD4CE
:1025F0009B794A06DBB21DD413F0500F35D1354814
:10260000334B0178344C4A1CD2B202701A796254AE
:102610009A7942F050029A719A79022142F050025E
:102620009A71D970BFF34F8F70BD10224906DA70CE
:1026300044D59B792749264B274800220A709A796E
:10264000C02542F020029A719D700A781979815450
:10265000032222709A79422142F050029A71D97075
:102660009B79DBB213F0500FC9D0194B1B489A79F4
:10267000194942F050029A719E7900F5204506F002
:10268000DF062A889E71C8269E700226DE70531CC3
:1026900002EB820200EB42000A222B8009F099FA39
:1026A0002B880D48C3F30B03202200212B8009F057
:1026B00092FA267070BD0222DA70B3E79A7902218D
:1026C00042F050029A71D97070BD00BFA4B00120D1
:1026D00000700640A3B0012068BC0020641C0020EC
:1026E000064B0438C0B203EB8000D0F81402013866
:1026F00002288CBF00200120704700BF1CA60120CB
:10270000064B0438C0B203EB8000D0F81402043842
:1027100001288CBF00200120704700BF1CA60120AB
:10272000074B0438C0B203EB8000D0F8140220F04D
:102730000400A0F10300B0FA80F04009704700BF28
:102740001CA60120034B0438C0B203EB8000D0F874
:10275000140270471CA6012004380B4BC0B2843011
:1027600003EB80004368012B0BD0032B06D0022B18
:102770000CBF07234FF0FF334360704706234360CD
:1027800070470023436070471CA6012004380B4BA0
:10279000C0B2843003EB8000436813B90123436067
:1027A0007047072B06D0062B0CBF02234FF0FF33D8
:1027B0004360704703234360704700BF1CA601209D
:1027C000043838B5C0B2164B00F1840403EB84041E
:1027D00000F588716268013A0125022A43F8215008
:1027E00003D94FF0FF33636038BD0E4D00EB80110D
:1027F00000EB400205EBC10500F58670002103EBFC
:102800008202C2E90D11C5F8F81143F8201001F059
:1028100029FD10B10423636038BD0523636038BD12
:102820001CA60120901000200438094BC0B284304F
:1028300003EB80004368052B06D0042B0CBF052357
:102840004FF0FF334360704707234360704700BF7A
:102850001CA6012004380C4BC0B2843003EB80026C
:102860005268511F012909D9023A022A03EB80005C
:1028700034BF07224FF0FF324260704703EB800005
:1028800007224260704700BF1CA601200438074B96
:10289000C0B2843003EB8000436823F00403032BB1
:1028A0000CBF06234FF0FF33436070471CA6012086
:1028B0000438104BC0B270B400F1840403EB8402FE
:1028C00000EB4001556800F58870012643F8206050
:1028D00003EB810125F002000022B0424A6303D0DD
:1028E000AA1E18BF4FF0FF3203EB840370BC5A607E
:1028F000704700BF1CA60120F8B5344E00EB8013D2
:1029000006EBC30505F5F87ED5F8F82102EB430385
:1029100006EB830484ED000AC4ED290A84ED521A03
:102920008401E9B10123A2F12001C2F1200C03FAD4
:1029300001F123FA0CFC41EA0C0CD5E97C7104444A
:10294000934006EBC40401323B4341EA0C01C5F855
:10295000F821C5E97C31D4F8F831292B1ED0F8BD17
:102960000127A2F12003C2F1200C07FA03F327FA92
:102970000CFC43EA0C0CD5E97C130444974006EBAD
:10298000C404013223EA0C0321EA0707C5F8F82141
:10299000C5E97C73D4F8F831292BE0D1C5B20C48D5
:1029A00005EB851306EBC30100EBC3004FF4027285
:1029B00009F00FF9284600F081F800230022C4E94D
:1029C0007C230023C4F8F831F8BD00BF901000202C
:1029D000700800202DE9F84F244F254D00F586782A
:1029E00000EB801457F8286006EB440E05EB8E09C7
:1029F00005EBC404D9F800A0D4E97CB9C1F800A063
:102A000005EB8E0A2BFA06F1DAF8A4B0C2F800B092
:102A1000C6F1200A09FA0AFAA6F1200229FA02F2FE
:102A200041EA0A0105EB8E0C1143002501F0010A71
:102A3000AB46DCF8481119605AEA0B020A9B4FF6C4
:102A4000FF7206F1010608BF2A4647F828601A609F
:102A5000D4F8F83157F828209A4201D2BDE8F88F0F
:102A600000F01CF847F82850BDE8F88F1CA601209C
:102A70005000002008B501210A20FEF733F9022199
:102A80002F20FEF72FF9FEF7E3FA72B6FEE700BF3C
:102A9000014B01221A707047A6B00120034A01239E
:102AA000117883400B43DBB213707047A5B001204F
:102AB000014B01221A707047A9B00120034A01237B
:102AC000117883400B43DBB213707047A7B001202D
:102AD000014B01221A707047A8B0012008B5094BBC
:102AE0000949186801231A4604F004FF38B9BDE803
:102AF0000840054905484FF4007209F06AB8FFF72D
:102B0000B9FF00BF04000020905C01201CA601203A
:102B100030B583B000230193019B1E2B11DC0B4DBC
:102B20000B4C0199019A206805EB412102320123E7
:102B300004F0E0FE38B9019B01330193019B1E2B89
:102B4000EFDD03B030BDFFF795FF00BF2463012028
:102B5000040000202DE9F04F764BDFF8E48185B0CA
:102B60000446414618680022012304F0C3FE0028F1
:102B700040F0DD80704BD8F800209A4202D1002C42
:102B800000F0B0806D4C002740F2544200212046F6
:102B900009F021F80197019AE76001230221032A35
:102BA000C4E90477C4E90033A161E761C4F828747B
:102BB000C4F82C74A3601EDC9C460199019A019D07
:102BC000019B0198019E01360196019E01EB410196
:102BD00002EB420203EB430304EB810104EB8202AC
:102BE00004EB830308306D01032E44F820C04F63CB
:102BF00097631D63E1DD4F485049006801231A4681
:102C000004F044FF002840F092800290029B1E2BAB
:102C100049DCDFF8309105464FF0030B029A03952B
:102C2000039BC4F80C52032BC4E9815BC4F8105217
:102C3000C4F8002227DC039F0399039A039E02989D
:102C4000039BDDF80CA00AF1010ACDF80CA004EBFF
:102C5000870C01EB4101039FCCF8145202EB4202B6
:102C600003EB430304EB810104EB8202013004EB2C
:102C7000830300EB4610032FC1F82852C2F82C52F0
:102C8000C3F82402D7DD2B4B029A186802320123C5
:102C9000494604F0FBFE002849D1029B0133029310
:102CA000029B1E2BBADD4FF4007200212448224CF7
:102CB00008F091FF1F4B22491868C8F8004042F203
:102CC0004E220725C8F8082001230022C8F8045026
:102CD00004F0DCFE58BBD8F80030A34202D005B0A7
:102CE000BDE8F08FD8F8084042F24E239C42F6D05F
:102CF00004F00F030E2B08BF24110121C4F30310AD
:102D0000FDF7F0FF04F00F000221FDF7EBFFFEF7E7
:102D10009FF90123ADF80230BDF802309BB25A1C76
:102D200092B2ADF80220002BF6D172B6FEE7FFF7A3
:102D3000A1FE00BF040000204B45454E1CA601200B
:102D400024A101201CA801202DE9F84F834D2B78E8
:102D5000002B77D1824D2B78002B40F09980814C4D
:102D60002378002B40F0BA807F4E337873B37F4DC9
:102D7000DFF810A2DFF81092DFF8FC817C4F00240E
:102D80003378E340DA071AD56B6B4B4500F2BC8011
:102D90002A6BD8F8000057F8222003F1010C1A44DE
:102DA00051460123C5F834C004F070FE002840F0FD
:102DB000D28033780122A24023EA02033370013427
:102DC000042C05F10C050AF5027AD9D1694E337845
:102DD00083B1664DDFF8A091DFF8B08105F5886B0F
:102DE00000243378E340DB0706D40134042C05F1DA
:102DF0000C05F6D1BDE8F88F5BF82430D9F8000057
:102E000004EB841108EBC101002B00F08B80D5E9A5
:102E10000C7CAA6B564B02F1010E53F827A0BEFBA7
:102E2000FCF30CFB13E35244AB63012304F062FD9B
:102E3000002840F0908033780122A24023EA020368
:102E40003370D2E7494C4C4BD4F814241868023242
:102E500004F50071012304F04DFD00287BD101F041
:102E6000E9F910B1D4F80032E3613E4C00230126A9
:102E70002B703B4D267001F013FA01F05DFC01F060
:102E800081FD3046FEF770F82B78002B3FF467AFDA
:102E90004FF400720021394808F09DFE3849374848
:102EA0004FF4007208F095FE304A334BD2F80022FE
:102EB000186832490232012304F0E8FD0646002872
:102EC00049D1284C0127277001F05CFD3846FEF7F8
:102ED0004BF82E702378002B3FF446AF4FF400726E
:102EE0000021264808F077FE204924484FF400725C
:102EF00008F06FFE204B2149186801231A4604F0A0
:102F0000C5FD40BB20702FE704F1040B5FFA8BFB7B
:102F10005846FFF7F5FBD0B95846FFF7F1FB90B9DB
:102F20006B6B35E7D5E9897CD5F82C22104B02F183
:102F3000010E53F827A0BEFBFCF30CFB13E3524435
:102F4000C5F82C3271E75846FFF76EFCE8E75846A3
:102F5000FFF76AFCE0E7FFF78DFD00BFA6B0012098
:102F6000A9B00120A8B00120A7B001201CA6012013
:102F7000A8C20000A5B0012004000020905E01203E
:102F80001CA80120700800205F5B03005000002097
:102F900070B51248124C134A134E144D14490023B5
:102FA00033702B702370037013700A68114C22F079
:102FB00001020A6020681946052208F0CFFB20684C
:102FC00005F0ACF940B9206804F002FF20B9206890
:102FD00004F080FC00B970BDFFF74CFDA9B00120E2
:102FE000A5B00120A6B00120A8B00120A7B0012003
:102FF00000D000400400002004207146084202D0A6
:10300000EFF3098001E0EFF3088081690A884BF64D
:10301000AB639A4200D0FEE702318161202101605A
:10302000704700BF80B586B000AF78600846114693
:103030001A460346FB700B46BB7013467B70002399
:103040003B613B6943F004033B61FB783B73BB7816
:103050007B737B7800221946786806F0F7FD012320
:10306000FB7503E000BFFB7D0133FB75FB7D002B8F
:10307000F8D107F10C013B690222786806F0B0FF35
:103080000123BB7503E000BFBB7D0133BB75BB7D76
:10309000002BF8D1786806F081FF00BF1837BD46D5
:1030A00080BD00BF80B586B000AF78600B46FB7076
:1030B0001346BB700023FB7300233B613B6943F065
:1030C00004033B61BB7800221946786806F0BEFD18
:1030D0000123FB7503E000BFFB7D0133FB75FB7D26
:1030E000002BF8D1F91C3B690122786806F078FFC3
:1030F0000123BB7503E000BFBB7D0133BB75BB7D06
:10310000002BF8D1BB7801221946786806F0C6FD7D
:1031100001237B7503E000BF7B7D01337B757B7DE5
:10312000002BF8D107F10F013B690122786806F006
:10313000A1FF01233B7503E000BF3B7D01333B75DD
:103140003B7D002BF8D1786806F028FFFB7B184602
:103150001837BD4680BD00BF2DE97043064689463D
:1031600090461D46412421462B464A463046FFF7ED
:1031700059FF611C0234C9B22B4642463046E4B2C4
:10318000FFF750FF592CEED1BDE870830B4609497B
:10319000094A31F8131010B4084C117103EB4303C2
:1031A00004EBC30301465DF8044B0548136107F0C7
:1031B0000FB800BF080000204CA4012064A4012027
:1031C000006006400B460949094A31F8131010B453
:1031D000084C117103EB430304EBC30301465DF894
:1031E000044B0548136106F0F3BF00BF0800002040
:1031F000ECA4012004A5012000600E402DE97841D7
:10320000DAB92E492E4D0B782E4C2F480133DBB204
:103210000B700B78042B08BF0A700B782B4A2C49D3
:10322000DBB203EB430635F81330137104EBC6042D
:103230001461BDE8784106F0CBBF244C24492248F4
:103240001F4E204DDFF8748007F03AF82822002145
:103250001F4808F0C0FC20461822002108F0BBFCE3
:10326000B6F800C084F804C04FF0180C2561C4F80B
:1032700014C04FF0040C0023C4F808C0154A1449C8
:10328000114823604FF0010C88F8003084F805C025
:1032900084F80CC006F052FF98F800300C490A4838
:1032A000DBB203EB430236F81330237105EBC205A2
:1032B00025612246BDE8784106F08ABFABB0012007
:1032C0000800002064A40120006006404CA40120F6
:1032D000C4A40120FD3100002DE97841DAB92E495E
:1032E0002E4D0B782E4C2F480133DBB20B700B7830
:1032F000042B08BF0A700B782B4A2C49DBB203EB76
:10330000430635F81330137104EBC6041461BDE8AD
:10331000784106F05DBF244C244922481F4E204DC1
:10332000DFF8748006F0CCFF282200211F4808F047
:1033300052FC20461822002108F04DFCB6F800C0CF
:1033400084F804C04FF0180C2561C4F814C04FF085
:10335000040C0023C4F808C0154A1449114823601E
:103360004FF0010C88F8003084F805C084F80CC0D8
:1033700006F0E4FE98F800300C490A48DBB203EB93
:10338000430236F81330237105EBC205256122464E
:10339000BDE8784106F01CBFACB001200800002059
:1033A00004A5012000600E40ECA4012064A50120CA
:1033B000D9320000014B1868704700BF24A30120D8
:1033C0000149024806F0A2BCC4A4012000600640E6
:1033D0000149024806F09ABC64A5012000600E4035
:1033E00070B55B4E36F811300C46DBB2632280219B
:1033F0000546FFF717FE36F814202846D2B25D21A5
:10340000FFF750FE242801D0002070BD36F814309C
:1034100028460022DBB25E21FFF704FE36F81430A6
:1034200028460122DBB22B21FFF7FCFD36F81430D1
:1034300028460122DBB22C21FFF7F4FD36F81430C8
:1034400028460022DBB22D21FFF7ECFD36F81430C0
:1034500028460022DBB22E21FFF7E4FD36F81430B7
:1034600028460122DBB22F21FFF7DCFD36F81430AD
:1034700028460122DBB23021FFF7D4FD36F81430A4
:103480002846FF22DBB23121FFF7CCFD36F814309D
:1034900028460222DBB23221FFF7C4FD36F8143091
:1034A00028460022DBB23321FFF7BCFD36F814308A
:1034B00028460022DBB23421FFF7B4FD36F8143081
:1034C00028460022DBB23521FFF7ACFD36F8143078
:1034D00028460222DBB20F21FFF73EFE36F81430F9
:1034E00028463F22DBB25C21FFF79CFD36F8143002
:1034F00028462022DBB25D21FFF794FD36F8143018
:1035000028460B22DBB27B21FFF78CFD36F8143006
:103510002846C922DBB27D21FFF784FD36F814303E
:1035200028468322DBB27E21FFF77CFD36F814307B
:103530002846B522DBB27F21FFF774FD36F8143040
:103540002846DBB20C225E21FFF76CFD012070BD26
:1035500008000020084B094810B403F1100453F888
:10356000041B026891423CBF026843F8042CA3424A
:10357000F5D15DF8044B7047A4A50120B4A5012046
:1035800070B43A4EDFF8F8C006F12C040025A4F11F
:1035900030016346D87D9A7D42EA002241F8042F2B
:1035A000A142A3F10203F5D10C35242DACF1180C86
:1035B00001F13004EBD1DFF8CCC02D4CA4F1300187
:1035C0006346D87D9A7D42EA002241F8042FA14249
:1035D000A3F10203F5D10C35482DACF1180C01F123
:1035E0003004EBD1234A244B2449D4891088B1F804
:1035F0005C50C6F820415860B1F85A40B1F8580004
:10360000B1F85EC0B1F856609D601C61B1F85450CD
:10361000B1F852409861B1F85000C3F800C01E6282
:10362000B1F84EC0B1F84C609D621C63B1F84A50CD
:10363000B1F848409863918850889E641D659C65E8
:103640005961C3F840C0D860D088118956899589DE
:10365000148AD8615962508A918AD28ADE625D6387
:10366000DC63586470BCD9645A65704728A3012094
:10367000E4A3012064A40120B8A5012004A5012031
:1036800034A50120ACA4012080B582B000AF002396
:10369000FB711AE0FB79DBB219463F48FFF7A0FE49
:1036A0000346002B01D1002372E0FB79DBB21946FF
:1036B0003A48FFF795FE0346002B01D1002367E04F
:1036C000FB79DBB20133DBB2FB71FB79DBB2032B9D
:1036D000E0D928220021324808F07DFA2822002172
:1036E000304808F078FA182200212F4808F073FAC1
:1036F000182200212D4808F06EFA2D4B1B889BB232
:10370000DAB2294B1A71284B01225A71264B042236
:103710009A60254B01221A73234B264A1A61224BC9
:1037200018225A61204B00221A60214B1B889BB241
:10373000DAB21E4B1A711D4B01225A711B4B042227
:103740009A601A4B01221A73184B1B4A1A61174BC5
:1037500018225A61154B00221A600023174A10499B
:103760000D4806F0EBFC0023154A0E490B4806F005
:10377000E5FC144B1B78DBB219460948FFF706FD40
:10378000114B1B78DBB219460648FFF71BFD0123DE
:1037900018460837BD4680BD0060064000600E40F8
:1037A000C4A4012064A501204CA40120ECA40120A4
:1037B0000800002064A4012004A50120FD310000C0
:1037C000D9320000ABB00120ACB00120144B154938
:1037D000D3F81C01144A70B4144C154D00F00100CC
:1037E0004FF0040CC3F81C010226C4F808C00120E5
:1037F0001024AE608C60802688604FF40035202451
:103800004FF400408E60956094609060D3F818216A
:1038100022F00102C3F81821BFF34F8F70BC70472C
:103820000070034080F00F4000F00F40C0F00F40E8
:1038300040F00F402DE9704FCD4ACE4ED2F80C31FA
:1038400003F001032DED028BC2F80C3133688CB00C
:1038500003333360FFF794FE00F07AFC002840F059
:10386000C781DFF870834FF0FF338346C8F800301C
:103870000446201DC0B2FEF743FF002840F08083BD
:103880000134042CF5D1D8F80030DFF84C934FF018
:10389000FF329342C9F8002000F00E81B64DDFF8E8
:1038A0003CA300240023201D45F8043BC0B2FEF7D2
:1038B00037FFE3B210BB0134042CF3D13268AF49B7
:1038C000AF4801F0A5FED8F80030002B2ADAD9F86D
:1038D0000030002BC0F2FC80AA4B1B68002B40F389
:1038E000F780A94E06EB8303D3ED007AF5EEC07A9C
:1038F000F1EE10FA00F35083A44C33E0A44AA5493A
:103900001846A54B02EB84024FF0010C009203EB2A
:1039100084030AEB840201EB840145F804CCFFF731
:1039200059F8C8E79A4A984E52F82350974C00F03D
:103930006BFC9A4AD8F8003052F82010984A02EBF3
:1039400083028D4206EB8300D2ED000A90ED001A4F
:1039500004EB830292ED000A94BF00210121184676
:10396000FEF7CAFF94ED004AD4ED014A94ED025AE5
:10397000D4ED035A96ED006AD6ED016A96ED027A0F
:10398000D6ED037A9FED878A874DDFF83082DFF826
:10399000289224EE084A64EE884A25EE085A65EE1D
:1039A000885A26EE086A66EE886A27EE087A67EE7D
:1039B000887ABCEEC44AFCEEE44ABCEEC55AFCEE82
:1039C000E55ABCEEC66AFCEEE66ABCEEC77AFCEECF
:1039D000E77A85ED064AC5ED0C4A88ED0C5AC5ED2F
:1039E0000E5A85ED126AC8ED0E6A89ED047AC8EDAB
:1039F0000A7A01F0CFFDFDF757FA002309930A93E5
:103A00000B9300F053FC012800F02782022800F0FD
:103A1000AA81002800F0CC8100F004FC012800F00D
:103A2000E781022800F0F281002800F0FD815F4B61
:103A30005F4A0492012102224FF003085D4DDFF836
:103A400090A10293994603913346002411464646BD
:103A500003EB8402D2ED007AF5EEC07AF1EE10FAB3
:103A60005BDD95F80080B8F1000F62D0032C32D1F5
:103A70003F4D4D4CD5F818314F49504A444843F01A
:103A80000103C5F818314FF0FF33D4F89850C4F84B
:103A90009830D1F89840C1F89830D2F89810C2F810
:103AA00098300021102208F096F8BFF34F8F0CB029
:103AB000BDEC028BBDE8708F0446201DC0B2FEF73E
:103AC0000FFE002840F075820134042CF5D1E5E6A4
:103AD0002E4C2D4E46E7DFF80881DFF808C158F874
:103AE0002420374902925CF82420049251F82420C3
:103AF000344EDFF8F490DFF8F4E033480392334AB1
:103B000056F824B059F824105EF824A050F8246028
:103B100052F82490013501349AE7012202FA06F6A0
:103B2000002102FA0BF2CAF80860C9F808202970CF
:103B30009CE7CDE90613164B53F82420059200F0BC
:103B400063FB164B059A53F820008242DDE9061309
:103B500000F2ED80012202FA0BF00399C9F804008B
:103B6000029802FA01F141602A7085F804807DE72D
:103B70000070034024A301207CAA0120B8A50120E5
:103B800028A30120381A0020ACAB01208CAC012006
:103B9000A4A5012024AB0120ECAA012008C5000047
:103BA00034AD012000F07F450080034040F00F401D
:103BB000C0F00F4094A5012000A0034000900B40EE
:103BC000E4C40000D8C40000F0C40000A8C4000091
:103BD00080F00F4020000020140000205CAB01208A
:103BE000B4C40000CCC40000FCC40000C0C4000089
:103BF000C94ACA48CA4CCB49CB4DDFF87CE3002305
:103C000013614FF0FF3C0361A3619361136303638E
:103C100093639364836323618362D2F89830C2F81C
:103C200098C0D4F89820C4F898C0D0F89840BF4BFA
:103C3000C0F898C0042402204FF0100CCEF80840C1
:103C4000A8600124C1F808C080204FF4003C8C60BB
:103C50008860C3F808C020204FF4004C9860C3F877
:103C600008C04FF0080CC1F808C0B14AAC604FF072
:103C7000400CC1F808C04FF0806E88604FF0007CA7
:103C80004FF4006105204FF48044C2F808E0C2F808
:103C900008C09C60A960FDF707F93268A549A648ED
:103CA00001F0B6FCA54A1378591C5B0711707FF42C
:103CB000FCAEA34CA34DD4ED007A95ED007AA24E54
:103CC000DFF8B882F4EE477AF1EE10FA96ED007A5A
:103CD00006D1D8ED006AB4EE667AF1EE10FA17D08C
:103CE000DFED9A6A67EEA67A27EE267AFCEEE77A8F
:103CF000BCEEC77A17EE903A17EE101AE22041EAAE
:103D00000341FEF785FA226833682A60C8F800305C
:103D10008F4C904D22782B789A423FF4C6AE4FF0EC
:103D2000FF31E420FEF774FA2B782370BDE605938B
:103D30004FF00108049B08FA01F108FA06F6CAF8E8
:103D40000460596000F066FA059B40B108FA0BF276
:103D50000399C9F80420029A08FA01F1516001227E
:103D60002A702A7182E67C4B1B68002BFFF654AE4A
:103D7000754A04EB830402EB830206EB8303D4ED64
:103D8000006A92ED007AD3ED007A66EE886A27EE3B
:103D9000087A27EE888AFCEEE66ABCEEC77ABCEEAB
:103DA000C88AC5ED046A88ED047A89ED068A33E68F
:103DB0006A4A6B4BD2ED007A67EE887AFCEEE77ABE
:103DC000C5ED047AD3ED007A664B67EE887AFCEE97
:103DD000E77AC8ED047AD3ED007A27EE888ABCEE44
:103DE000C88A89ED068A00F01DFA01287FF419AE11
:103DF0004C4B4F494D4A0820402498609C604FF03E
:103E000080604FF480438860936010E6464B454ADB
:103E1000474901202024986094604FF000704FF4CF
:103E2000006288609A6002E63E4B3F4A40493F4844
:103E300008249C600124946040249C6020249C60A1
:103E40004FF080644FF000738C608B604FF48044BF
:103E50004FF4006384609360E9E5434B4349444A6F
:103E600003F13800F3EC017A9DED097AF2EC016A76
:103E7000F5EEC07AF1EE10FAD8BFF1EE677A37EEC0
:103E8000277AF5EEC06A8DED097ADDED0A7AB1EC9C
:103E9000017AF1EE10FAD8BFF1EE666A77EEA67AF3
:103EA000CDED0A7ADDED0B7AB4EEE77AF1EE10FA99
:103EB000C8BF8DED0B7A9842D4D1DDED0B7AB7EE09
:103EC000007AF4EEC77AF1EE10FA62D5F5EEC07A18
:103ED000F1EE10FA6ADDCDED0B7A9DED097ADFED9A
:103EE000256A0D490D4A0E4B27EE267ABCEEC77A9D
:103EF00081ED047A9DED0A7A27EE267ABCEEC77A28
:103F000082ED047ADDED0B7A67EEA67AFCEEE77AB5
:103F1000C3ED067A80E500BF0080034000900B40AF
:103F200000A0034080F00F4040F00F4000F00F4031
:103F300000F10F40B8A5012028A30120AAB001205C
:103F40008CAC01208CA5012034AD012000FEFF4681
:103F5000ADB0012048000020381A0020A8AB012095
:103F600098AB0120A0AB01201CAC0120E4AB0120E8
:103F700054AC012000F07F45C0F00F4090A5012017
:103F8000DFF83C90C8F800404FF0FF33C9F800302C
:103F900084E4F0EE477A9EE700F0F2F8D9F80000EA
:103FA000054C0430C0B2FEF70BFCDBE4DFED037A16
:103FB00091E7C9F8004071E48CAC012000000000DA
:103FC0001400002010B55E4C94F85034032B05D13A
:103FD000D4F81C0410F0FF0002D110BD002010BD69
:103FE00094F850340A2B00F2A880DFE803F05A4D11
:103FF0003F726C82332A1E12060032200121FCF728
:1040000071FE60691030C0B20221FCF76BFE012026
:1040100010BD01211520FCF765FE20690130C0B2FA
:104020000221FCF75FFE012010BD01211F20FCF7DB
:1040300059FEE0682030C0B20221FCF753FE012097
:1040400010BD01210F20FCF74DFE2368032B5CD827
:104050002068D7E701212420FCF744FE6068253062
:10406000C0B20221FCF73EFE012010BD012120203C
:10407000FCF738FED4F80402C0F12E00C0B20221D1
:10408000FCF730FE012010BD01212820FCF72AFE9C
:10409000D4F808022930C0B20221FCF723FE012027
:1040A00010BD01210C20FCF71DFED4F80C32CBB35F
:1040B000D4F80C42012C4FF0020139D02220FCF739
:1040C00011FE012010BD31200121FCF70BFEA0697B
:1040D00098E701213020FCF705FED4F828340221AE
:1040E000CBB10846FCF7FEFD0023C4F828340120BC
:1040F00010BD01211620FCF7F5FDA0681730C0B2F5
:104100000221FCF7EFFD012010BD02212320FCF766
:10411000E9FD012010BD3420FCF7E4FD0120C4F8C6
:10412000280410BD02211D20FCF7DCFD012010BD7C
:104130001E20FCF7D7FD204610BD012010BD00BF9A
:104140001CA60120014BC3F82C0470471CA60120BB
:10415000014BD3F82C0470471CA60120064BD3F862
:10416000003413F0FF0F00D170470121034B0846C4
:104170001960FCF731BC00BF1CA6012014A6012069
:104180000B4BD3F8102442B9D3F8002412F0FF0FE0
:1041900004D00122C3F8102470477047D3F80404F8
:1041A00010F0FF00F5D10121C3F81014FCF714BC86
:1041B0001CA6012038B5124C124A0025C4F8105430
:1041C000D4F80034156013F0FF0F0AD1D4F80414AA
:1041D00011F0FF0100D038BDBDE838400846FCF7BB
:1041E000FBBB29460120FCF7F7FBD4F80C3413F095
:1041F000FF0FF0D028460121BDE83840FCF7ECBBAA
:104200001CA6012014A60120014B1868C0B27047FB
:104210001CA60120024BD3F80402C0B2704700BFB5
:104220001CA60120024BD3F80802C0B2704700BFA1
:104230001CA60120024BD3F80004C0B2704700BF97
:104240001CA60120024BD3F80404C0B2704700BF83
:104250001CA60120024BD3F81C04C0B2704700BF5B
:104260001CA60120014BD868C0B270471CA60120D3
:10427000024BD3F80C04C0B2704700BF1CA601204B
:10428000024BD3F81004C0B2704700BF1CA6012037
:10429000024BD3F81404C0B2704700BF1CA6012023
:1042A000014BD3F8100270471CA60120014BD3F834
:1042B0000C0270471CA60120024B0122C3F8042403
:1042C000704700BF1CA601200B4B93F85024032A13
:1042D00010D0D3F82024B2FA82F25209C3F8202475
:1042E000D3F820341BB101210846FCF729BE012078
:1042F000FCF73ABE704700BF1CA6012010B5C94CA0
:104300000023C4F828341028D4F820343CD0EBB96A
:1043100094F85034032B00F0388194F85034002B7B
:104320007ED1022384F8503494F850340A2B00F2E2
:10433000DE80DFE813F0FE00F100DD00CD00C100FB
:10434000B500A9009F0093008700EB0094F850345B
:104350000A2BE9D801A252F823F000BF354600002D
:104360004B460000614600002943000069460000FA
:104370007F460000F945000009460000194600008C
:104380001F460000E94500006BBB94F85034022B37
:1043900040F2088194F850340133DBB284F8503491
:1043A00094F85034062B05D194F850340133DBB225
:1043B00084F85034D4F80034002B00F0CF80236907
:1043C000002B40F0CB8094F85024974BD2B2A3FB43
:1043D0000213DB0803EB830103EB4103D31ADBB2C7
:1043E00084F85034C8E094F850340A2B9CD801A2C9
:1043F00052F823F015470000FF460000F746000082
:1044000029430000E9460000DB460000CB460000DF
:10441000BB460000B5460000AF4600009F460000C6
:1044200094F85034013BDBB284F8503494F85034A3
:10443000062B7FF479AF94F85034013BDBB284F85B
:10444000503471E701211520FCF74CFC2069013044
:10445000BDE81040C0B20221FCF744BC01211F207E
:10446000FCF740FCE0682030BDE81040C0B20221FB
:10447000FCF738BC01210F20FCF734FC2368032B28
:1044800000F2AC8020681CE001212420FCF72AFC0B
:1044900060682530BDE81040C0B20221FCF722BCA4
:1044A00001211620FCF71EFCA0681730BDE8104063
:1044B000C0B20221FCF716BC31200121FCF712FC2E
:1044C000A0691030BDE81040C0B20221FCF70ABC60
:1044D00001213020FCF706FCD4F828340221002BFF
:1044E00075D00846FCF7FEFB0023C4F8283410BD45
:1044F00001212020FCF7F6FBD4F80402C0F12E00C5
:10450000BDE81040C0B20221FCF7ECBB3220012113
:10451000FCF7E8FB6069D4E701212820FCF7E2FB07
:10452000D4F808022930BDE81040C0B20221FCF7DF
:10453000D9BB01210C20FCF7D5FBD4F80C32002BA1
:1045400000F0F380D4F80C32012B4FF0020100F0A0
:10455000A180BDE810402220FCF7C4BB94F8503481
:10456000324ADBB2A2FB0312D20802EB8202A3EBB7
:104570004203DBB284F8503494F85034022B3FF6F7
:10458000D3AE032384F85034CEE6D4F800342BB1F4
:1045900023691BB90A2384F85034C5E6092384F83B
:1045A0005034C1E694F8502421490132D2B284F843
:1045B000502494F85034DBB2A1FB031202F0FE0148
:1045C00001EB52029B1ADBB284F85034ACE6342083
:1045D000FCF788FB0123C4F8283410BDBDE8104067
:1045E00002212320FCF77EBB6369032B3FF69CAEC0
:1045F00063690133636197E66368002B3FF494AE0F
:104600006368013B63608FE62368032B3FF68CAE43
:1046100023680133236087E60023E36084E60023F8
:10462000236181E61CA60120A38B2EBACDCCCCCC75
:10463000ABAAAAAAD4F80C32002B3FF475AED4F87A
:104640000C32013BC4F80C326EE6D4F80832002B71
:104650003FF46AAED4F80832013BC4F8083263E68E
:104660000023C4F804325FE6A369032B02D8A369D0
:104670000133A361A069C0B200F07EFD54E6A368D7
:10468000032B02D8A3680133A360A068C0B200F076
:1046900069FD49E6BDE810401E20FCF723BB6369B5
:1046A000002B3FF441AE6369013B63613CE60123AB
:1046B000236139E60123E36036E62368002B3FF4EB
:1046C00033AE2368013B23602EE66368012B3FF67F
:1046D0002BAE63680133636026E6A368002BD4D059
:1046E000A368013BA360D0E7A369002BC2D0A369F4
:1046F000013BA361BEE70123C4F8043214E6D4F8F9
:104700000832022B3FF610AED4F808320133C4F859
:10471000083209E6D4F80C32022B3FF405AED4F887
:104720000C320133C4F80C32FEE5BDE81040022122
:104730001D20FCF7D7BA00BF38B5104DC5F81002E0
:1047400070B9044602210420FCF746F921460320F3
:10475000FCF742F9D5F81002BDE8384000F0D8BCAB
:1047600000210420FCF738F903200221FCF734F97A
:10477000D5F81002BDE8384000F0CABC1CA60120E4
:10478000012810B57E4C18D0022836D0C8B10020C0
:10479000FCF7EAFBD4F81C341BB1BDE81040FEF76F
:1047A00097B900F0EFF8BDE81040FEF791B994F822
:1047B0005034022BEBD80029E9D00023C4F81C3474
:1047C000E5E7C4F8280494F8503411BB022B02D852
:1047D000042384F8503400230122C4F81C24C4F8B4
:1047E000203494F850340A2BD1D8DFE803F09F939B
:1047F00086766B6055473C3126000023C4F8283488
:10480000D4F81C3453B9A9B194F85024022AE2D93F
:10481000DFE7022BDFD984F85004DCE794F850344A
:10482000022BC4D9002940F09380C4F81C1494F8DA
:104830005034ACE794F85034C8E701213220FCF73B
:1048400051FA60691030C0B20221FCF74BFA9EE7C2
:1048500001211520FCF746FA20690130C0B202217F
:10486000FCF740FA93E701211F20FCF73BFAE068D0
:104870002030C0B20221FCF735FA88E701210F2071
:10488000FCF730FA2368032B68D820681030C0B2D8
:104890000221FCF727FA7AE701212420FCF722FA0B
:1048A00060682530C0B20221FCF71CFA6FE70121D5
:1048B0001620FCF717FAA0681730C0B20221FCF7E7
:1048C00011FA64E701213120FCF70CFAA0691030DD
:1048D000C0B20221FCF706FA59E701213020FCF7AB
:1048E00001FAD4F828340221002B3CD00846FCF70A
:1048F000F9F90023C4F8283449E701212020FCF706
:10490000F1F9D4F80402C0F12E00C0B20221FCF784
:10491000E9F93CE701212820FCF7E4F9D4F8080282
:104920002930C0B20221FCF7DDF930E701210C206B
:10493000FCF7D8F9D4F80C32E3B1D4F80C32012BDF
:104940004FF002010CBF1E202220FCF7CBF91EE71E
:1049500094F85034022B7FF630AF18E70221232061
:10496000FCF7C0F913E73420FCF7BCF90123C4F8C5
:1049700028340CE702211D20FCF7B4F907E700BF3B
:104980001CA6012038B5244CD4F81C3413F0FF0FBA
:1049900035D1D4F81404D4F81454D4F800221D2AC4
:1049A00024D81E4A0130A2FB0030C0F3C700012109
:1049B000D0B1FCF797F919486B1CA0FB0320C00885
:1049C00000EB8000A3EB4000C0B20221FCF78AF9A3
:1049D000D4F80022D4F814349A4204D0D4F80C3419
:1049E00013F0FF0F11D138BD0A20E2E701210A20A0
:1049F000FCF778F902210A20FCF774F9E8E7BDE832
:104A0000384000210120FFF7BBBE0021BDE838403F
:104A10000846FCF795BA00BF1CA60120CDCCCCCC33
:104A200008B5104B1028D3F8142411D052B91D2208
:104A3000C3F81424FFF7A6FFBDE8084001210020B9
:104A4000FCF77EBAD3F81424013AC3F81424F1E732
:104A50001C2A96BFD3F8142400220132C3F8142470
:104A6000E8E700BF1CA60120012810B522D00228CB
:104A7000164C10D048B1D4F81C3413F0FF0F00D0FE
:104A800010BDBDE81040FFF77DBF0121C4F80C1434
:104A9000FBF7A2FFEFE7D4F80C34B3FA83F35B091A
:104AA000C4F80C34D4F80C1461B101210020FBF7D8
:104AB00093FFE0E70021054C0846C4F80C14FBF70F
:104AC0008BFFD8E70846FBF787FFD4E71CA6012039
:104AD000234BD3F8002412F0FF0F21D0D3F8242465
:104AE00010B5F2B90124FF211720C3F82444FDF7C3
:104AF0008FFB2046FFF7B8FF02210846FBF76CFF4B
:104B0000184B1949D3F8382122F00102C3F8382193
:104B1000C3F83011D3F838212243C3F8382110BD2F
:104B20007047FF2100241620C3F82444FDF770FBD2
:104B30002046FFF799FF01210220FBF74DFF094BAB
:104B40000949D3F8382122F00102C3F83821C3F80B
:104B50003011D3F8382142F00102C3F8382110BDDA
:104B60001CA6012000700340FD4395082DE9F04F7D
:104B7000A54CD4F80C3485B01A4312F0FF0F8046D0
:104B800001910DD1D4F8003413F0FF0F03D0019B35
:104B9000002B40F0348105B0BDE8F04FFFF70ABBB1
:104BA0009A4E002506EB4026AA4604F5097705F142
:104BB000040B5FFA8BFB584605F58879FDF790FDED
:104BC000002840F008815846FDF79AFD002840F083
:104BD000F58054F82930002B40F0E380D4F80032FF
:104BE0004345394630464FF00C0201D006F0F1FF44
:104BF0000135042D44F829A007F10C0706F10C0635
:104C0000D5D1DFF80C920125A9F5785B2A466FF023
:104C10001F0E6FF03F0C00230DE01F2B29D8206AD8
:104C200002FA03F1014321620135EDB201330CF1C7
:104C3000010C0EF1010E5E460020A6F130014F6A14
:104C40009F4203D18F6A002F18BF01200C31B1425F
:104C5000F5D101F500764E45EFD1D9B20028DCD16F
:104C60001F2B0ED8216A02FA03F021EA000121620B
:104C7000DAE73F290ED8606A02FA0EF10143616259
:104C8000D2E73F2969D8616A02FA0EF021EA0001F1
:104C90006162C9E75F2946D9E06AA3F1600102FABF
:104CA00001F10143E1622906BED500210846212613
:104CB000012501EB410204EB82028DF80F005063E5
:104CC00090639DF80F301F2B17D8002707F10803BA
:104CD00054F823309DF80FC023FA0CF3DB0728D5D6
:104CE0000137042FF2D19DF80F300133DBB28DF87C
:104CF0000F309DF80F301F2BE7D901310429D8D18F
:104D0000C4F80082C4F81484D4F8003413F0FF0F00
:104D100002D0019B002B6BD1FDF7CAFE05B0BDE8A8
:104D2000F04FFFF747BAA06A02FA0CF10143A16203
:104D30007AE79DF80F3003EB471313639DF80F30AC
:104D400003EB4713DBB21F2B19D8276A05FA03F3CD
:104D50003B4323628DF80F60C5E75F2908D9E16AFC
:104D6000A3F1600002FA00F021EA0001E1629AE793
:104D7000A16A02FA0CF021EA0001A16254E73F2B7C
:104D800006D8676A203B05FA03F33B436362E1E719
:104D90005F2B24D8A76A403B05FA03F33B43A36289
:104DA000D8E7A7F5FA710C223846009106F011FFFA
:104DB00000990C22304606F00CFF19E75846FDF723
:104DC00033FD5846FDF79CFC00283FF402AF5846DF
:104DD000FDF72AFDFDE65846FDF7BEFCF3E61F068B
:104DE000B8D4E76A603B05FA03F33B43E362B1E7FB
:104DF00041460220FDF70CFAFDF75AFE8EE7014608
:104E00000220FDF705FAC6E61CA601204863012032
:104E100054A10120F8B5194DD5F81C3413F0FF0F3B
:104E200006460F4614461CD1C5F81464D5F80C2468
:104E3000134B144314F0FF0F4FF000021A600BD114
:104E4000FFF7A0FD0120FCF78FF8D5F8003413F030
:104E5000FF0F00D057B9F8BDFFF7ACF9FDF718FE0A
:104E6000F3E700210120FFF78BFCDDE7314601204D
:104E7000FDF7CEF9C5F81864F8BD00BF1CA60120E7
:104E800014A6012010B52D4C2D4840F254420021AB
:104E900006F0A1FE2B4A2046002103F027FD2748FB
:104EA000002103F03FFD0306F9D52369244C40F6A9
:104EB000B832934294BF00230123C4F80034FDF7B5
:104EC0000DFEA068C0B200F04DF9A069C0B200F0BC
:104ED00053F9FDF71DFED4F8001411F0FF0122D0A4
:104EE0002369E3B90123C4F80834626916481749F5
:104EF000174B00FB0212C3F83021D3F8382142F0DF
:104F00000102C3F83821E369C4F81434D4F8140456
:104F10000122BDE81040C0B20021FFF77BBF002096
:104F2000FFF7A2FDEFE71E23C4F81434D4F81404ED
:104F30000122BDE81040C0B2FFF76CBF00B00B40CB
:104F40001CA6012040000020FF1AB700FF6BDC0206
:104F50000070034070B51F481F4D04F059FD044612
:104F6000FEF728FA2B68C01AC82808D91B4ED6F8B5
:104F7000003413F0FF0F09D1FEF71CFA2860154822
:104F8000214604F073FDBFF34F8F70BD62060DD450
:104F9000A307F1D5D6F80032D3B1D6F80002013814
:104FA000C0B200220121FFF735FFE5E7D6F8000285
:104FB0000B4B0130A3FB002323F00F02A2EB1313D2
:104FC000A0EB4300C0B200220121FFF723FFDFE77F
:104FD0001D20E6E7C0F00F4018A601201CA6012006
:104FE00089888888174BD3F83C2102F0010210B55C
:104FF000C3F83C21D3F83821134C22F00102C3F846
:105000003821D4F8081439B90220C4F82414FBF765
:10501000E3FCBFF34F8F10BDFF211420FDF7F8F81C
:10502000FF211620FDF7F4F8D4F814140120FDF741
:10503000EFF80020FFF718FD0023C4F80834BFF391
:105040004F8F10BD007003401CA601202A4BDFEDDE
:105050002B7A93ED007A20EE070AB4EEE70AF1EE20
:1050600010FA16D520EE000AF1EE047A20EE270A97
:10507000234B1B68032B03D8DFE803F03237290AE0
:10508000B0EE407A90EE007AFEEE007AA7EE270AA4
:105090007047DFED1C7AB4EEE70AF1EE10FA04D5A2
:1050A000DFED197A30EE670AE2E7F0EE007AB4EE4F
:1050B000E70AF1EE10FA1BD5B6EE007AFFEE007AA1
:1050C000E0EE077AB7EE000AA7EEE70AD0E7B0EE07
:1050D000407A90EE007ADFED0D7AA7EE270A70474E
:1050E00060EE007A20EE270A704720EE000A704733
:1050F000B7EE000ABCE700BF18000020CDCCCC3DC5
:105100001C0000202DF9E43ECDCC4C3D9A99193F6E
:10511000114A1368834230B415D0104B10494FF038
:10512000FF344FF0FF35C3E90045C3E90245C3E949
:105130000445C3E90645C3E90845C3E90A45C3E98F
:105140000C4500230B60A0F10100B0FA80F040098B
:1051500030BC1060704700BF70AA0120381A0020D0
:1051600074AA01200428034BA8BF042020EAE070A1
:10517000186070471C0000200428A8BF042020EA03
:10518000E07007EE900ADFED066A9FED067A064BA7
:10519000F8EEE77AA7EEA67A83ED007A704700BFB3
:1051A000CDCC4C3ECDCC4C3F18000020DE4BDFED8B
:1051B000DF7ADF49DF4ADFF8B4C32DE9F04F4FF063
:1051C000FF384FF0FF39DC4DDC4CDD4EDFF8A0A39B
:1051D000DFF8A0E3DB4FDFF8A0B3C5ED007AC3E949
:1051E0000089C3E90289C3E90489C3E90689C3E9DF
:1051F0000889C3E90A89C3E90C89DFF88083C5ED12
:10520000017A0020C6E90000B060C4ED007AC4ED68
:10521000017AC1ED007AC1ED017AC2ED007ACBE9E5
:105220000000C94BCAED007ACAED017ACBF808003C
:10523000CAED027ACEED007ACEED017ACEED027A99
:10524000CCED007ACCED017ACCED027AC7ED007A94
:10525000C7ED017AC2ED017AC5ED027AC4ED027A9A
:10526000C1ED027AC2ED027AF060C5ED037AC4EDB9
:10527000037AC1ED037AC2ED037A3061C5ED047A99
:10528000C4ED047AC1ED047AC2ED047A7061C5ED13
:10529000057AC7ED027ACBF80C00CAED037ACEEDA1
:1052A000037ACCED037AC7ED037ACBF81000CAED90
:1052B000047ACEED047ACCED047AC7ED047ACBF80B
:1052C0001400CAED057ACEED057ACCED057AC7ED6E
:1052D000057AC4ED057AC1ED057AC2ED057AB061B3
:1052E000C5ED067AC4ED067AC1ED067AC2ED067AFE
:1052F000F061C5ED077AC4ED077AC1ED077AC2ED1A
:10530000077A3062C5ED087AC4ED087AC1ED087AF3
:10531000C2ED087ACBF81800CAED067ACEED067A0F
:10532000CCED067AC7ED067ACBF81C00CAED077AF9
:10533000CEED077ACCED077AC7ED077ACBF82000DF
:10534000CAED087ACEED087ACCED087AC7ED087A76
:10535000CBF824007062C5ED097AC4ED097AC1ED7D
:10536000097AC2ED097AB062C5ED0A7AC4ED0A7A0B
:10537000C1ED0A7AC2ED0A7AF062C5ED0B7AC4ED8E
:105380000B7AC1ED0B7AC2ED0B7A3063CAED097A64
:10539000CEED097ACCED097AC7ED097ACBF8280071
:1053A000CAED0A7ACEED0A7ACCED0A7AC7ED0A7A0E
:1053B000CBF82C00CAED0B7ACEED0B7ACCED0B7A44
:1053C000C7ED0B7ACBF83000CAED0C7ACEED0C7A33
:1053D000C5ED0C7AC4ED0C7AC1ED0C7AC2ED0C7AF5
:1053E0007063C5ED0D7AC4ED0D7AC1ED0D7AC2ED95
:1053F0000D7A564ECCED0C7AC7ED0C7ACBF8340012
:10540000CAED0D7ACEED0D7ACCED0D7AC7ED0D7AA1
:10541000C8F80000C8F80800C8F81000C8F818005C
:10542000C8F82000C8F82800C8F83000C8F83800CC
:10543000C8F84000C8F80400C8F80C00C8F8140008
:10544000C8F81C00C8F82400C8F82C00C8F83400BC
:10545000C8F83C00C8E91200C8E91400C8E9160001
:105460000446C8F844000146C8F8600003F590758A
:10547000324643E9044143E9024110339D4242F878
:10548000040BF6D1324F334BDFF8F480A6F8480016
:10549000C7E948004FF4FA71196099601961996180
:1054A0001962996219639963196499641965996518
:1054B0005960D9605961D9615962D9625963D96318
:1054C0005964D96459650C4686F84A000D46C7F8F8
:1054D0002801434608F59072E3E802459342FBD168
:1054E000DFF8A0A0DFF8A090DFF8A0E0DFF8A0C010
:1054F000194F1A4E1A4D1B4C1B484FF07C534FF05E
:10550000FF324FF4FA71CAF80030C9F80030CEF813
:105510000030CCF800303B6033602A6022600260CB
:10552000C8F82011BDE8F08F381A002000000000F4
:1055300054AC0120E4AB0120FCAC01201CAC0120E8
:105540007CAA0120C4AC0120801A002070AD01208B
:10555000701A0020D81900209CAB0120A0AB0120BC
:1055600020000020240000201400002034AD012081
:10557000ACAB01208CAC0120B4AA0120A01B002000
:10558000B018002094AB012098AB0120A4AB0120FF
:10559000A8AB0120194B1B68002BF0B425DB0422BB
:1055A0000E21174B174D1B68174F13445E1A01E06D
:1055B000914216DD99421846D8BFB01805EB800419
:1055C000D4ED007AF5EEC07AF1EE10FA03F10103A2
:1055D00002F10102ECD857F82040002CE8D1F0BCD1
:1055E00070474FF0FF30F0BC7047084B1B68002B32
:1055F000ABBF042200220E210421D2E720000020AC
:1056000074AA0120ACAB01207CAA01201400002068
:105610002DE9F04F494C2DED0A8B236895B0002BF6
:1056200001F0FB858C4646499FED46AADFED467AA0
:105630000C68934208BFB0EE67AA002C06DD013C5F
:105640000C601CB9414B4FF0FF321A60404B1B6895
:10565000002B00F05A843F4B08933F4B05933C4B83
:105660005B6823B9089B5B68002B41F04386384B8D
:105670009B6823B9089B9B68002B41F01D86344B27
:10568000DB6823B9089BDB68002B41F01086304BA8
:105690001B6923B9089B1B69002B41F003862C4B27
:1056A0005B6923B9089B5B69002B41F0F685284BA9
:1056B0009B6923B9089B9B69002B41F0E985244B2A
:1056C000DB6923B9089BDB69002B41F0DC85204BAB
:1056D0001B6A23B9089B1B6A002B41F0CF851C4B2A
:1056E0005B6A23B9089B5B6A002B41F0C285184BAB
:1056F0009B6A23B9089B9B6A002B41F0B585144B2C
:10570000DB6A23B9089BDB6A002B41F0A885104BAC
:105710001B6B23B9089B1B6B002B41F09B850C4B2B
:105720005B6B23B9089B5B6B002B41F08E85051FDB
:105730000A4C00F590762A4615E000BF78AA0120B1
:105740006CAD0120ABAAA643FFFFF944280000205E
:105750007CAA0120B4AA0120ACAB0120B018002023
:10576000B24201F05B8654F8043B52F8041F1E3B22
:105770009942F5DAB44AB54C02F592701746AE4636
:1057800057F8041F5EF8046FC1EB0113B1423344B4
:1057900006DA13F1080148BF03F117010911396056
:1057A0008742EDD1DFF804B3DA465E4652F8043F93
:1057B00055F8041F8242A3EB010346F8043FF5D1DC
:1057C000A34AACF104010F46154655F8040F57F8EB
:1057D000046FC0EB0013B042334406DA13F1080043
:1057E00048BF03F1170000112860A542EDD1994B85
:1057F0000D931D46184652F8043F51F8046FA2421B
:10580000A3EB060345F8043FF5D1934B002203F1C7
:1058100064010260026653F8042F22EAE2728B42AE
:105820001A60F8D103688B48044654F8042F02EB41
:10583000420213449B088C422360F6D1036E8749D1
:105840000D9851F8042D02EB420213449B0881424B
:105850000B60F6D1824B002203F59671CAF8002046
:10586000CAF8282153F8042F22EAE2728B421A6008
:10587000F8D1DAF80030DFF834A2504650F8042F9F
:1058800002EB420213449B0888420360F6D1DAF827
:105890002831744951F8042D02EB420213449B084D
:1058A00059450B60F6D170480022A0F1580353F817
:1058B000041F8A42B8BF0A468342F8D1A2F11E03F0
:1058C00009EE903ADFED697AF8EEE99A69EEA79A67
:1058D000F7EE007AF4EEE79AF1EE10FA41F1DA838E
:1058E000F5EEC09AF1EE10FA41F3AB84604B614AD9
:1058F0001B681093DAF808300B93DAF804300C9335
:10590000DAF820310A93DAF8243109935A4B0793D5
:105910009FED5A4A5A4BDFED5B4A9FED5B2ADFED64
:105920005B2A9FED5B3ADFED5B3ACDF848B0009221
:10593000D346069305924FF000089246BAEC016AEE
:10594000B5EEC06AF1EE10FA40F3E480524B53F822
:105950002830002B40F0DE80504800EB8800D0ED6E
:10596000006A76EE847A4FEA8801FDEEE77A17EE58
:10597000906A17EE902A012EB8BF0122492AA8BFCB
:105980004922012E40F33E84541E5BF822305BF81E
:1059900024509D4240F31B84531C5BF823309D42EE
:1059A00040F31584012C41F04E850C9D0B9A9542D5
:1059B00007DADBF80C500B9B032402269D4241F3CF
:1059C00088851D2D0ADD631E5BF82360AE4205DC71
:1059D000631C5BF82370AF4241F377834AED014AC1
:1059E0002F4A1099536B0193D36A0293136B03935D
:1059F000D2E9019E2B4B106819602B4B1469019959
:105A00000490D2E90765D068CDF804900F94D2E9EC
:105A100005C71190C3F80080D2E90940019BCDF879
:105A200038A0C24613969A456646A046DDF84CC09B
:105A300074468146AE460F9DCDF83CB0DDF844B0CB
:105A400000F0C88234E000BFAC180020301A0020FB
:105A5000D4190020A01B00209C1B0020001C00204B
:105A60006C1A0020981B0020F81B0020CDCC4C3E67
:105A700010000020ACAB01201CAC01200AD7A33BD6
:105A8000E4AB01200000000089D2DE3A4260E53B31
:105A9000CDCCCC3D0AD7A33C7CAA0120C4AC0120CC
:105AA000381A00206CAD012028000020701A002058
:105AB000049BBAEB030318BF4FF0FF33A24508BFA6
:105AC0000223DA4508BF0323AA4508BF0423B245D1
:105AD00008BF0523BA4508BF0623E24508BF0723D0
:105AE000F24508BF0823C24508BF0923CA4500F094
:105AF0002F830298824500F023830398824500F0AB
:105B0000B1828A4500F05E82581C40F00B82D0467C
:105B1000DDE90EAB08F10108B8F10E0F7FF40EAF0E
:105B2000944BDDF848B00193934B944D9FED94BA9C
:105B3000DFED948ADFED94AA9FED94CADFED94BA6D
:105B4000059F02930224CDF810B005E001344A2CE1
:105B500005F1040500F0E2806968212904F1FF36AF
:105B6000F4DD28688142F1DDD5F808904945EDDB88
:105B7000884B234413F8013C002BE7D10B184B440E
:105B800000EE103AB8EEC00AF3EE0E7A30EE670A75
:105B900020EE0B0AFFF75AFA07EE900AB8EEE77A02
:105BA00007EE901AF8EEE77A06EE909AB4EE677A6E
:105BB000F1EE10FAF8EEE66AB0EE409A05D1F4EE96
:105BC000667AF1EE10FA01F0598237EE267AB6EED7
:105BD000006AF0EE675AD7EE065AB0EE657A76EEB6
:105BE000C76AFFEE005A76EEE77A87EE878A68EE9C
:105BF000067AF4EEE57AF1EE10FA07DDB7EE007AF8
:105C0000F4EEC77AF1EE10FA01F157829FED628A45
:105C1000F5EEC07AF1EE10FA48BFB0EE6B8AB5EE41
:105C2000C09AF1EE10FA91DD009B5C4EDFF8A0A166
:105C3000B34603F138089946F9EC017AF5EEC07ADB
:105C4000F1EE10FA0EDDDAF800305BB99BED000AD8
:105C500030EE480A05F0B5FFB4EEE80AF1EE10FAAE
:105C60007FF674AFC8450AF1040A0BF1040BE3D1C7
:105C70004B4BD3F800E0BEF1000FC0F2AD8173468C
:105C80004FEA8E00474A4849D2ED007A474A92EDE2
:105C9000007A474A064486ED008A166B5663D66A38
:105CA0001663966AD662566A9662166A5662D66914
:105CB00016629669D6615669966116695661D6680C
:105CC00016619668D6605668966016681360019BE8
:105CD000566077EE877A01441A18B6EE007A079B71
:105CE00081ED008A029967EE877A3E1803440144E9
:105CF000BEF1000F86ED009AC2ED007AC3ED00AA56
:105D0000C1ED00AAC0F24282069B013418444A2C1D
:105D1000C0ED00AA05F104057FF41EAF154BDFF8B6
:105D20005890DFF8B0A0234F234DDDF810B0039357
:105D300019460193DFF8A0C020489FED213A9FED5E
:105D4000212A9FED214ADFED112A9FED0F6A1F4A9C
:105D5000DDF820800497099507974E46CDF8089006
:105D60000695D6460023F6EE003AF7EE004ACDF847
:105D700028A04BE034AD012054AC0120701A002063
:105D800089D2DE3A66660640000000000AD7A33CCE
:105D900058FF7FBF70AD012058FF7F3FC4AC01208A
:105DA00028000020A8AB0120FCAC0120A0AB012002
:105DB000381A00201CAC0120E4AB0120ACAB012060
:105DC0006666663FE6D0023FCDCCCC3D8CAC012070
:105DD0007CAA012078AA0120ECAA012087ED006AA4
:105DE00086ED006A85ED006A0433382B07F104075D
:105DF00006F1040605F1040502F1040201F10401B3
:105E000000F104000CF1040C00F040825EF8044F35
:105E1000002CE9D0D54CDCED007AD2ED006AD1ED52
:105E2000001A90ED005AC0ED007A04EB030AD04C42
:105E3000DAF800A0C2F800A01C4494ED007A58F8EB
:105E4000034081ED007A002CC8D0F5EEC07AF1EE67
:105E500010FA40F3FD8177EE666AD7ED005A66EEE0
:105E60008A6A66EE826AF4EEE46AF1EE10FA40F1B4
:105E70000282BFEE001AF4EEC16AF1EE10FAD8BF4A
:105E8000F0EE416A37EE617A76EEE56A27EE0A7A3D
:105E9000E6EE845A27EE237AD6ED006AC7ED005A63
:105EA000B4EEE47AF1EE10FA40F1EB81FFEE005A25
:105EB000B4EEE57AF1EE10FAD8BFB0EE657A77EE7F
:105EC000C57A37EE667A67EE8A7AE7EE046A67EE9D
:105ED000A27AF2EE045AF4EEE57AF1EE10FA95EDBC
:105EE000007AC6ED006A40F1C981F5EEC07AF1EEA4
:105EF00010FA01DCF0EE467A77EEC77AF5EE006A2A
:105F0000A7EEA67A85ED007A6EE79A4B08931B6898
:105F1000002B01F0D681984B05931A46002313609D
:105F2000FFF79DBB013302EB8304043C02EB8305C6
:105F300045EA0401490740F09880C3F10D010A29A0
:105F400040F29380D5E90001C3F10E067708012FD6
:105F5000C4E900011BD0D5E90201022FC4E9020106
:105F600015D0D5E90401032FC4E904010FD0D5E908
:105F70000601042FC4E9060109D0D5E90801062F5E
:105F8000C4E9080103D1D5E90A01C4E90A0126F0F0
:105F900001018E420B4404D0591E52F8233042F8BE
:105FA00021301368049353680193D2E90A93D2E92C
:105FB000024BD2E90456D2E9067CD2E908E8029302
:105FC000136B03934FF0FF3353631946019B9A45BC
:105FD0007FF46EAD012371E5684B1B68002BC0F2A6
:105FE0002A8101234FF00E0C04210393DFF898A1BE
:105FF000DAF800200A44A2EB0C0BA04602E08C4524
:1060000040F3B18094451346D8BF0BEB010307EB77
:106010008300D0ED007AF5EEC07AF1EE10FA02F1CD
:1060200001024FEA830001F10101E8D8544C54F811
:106030002340002CE3D1534A1268A14644465AB18A
:10604000039A002A41F0E6805A1C514201F00301F4
:1060500002F0030258BF4A42002BCAF80020FFF6A4
:1060600075AD0FE68A45ADD00D23591E52F82300B9
:1060700042F821000D2B03F1010192D052F82100CA
:1060800042F823000C2B03F102008AD052F8204082
:1060900042F821400B2B03F1030182D052F821403A
:1060A00042F820400A2B03F104003FF47AAF52F883
:1060B000204042F82140092B03F105013FF471AF64
:1060C00052F8214042F82040082B03F106003FF42B
:1060D00068AF52F8204042F82140072B03F1070136
:1060E0003FF45FAF52F8214042F82040062B03F105
:1060F00008003FF456AF52F8204042F82140052BEB
:1061000003F109013FF44DAF52F8214042F820401D
:10611000042B03F10A003FF444AF52F8204042F848
:106120002140032B03F10B013FF43BAF52F8213028
:1061300042F820300C297FF434AF536B136330E7FF
:10614000039B9A458ED08A453FF43CAF0C238CE7E5
:10615000029B9A45F4D0039B9A4583D08A453FF42D
:1061600031AF0B2381E74446F0E400BF24AB0120AC
:106170005CAB0120B4AA0120ACAB012020000020C0
:106180007CAA012070AA012074AA012069EE0A7A73
:10619000069B67EE8C7AF2EE046AF4EEE67A03442C
:1061A000F1EE10FA93ED007A4FD5F5EEC07AF1EEEC
:1061B00010FA01DCF0EE6A7A77EEC77AF5EE006A43
:1061C000A7EEA67A069B184480ED007ABEE4482E1E
:1061D00018DD0A9A099CA24229DDDBF828319A428F
:1061E0001BDD17464826741E5BF82450BD4241F360
:1061F0007481731C5BF82330AB42FFF6E2AB34468C
:1062000001F041B9561C5BF822505BF82670AF4292
:1062100040F34487492E41F03081DDE90923934260
:1062200005DD1A46DBF828319A4201F30680099D04
:106230004924FFF7C6BB144B1B68002BBFF6D1AE39
:10624000002103914FF0040CD0E6F0EE667AB3E73C
:10625000D7ED006A96ED007AD5ED007A66EE836A96
:1062600027EE037A67EEA37AC7ED006A86ED007A1F
:10627000C5ED007AB8E5F7EE006A03E6F0EE657A60
:106280003AE6B7EE007A1AE614000020DDF828A0FE
:10629000C948CA4ECA4DDFF87483DFEDCAAA9FED24
:1062A000CA9ADFEDCA8A9FEDCABA4B22002105F0D7
:1062B00092FC002400224FF07E53CDF83090DDF8A0
:1062C0001C903260CDE90AAB2B60A8F13807A246DA
:1062D000F7EC017AF5EEC07AF1EE10FA40F38D801A
:1062E000BC4B1B59002B40F0E781BB4BBB4A03EB77
:1062F000040B22449BED008A92ED007A77EE48BAB7
:10630000B0EE6B0A05F05DFC20EE090AF7EE007AAC
:10631000B4EEE70AF1EE10FA08D5B4EECB0AF1EECE
:1063200010FACCBF6BEE80BA6BEE8BBA09EB0402AD
:10633000D2ED007AD6ED006AA94B38EE2B7A1A1905
:1063400037EE277AF7EE007A77EE677A8BED007AF0
:1063500067EEA87A95ED007AC2ED007AF4EEE76A6E
:10636000F1EE10FAB4EEE77A48BFC6ED007AF1EE2E
:1063700010FA01DDC5ED007A57ED017AF5EEC07A2D
:10638000F1EE10FA0AF1010A37DD924B1B59A3BB5B
:10639000924B2344D3ED007A77EEAA7AFDEEE77AAA
:1063A00017EE902A511E01324A2A21EAE171A8BF54
:1063B0004A228A4221DB531A022B03F1010E0FD924
:1063C0007D4B2EF003000B4418444FF0013C43F882
:1063D00004CB8342FBD12EF003039E4519440CD01D
:1063E0000123754801EB030C6245435405DB023180
:1063F0008A4200F80C30A8BF4354474504F1040416
:106400007FF466AF774BDDF82CB0D3ED005A764BB6
:10641000DDF8309093ED005AF5EEC09AF1EE10FAE7
:106420005246DDF828A040F33C86012A40F36D87F0
:106430006E4B9FED6F2ADFED6F2ADFED6F1AF0EEE6
:10644000457AB0EE657A01210025B6EE004ABFEE2E
:10645000003AF7EE003A5A681E2A43DD1868824275
:1064600040DB9C68A2423DDB07EE900AF8EEE76A4B
:1064700007EE902AF8EEE77A06EE104AF4EE676A25
:10648000F1EE10FAB8EEC66A05D1F4EE467AF1EEF6
:1064900010FA00F0EE8776EE866AF0EE674AD6EEE6
:1064A000844A36EE646A76EE677AC7EEA46A66EED0
:1064B000846AF4EEC36AF1EE10FA05DDF4EEE36AE5
:1064C000F1EE10FA00F1EF87F5EEC06AF1EE10FA86
:1064D00054BFF0EE627AF0EE427A002D08BFB0EEC3
:1064E000677A01350131182903F10403B3D1002D76
:1064F00000F0118741484249424A534653F8044F3D
:10650000B4B1D2ED006AF5EEC06AF1EE10FA0FDD1B
:10651000D1ED006AF4EE676AF1EE10FAF4EE476A24
:10652000C8BFF0EE667AF1EE10FA48BFB0EE667AB8
:10653000984202F1040201F10401DFD1F7EE006A92
:10654000F4EEE67AF1EE10FA40F19C85F5EEC07AB1
:10655000F1EE10FA40F36D8677EEC57AF5EE006A3B
:10656000A7EEA65A204BF7EE007AB4EEE77AF1EEEA
:1065700010FA83ED005A40F18985B5EEC07AF1EE4C
:1065800010FA40F3528637EE657AF5EE004AE7EEF0
:10659000245A144B009A9FED1C4AC3ED005A9FEDFC
:1065A000093A099CDDE90331B6EE006AF7EE003ADC
:1065B000FFEE002A62E000BF70AD01209CAB01201D
:1065C000A4AB0120CDCCCC3D9A99993E3870603C6B
:1065D000CDCC4C3E7CAA0120FCAC0120C4AC0120F7
:1065E0008CAC0120A8AB0120A0AB0120A01B002097
:1065F0000916B2BD38BDE9B44316323DB0AA012038
:1066000034AD0120ACAB01206666663FE4AB0120EF
:10661000D3ED007A99ED007A75EE856AB0EE672ABF
:1066200096EE862AF0EE426AB0EE672AA6EEA42A1B
:1066300072EE677A83ED002A67EE8A7A67EE867AD1
:10664000F4EEE37AF1EE10FA4ED5F4EEE27AF1EEE2
:1066500010FAD8BFF0EE627A77EEC77AA7EE837AA7
:1066600089ED007A504501F1040109F1040904F1B2
:10667000040403F1040302F104023BD05AF8045F5E
:10668000002DEFD1D2ED007AF5EEC07AF1EE10FADE
:10669000BEDCD1ED006A99ED007AD4ED007A66EEA9
:1066A000846A27EE047A67EE867AC1ED006A89ED86
:1066B000007AC4ED007AD5E70D4B96ED007A2344BD
:1066C000D3ED007AF4EEC77A95ED007AF1EE10FA88
:1066D000F4EEC77AC8BFC6ED007AF1EE10FA7FF586
:1066E0008CAEC5ED007A88E6F7EE007AB4E700BF1D
:1066F0008CAC0120D54B1C68002C00F0BB84059BA2
:10670000D3ED007AF5EEC07AF1EE10FA40F3B284E0
:106710009FEDD16ACE4BDFEDCF6A93ED007A67EE45
:10672000867A27EE267AFDEEE77AF8EEE76A17EE2C
:10673000901A67EE267A0131FDEEE77A17EE900A9D
:10674000C24B5D6805B3059B93ED017AB5EEC07A47
:10675000F1EE10FA18DD9FEDC06ABD4BDFEDBD6AAA
:10676000D3ED017A27EE067A67EEA67ABDEEC77AF8
:10677000F8EEC76A17EE103A67EEA67A1944FDEEF6
:10678000E77A17EE903A1844B04B9E6806B3059B23
:1067900093ED027AB5EEC07AF1EE10FA18DD9FEDB6
:1067A000AE6AAB4BDFEDAB6AD3ED027A27EE067A29
:1067B00067EEA67ABDEEC77AF8EEC76A17EE103A12
:1067C00067EEA67A1944FDEEE77A17EE903A184480
:1067D0009E4BDF6807B3059B93ED037AB5EEC07A55
:1067E000F1EE10FA18DD9FED9C6A994BDFED996A86
:1067F000D3ED037A27EE067A67EEA67ABDEEC77A66
:10680000F8EEC76A17EE103A67EEA67A1944FDEE65
:10681000E77A17EE903A18448C4BD3F810C0BCF1CD
:10682000000F20D0059B93ED047AB5EEC07AF1EE0F
:1068300010FA18DD9FED886A854BDFED866AD3ED8F
:10684000047A27EE067A67EEA67ABDEEC77AF8EEEE
:10685000C76A17EE103A67EEA67A1944FDEEE77A9A
:1068600017EE903A1844794BD3F814E0BEF1000FBC
:1068700020D0059B93ED057AB5EEC07AF1EE10FAC3
:1068800018DD9FED756A724BDFED726AD3ED057A04
:1068900027EE067A67EEA67ABDEEC77AF8EEC76AEB
:1068A00017EE103A67EEA67A1944FDEEE77A17EE76
:1068B000903A1844654BD3F81880B8F1000F20D0F7
:1068C000059B93ED067AB5EEC07AF1EE10FA18DD6D
:1068D0009FED616A5E4BDFED5F6AD3ED067A27EECE
:1068E000067A67EEA67ABDEEC77AF8EEC76A17EEAB
:1068F000103A67EEA67A1944FDEEE77A17EE903A61
:106900001844524BD3F81C90B9F1000F20D0059BCE
:1069100093ED077AB5EEC07AF1EE10FA18DD9FED2F
:106920004E6A4B4BDFED4B6AD3ED077A27EE067AC2
:1069300067EEA67ABDEEC77AF8EEC76A17EE103A90
:1069400067EEA67A1944FDEEE77A17EE903A1844FE
:106950003E4BD3F820A0BAF1000F20D0059B93ED59
:10696000087AB5EEC07AF1EE10FA18DD9FED3A6ABA
:10697000374BDFED386AD3ED087A27EE067A67EEFB
:10698000A67ABDEEC77AF8EEC76A17EE103A67EE40
:10699000A67A1944FDEEE77A17EE903A18442B4B8D
:1069A0005B6A039303B3059B93ED097AB5EEC07A56
:1069B000F1EE10FA18DD9FED286A254BDFED256A10
:1069C000D3ED097A27EE067A67EEA67ABDEEC77A8E
:1069D000F8EEC76A17EE103A67EEA67A1944FDEE94
:1069E000E77A17EE903A1844184B9B6A049303B366
:1069F000059B93ED0A7AB5EEC07AF1EE10FA18DD38
:106A00009FED156A124BDFED136AD3ED0A7A27EE7C
:106A1000067A67EEA67ABDEEC77AF8EEC76A17EE79
:106A2000103A67EEA67A1944FDEEE77A17EE903A2F
:106A30001844064BDB6A09934BB3059B93ED0B7A25
:106A4000B5EEC07AF1EE10FA21DD07E07CAA012054
:106A50008CAC012000009242000048441FED026A05
:106A6000DF4BDFEDE06AD3ED0B7A27EE067A67EEB7
:106A7000A67ABDEEC77AF8EEC76A17EE103A67EE4F
:106A8000A67A1944FDEEE77A17EE903A1844D64BF1
:106A90001B6B0A9303B3059B93ED0C7AB5EEC07A9A
:106AA000F1EE10FA18DD9FEDD26ACD4BDFEDCD6A25
:106AB000D3ED0C7A27EE067A67EEA67ABDEEC77A9A
:106AC000F8EEC76A17EE103A67EEA67A1944FDEEA3
:106AD000E77A17EE903A1844C34B5B6B009303B30D
:106AE000059B93ED0D7AB5EEC07AF1EE10FA18DD44
:106AF0009FEDBF6ABA4BDFEDBB6AD3ED0D7A27EE8F
:106B0000067A67EEA67ABDEEC77AF8EEC76A17EE88
:106B1000103A67EEA67A1944FDEEE77A17EE903A3E
:106B2000184401225BF8043F1E3B23EAE37302FB97
:106B3000030001324A2A1944F4D107EE901A9FED5E
:106B4000A97AAA4BF8EEE77AD3ED006A67EE877A66
:106B500007EE100AB8EEC77A87EE276AB5EE007A1C
:106B600076EE667AE7EE876AC3ED006A002C00F0E5
:106B70007F82059BD3ED007AF5EEC07AF1EE10FA34
:106B800040F37582DFED9A6A019B67EEA67A93ED7A
:106B9000007AFDEEE77AF3EE076A27EE267AF8EE42
:106BA000E76A17EE903A67EE267A0133FDEEE77A50
:106BB00017EE904A05B3059A92ED017AB5EEC07AC8
:106BC000F1EE10FA18DDDFED8A6A019A27EE267AD7
:106BD000D2ED017ABDEEC77AF3EE076A67EEA67AC8
:106BE000F8EEC76A17EE102A67EEA67A1344FDEE98
:106BF000E77A17EE902A144406B3059A92ED027ACA
:106C0000B5EEC07AF1EE10FA18DDDFED796A019A7F
:106C100027EE267AD2ED027ABDEEC77AF3EE076A46
:106C200067EEA67AF8EEC76A17EE102A67EEA67A24
:106C30001344FDEEE77A17EE902A144407B3059A41
:106C400092ED037AB5EEC07AF1EE10FA18DDDFEDC1
:106C5000686A019A27EE267AD2ED037ABDEEC77AEA
:106C6000F3EE076A67EEA67AF8EEC76A17EE102A07
:106C700067EEA67A1344FDEEE77A17EE902A1444E5
:106C8000BCF1000F20D0059A92ED047AB5EEC07ADF
:106C9000F1EE10FA18DDDFED566A019A27EE267A3A
:106CA000D2ED047ABDEEC77AF3EE076A67EEA67AF4
:106CB000F8EEC76A17EE102A67EEA67A1344FDEEC7
:106CC000E77A17EE902A1444BEF1000F20D0059AFF
:106CD00092ED057AB5EEC07AF1EE10FA18DDDFED2F
:106CE000446A019A27EE267AD2ED057ABDEEC77A7C
:106CF000F3EE076A67EEA67AF8EEC76A17EE102A77
:106D000067EEA67A1344FDEEE77A17EE902A144454
:106D1000B8F1000F20D0059A92ED067AB5EEC07A50
:106D2000F1EE10FA18DDDFED326A019A27EE267ACD
:106D3000D2ED067ABDEEC77AF3EE076A67EEA67A61
:106D4000F8EEC76A17EE102A67EEA67A1344FDEE36
:106D5000E77A17EE902A1444B9F1000F20D0059A73
:106D600092ED077AB5EEC07AF1EE10FA18DDDFED9C
:106D7000206A019A27EE267AD2ED077ABDEEC77A0D
:106D8000F3EE076A67EEA67AF8EEC76A17EE102AE6
:106D900067EEA67A1344FDEEE77A17EE902A1444C4
:106DA000BAF1000F2CD0059A92ED087AB5EEC07AB0
:106DB000F1EE10FA24DDDFED0E6A019A27EE267A55
:106DC000D2ED087ABDEEC77AF3EE076A67EEA67ACF
:106DD000F8EEC76A17EE102A67EEA67A0AE000BF3F
:106DE0008CAC0120000092427CAA012094AB0120CF
:106DF000000048441344FDEEE77A17EE902A14444D
:106E0000039A02B3059A92ED097AB5EEC07AF1EED3
:106E100010FA18DD5FED0A6A019A27EE267AD2EDA4
:106E2000097ABDEEC77AF3EE076A67EEA67AF8EE46
:106E3000C76A17EE102A67EEA67A1344FDEEE77ACA
:106E400017EE902A1444049A02B3059A92ED0A7A36
:106E5000B5EEC07AF1EE10FA18DD5FED1B6A019A0B
:106E600027EE267AD2ED0A7ABDEEC77AF3EE076AEC
:106E700067EEA67AF8EEC76A17EE102A67EEA67AD2
:106E80001344FDEEE77A17EE902A1444099A02B3F0
:106E9000059A92ED0B7AB5EEC07AF1EE10FA18DD94
:106EA0005FED2D6A019A27EE267AD2ED0B7ABDEEC0
:106EB000C77AF3EE076A67EEA67AF8EEC76A17EEAE
:106EC000102A67EEA67A1344FDEEE77A17EE902AB1
:106ED00014440A9A02B3059A92ED0C7AB5EEC07A80
:106EE000F1EE10FA18DD5FED3E6A019A27EE267A80
:106EF000D2ED0C7ABDEEC77AF3EE076A67EEA67A9A
:106F0000F8EEC76A17EE102A67EEA67A1344FDEE74
:106F1000E77A17EE902A1444009A02B3059A92ED8C
:106F20000D7AB5EEC07AF1EE10FA18DD5FED506A19
:106F3000019A27EE267AD2ED0D7ABDEEC77AF3EEEE
:106F4000076A67EEA67AF8EEC76A17EE102A67EEB0
:106F5000A67A1344FDEEE77A17EE902A14440D98B2
:106F6000012150F8042F1E3A22EAE27201FB02448A
:106F7000013118291344F4D107EE903AB8EEE77ABC
:106F8000F3EE077A27EE277A07EE904AF8EEE77AD3
:106F9000CE4BCF4AD3ED006A126887EE876A002A8B
:106FA000B5EE007A76EE667AE7EE876AC3ED006AA0
:106FB0007DDBC84B1B68002B2DDB059DC64905EB0F
:106FC000830001EB8301076801980C6800EB8301E3
:106FD00005EB82050E68C0492F6001EB8200019924
:106FE000046001EB8201079F069C02980E6000EB93
:106FF000830007EB83050299069E2D6804EB83034B
:1070000001EB8201046818680C6007EB820306EB51
:1070100082021D601060B14A089D42EA05035B07C9
:1070200040F0D681D2E900301446D2E902126860FD
:107030006069A9606861A1692B6020462369EA60E4
:10704000A961E2692B610146236AEA610A462B6263
:10705000D2E90C23646A806AC96A6C62C5E90A01D4
:107060002A636B6315B0BDEC0A8BBDE8F08F00247A
:1070700001239FE500200121FFF762BBB0EE6A8A81
:10708000FEF7CDBDF0EE667AFFF766BAB0EE677A2E
:10709000FFF779BAF0EE679AFEF728BC1446FEF7C0
:1070A00081BCF0EE457AB0EE657AFFF723BA8C4BDF
:1070B0001B68002BBFF67DAFADE707EE106AB8EE98
:1070C000C78A38EE678AFEF7AABD73193B4400EE03
:1070D000103AB8EEC00AF3EE0E7A30EE670A20EEF0
:1070E000020AFDF7B3FF07EE906A05EE905AB8EE7C
:1070F000E77AB8EEE55A05EE907AB4EE457AF1EE0D
:1071000010FAF8EEE55AF0EE407A0AED010A05D1E0
:10711000B4EE655AF1EE10FA00F0D18137EE257A1F
:10712000F6EE001AB0EE451A97EE211AFFEE000AAD
:1071300035EEC17A37EE457AC7EE015A25EEA17ACF
:10714000B4EEE07AF1EE10FA07DDF7EE005AB4EE95
:10715000E57AF1EE10FA00F1B581B5EEC07ADFED17
:10716000615A9FED617AF1EE10FA58BFF0EE475A7E
:10717000F5EEC07AF1EE10FA7EF732AC35EEE67A33
:10718000079BC0ED005A27EE0A7AB7EE005A27EEA9
:10719000227A0B44B4EEC57AF1EE10FAD3ED006A10
:1071A00040F1B080FFEE005AB4EEE57AF1EE10FA4D
:1071B000D8BFB0EE657A77EEC67A37EE667A67EEBC
:1071C0008A7AE7EE036A069A67EEA37AB2EE046A59
:1071D000F4EEC67A1144F1EE10FA91ED007AC3EDA7
:1071E000006A40F18C80F5EEC07AF1EE10FA01DC15
:1071F000F0EE647A77EEC77AF5EE006AA7EEA67A2B
:1072000008F10108B8F10E0F81ED007A7EF496AB1B
:10721000FEF786BC4A46FEF71FBF226015B0BDECE4
:107220000A8BBDE8F04FFDF7C1BF9FED307AFFF745
:10723000AAB9DFED2E7AFFF78FB915464824FEF77D
:10724000C0BBDFED2A9AFEF751BB059A00235363BA
:10725000FEF76DBA059A00231363FEF760BA059A2C
:107260000023D362FEF753BA059A00239362FEF718
:1072700046BA059A00235362FEF739BA059A0023ED
:107280001362FEF72CBA059A0023D361FEF71FBAEA
:10729000059A00239361FEF712BA059A0023536101
:1072A000FEF705BA059A00231361FEF7F8B9059AAF
:1072B0000023D360FEF7EBB9059A00239360FEF735
:1072C000DEB90B4B0593FEF7CAB900BF98AB01209E
:1072D00020000020381A00208CAC01207CAA01205C
:1072E0001400002058FF7FBF58FF7F3F00000000C0
:1072F000ACAB0120059A00235360FEF7B8B9F0EE5D
:10730000467A77E7B0EE457A55E7F0EE457AB0EE8B
:10731000657A7FF4EFA8764BDFED762A9FED763A1B
:107320009FED762A01220025F6EE004AFFEE003A94
:10733000B7EE004A2AE077EE877AB0EE666A97EEFB
:10734000A46A77EE467A77EEE67A87EE867A67EE7B
:10735000247AF4EEE37AF1EE10FA05DDF4EEC47A65
:10736000F1EE10FA00F19480F5EEC07AF1EE10FA29
:1073700054BFB0EE437AB0EE627AF0EE477A0D4633
:107380000132182A03F104033FF4B4A85968A94252
:10739000F6DD18688142F3DD9C68A142F0DB07EE60
:1073A000101A07EE900AF8EEC76AF8EEE77A07EED1
:1073B000104AF4EE667AF1EE10FAB8EEC77ABAD156
:1073C000F4EE476AF1EE10FAB5D19FED4D7AD4E7AD
:1073D0004C4CD4E90130D4E90312A860A069E960FB
:1073E000A861E1696B60204663692A61E961226AEC
:1073F0006B610146636A2A620A466B621346A46A9D
:10740000C06A096B526B1B68AC62C5E90B016A6309
:107410002B6015B0BDEC0A8BBDE8F08F3A4A1346DD
:1074200002F5927053F8041F013983421960F9D1B3
:10743000364B03F15C0453F8041F0139A342196071
:10744000F9D1FEF79BB9661E5BF82670BD4204DADF
:10745000631C5BF82330BB4203DB2F462646FEF756
:10746000D9BE012E7EF4BFAEDDE90B530224FEF738
:10747000A5BADFED237AFFF730B8741C5BF824302F
:107480009F42BEF6B0AE492C28D1099DFEF799BAAD
:1074900007EE102AB8EEC77A37EE677A37EE447AED
:1074A00027EE027A69E707EE901AF8EEE77A77EEB0
:1074B000E67A77EEE37A67EEA17AFFF70EB8F0EEA0
:1074C000645A55E605EE904AF8EEE55A75EEC75A4D
:1074D0004EE61D463446FEF774BA3446621C5BF82D
:1074E00024305BF8225026461446FEF767BA00BFE8
:1074F000A01B00200916B2BD38BDE9B44316323DC9
:10750000431632BD7CAA0120AC180020D4190020FB
:1075100070B590B038B39200C9070F24944061F061
:107520007F41934021EA0401149A069219430023F3
:1075300001220A93CDE90B33CDE90D330991039371
:107540000F93079303AC08AB0626402501A90068FA
:107550000194CDE9045208968DF82920029301F098
:107560004FF810B070BD014804F024F91CC50000AC
:107570002DE9F04186B0002800F09E8000270446E7
:1075800000F130060D469046304639464022CDE99E
:107590000377059704F01FFBA36A012B13D9B4F8F6
:1075A000503259050FD50096394643462A462046A3
:1075B000FFF7AEFF00284CD123685B7A012B5DD02A
:1075C000022B4BD023B14FF4E16006B0BDE8F0814F
:1075D000D4E90D02D4E90F31170CADF80E2006AA3C
:1075E000ADF8120002EB4502180CADF81070ADF8C2
:1075F0000C0032F80C2C1B0242FA08F29BB2D207A4
:1076000043EA1163DFD5AF00FB4003F00F034345AE
:10761000D9D100962A46434601212046FFF778FF3C
:10762000B8B923685B7A012B3FD0022B36D0002BF0
:10763000C9D1D4E90F321B029BB243EA126323FA89
:1076400007F707F00F0740F21673474518BF1846B3
:10765000BBE740F2097006B0BDE8F081D4E90C70D8
:10766000D4E90E23216C3FBA00BA12BA1BBA09BA88
:10767000C4E90C70C4E90E232164ADE7236B5BBA47
:10768000606B236340BAA26B606352BAE36BA26380
:107690005BBA216CE36349BA21649DE7D4E90F32F8
:1076A0001BBA12BAC4E90F32C5E7E36B5BBA226CAE
:1076B000E36352BA2264BEE7014804F07BF800BFDE
:1076C00034C500002DE9F047DFF858A08AB08046A5
:1076D0000F46164600254FF00C093946D8F8000031
:1076E00000F08EFF40F2032269460446B0B13B68C9
:1076F0008BB102ABD8F800000895CDE90455CDE96F
:107700000655CDE90295CDE90053ADF81020CDF82E
:1077100024A000F075FF0EB1013EDEE720460AB05E
:10772000BDE8F0870800F9FF70B58AB008B30024FF
:10773000436A0994CDE90544CDE907441B040D21B2
:107740000122CDE90334064602918DF8112002ADE5
:10775000032269463046CDE90045FFF7B3FF30B953
:10776000059BDA05F4D5C3F34323072BF0D00AB009
:1077700070BD014804F01EF84CC50000F0B591B092
:10778000002800F09480002504462946202208A8FD
:1077900004F13006CDE9015504F01DFA29463046C2
:1077A0004022CDE90355CDE90555079504F013FABC
:1077B0002046FFF7B9FF60BB616A206800F0FEFD5C
:1077C000054608BB08AA03A80123029201904022A3
:1077D00020688DF8293001A90D27CDE904230696EC
:1077E000089700F00DFF0B9A324B134003435BD117
:1077F00023685B7A012B11D0022B4AD0C3B14FF41E
:10780000E165284611B0F0BD40F21575284611B06B
:10781000F0BD4FF4E365284611B0F0BD04F12C0330
:1078200004F16C0153F8042F52BA99421A60F9D14D
:10783000D4E90E23180E40EA0220A4F88002100EAC
:10784000216B84F87C02100CC2F3033284F87D02B1
:1078500084F87E22C3F30140C3F3033284F8830229
:1078600084F88422880F626BA4F87612C3F38546ED
:10787000C1F34071C3F3032384F87402284684F8EB
:10788000826284F8853284F87512C4F8782211B0C7
:10789000F0BD04F12C0304F16C0153F8042F12BA6B
:1078A00099421A60F9D1C3E740F20975AEE7024880
:1078B00003F080FF0800F9FF64C5000020B10A460C
:1078C000416A006800F052BD08B5014803F072FF3C
:1078D0007CC5000038B1B0F8540200F4C060003834
:1078E00018BF0120704708B5014803F063FF00BFCF
:1078F00094C500002DE9F04F95B0CDE90021002896
:1079000000F0B5801C46019B002B00F0AD80002CE0
:1079100000F0A780009BD0F88822E11891428346AE
:1079200000F29C8000F1300222F003030393043341
:10793000012602930025019B9BF81D2003EB45289F
:10794000002A67D1002E7ED018F003027BD1B4F557
:10795000803F70D227461446009BC24603EB0509C0
:107960000126002120220CA8CDE9051104F033F9ED
:10797000DBF88C220021B2F5007FCDE90711CDE9BB
:1079800009110B9140D35846FFF7CEFE00283BD19A
:10799000DBF82C20012F4FF001030CBF1121122125
:1079A0008DF81C3093074FF001038DF83930314BBF
:1079B0001393CDE90C1958BF4FEA49224FF40071D7
:1079C0000CAB089158BF0D92069305A907AB032293
:1079D0005846CDE9097A0593FFF774FE814698B9B8
:1079E0009BF81D203D4402B92EB1002CA3D148467E
:1079F00015B0BDE8F08F029940464FF4007204F0D4
:107A0000E8F8002C97D1F2E740F20979484615B022
:107A1000BDE8F08FB4F5803F0DD227460024002E3C
:107A20009AD1009B03EB0509039B043313D0DDF8C7
:107A300008A0002695E7A4F57F44FF3C4FF6FF77AA
:107A4000002E89D1EDE702984FF40072002104F076
:107A5000C2F80127E5E7084803F0ACFE074803F049
:107A6000A9FE074803F0A6FE064803F0A3FE064859
:107A700003F0A0FE0800F9FF38C60000F8C50000BA
:107A8000DCC50000C4C50000ACC500002DE9F04F06
:107A9000A5B0CDE90031002800F0F680019B002B55
:107AA00000F0EF80009B002B00F0E880009BD0F8F6
:107AB000881213448B42029300F2DD8000F1300300
:107AC0000593009D23F00303039303F1040B4FF090
:107AD000010900248046009B98F81D205E1B019B35
:107AE00003EB4626002A40F0A880B9F1000F00F011
:107AF000B780B70740F0B4804FF6FF77AF4228BF9A
:107B00002F46029B4FF00109A3EB050A202214A87F
:107B10000021CDE9064404F05EF8D8F88C220E94DA
:107B2000B2F5007FCDE90A44CDE90C447FD340464D
:107B3000FFF7FAFD0490002879D1D8F800201168E9
:107B40004B6AD801FCD5012F0CBF18221922D8F896
:107B50002C104F4B1B93CDE9142A01228B078DF873
:107B600028208DF859204FF400720B9214AB5CBFA3
:107B70004FEA4A221592079306A90AAB0322404610
:107B80000C970E960693FFF79DFDB8B998F81D2047
:107B9000ED1B12B9B9F1000F07D0002D9BD1DDF814
:107BA0001080404625B0BDE8F08F4FF40072494682
:107BB000584604F010F8002D8DD1F0E72022002166
:107BC0001CA8CDE9084404F006F8059E139404228D
:107BD00000213046CDE90F44CDE9114403F0FBFF0D
:107BE0004046FFF7A1FD10BBD8F82410D8F80000DC
:107BF00000F0E4FBD8B916201CAB012212960993C1
:107C000004260FAB1C9008A9D8F800000893CDE912
:107C100010628DF8792000F0F3FC40B91F9A1C4BDC
:107C20001342B3D1D8F8302017BA002AAED140F2AF
:107C30000978404625B0BDE8F08F4FF6FF77AF4298
:107C400028BF2F46B9F1000F7FF45BAF029BA3EB77
:107C5000050A039B04330BD05E464FF0000955E73D
:107C600031464FF40072584603F0B3FF0127EDE7A9
:107C7000084803F09FFD084803F09CFD074803F007
:107C800099FD074803F096FD064803F093FD00BFF9
:107C90000800F9FFDCC600009CC6000080C600009A
:107CA00068C6000050C60000F0B58BB0002800F098
:107CB00087800123044680F89332006800F0A8FB17
:107CC00020B140F2137528460BB0F0BD0822049095
:107CD000CDE90500CDE907004FF4D57309250090E3
:107CE00009900DEB020620688DF811506946CDE928
:107CF0000223019600F084FC40B1002D50D0206892
:107D00006946013D00F07CFC0028F6D19DF8143056
:107D1000AA2BF2D1E36A2C4A43F00803E362002362
:107D20000493CDE90033CDE90533CDE90733039260
:107D300009932922042302928DF811304FF47A77A7
:107D4000012507E0059B002B19DB0A2000F0E4FB6E
:107D5000013F2DD02068002100F030FB03460028B1
:107D6000F6D120686946CDE9003600F049FC0546A9
:107D70000028E7D040F2147528460BB0F0BD59003A
:107D800003D5E26A42F00202E262DA0103D5E26A56
:107D900042F02002E2622846C4F834320BB0F0BD53
:107DA000206800F035FB00288BD14FF44812B6E76D
:107DB000002D40F2147318BF1D4628460BB0F0BDCD
:107DC000024803F0F7FC00BF00003240F4C6000098
:107DD0002DE9F04190B0002800F09282037F044624
:107DE000002B00F08A820025C5622946006800F059
:107DF000A1FC2368474AD3E9000102F0A7FC2368ED
:107E000020626421186802F009FD2046FFF74CFF4C
:107E100040F22A739842064616D002232068039542
:107E200003A9032708AECDE90955CDE90B55CDE9E6
:107E30000D550F9508938DF82970049600F0E0FB1E
:107E4000054628B140F20D76304610B0BDE8F0810D
:107E500004F130080BA91022404603F0BAFED4E921
:107E60000C12D4E90E034FEA116C4CEA022CC1F358
:107E70000B21120E84F83C32C4F844C24FEA136C52
:107E80001B0AA4F8481284F84122010E020CA4F83F
:107E90003A32030A84F8400284F83D1284F83F32F3
:107EA000206884F838C2082384F83E2203A9CDE96B
:107EB0000A55CDE90C55CDE90E55CDE90875CDE94A
:107EC00003568DF8293000F09BFB28B140F20E7666
:107ED000304610B0BDE8F0810B9B0A901A0C134697
:107EE000CDE90C00CDE90E00CDE903061204636272
:107EF0000B90092320688DF8297003A9CDE9083279
:107F000000F07EFB40B140F20F76304610B0BDE885
:107F1000F08100BF801A06000BA91022404603F032
:107F200058FED4E90E32A18F170C49BA900FA4F86D
:107F30004E121D0D84F84D72C3F303411F0484F8E3
:107F40004C020246A4F8505284F8521205D5B4F8F7
:107F5000545245F00105A4F854525D0405D5B4F817
:107F6000545245F00105A4F854529F0405D5B4F8C5
:107F7000545245F00405A4F85452DD0405D5B4F874
:107F8000545245F00805A4F85452002A00F03C81F0
:107F9000012800F02081626B530405D5B4F85432F7
:107FA00043F01003A4F85432236BC3F38261C3F38C
:107FB000835084F863129F02C2F3C61102F07F025D
:107FC00084F8640284F8611284F8622205D5B4F85A
:107FD000542242F04002A4F854221D0405D5B4F8FE
:107FE000542242F08002A4F85422580405D5B4F873
:107FF000542242F48072A4F85422990405D5B4F8AE
:10800000542242F40072A4F85422DA0405D5B4F8DC
:10801000542242F48062A4F85422C3F3812384F8EA
:10802000653201212046FFF749FC0546002840F053
:10803000CF802368B44AD3E9000102F087FB2022F5
:10804000206229463046CDE9015503F0C4FD29469A
:1080500008224046CDE90355CDE90555079503F0C3
:10806000BAFD616A206800F0A9F9002840F0AD80EF
:10807000099003A80123CDE90106332508222068D1
:10808000CDF8188001A9CDE9042308958DF8293091
:1080900000F0B6FA002840F098800B9A9B4B1340F2
:1080A000002B40F0068125686B7A012B00F00D81D2
:1080B000022B00F00381002B40F08780D4E90C30C4
:1080C000190FC3F303621F0284F8681284F869224F
:1080D00005D5B4F86A1241F00101A4F86A12C3F39D
:1080E0000341C3F3025784F86D12190484F86C72CB
:1080F000C3F3074705D5B4F86A1241F00201A4F8AA
:108100006A12990A01F01E01C4F87002012A03F0F4
:10811000030084F86E1284F86F02DBB200F0EA808C
:10812000022A00F0DC80002A00F0D680E26A7F0795
:1081300044BF42F00402E262D80744BF42F080022A
:10814000E262990702D542F04002E262530722D56B
:10815000002120223046CDE9031103F03CFD616A85
:10816000284600F02BF9002840F09D8006220125CA
:108170000223039003A92068049608928DF82950E1
:10818000099300F03DFA002840F08D8029462068D0
:1081900000F0D0FA256828464FF4007100F052F93B
:1081A0000646002840F0828094F89332032B5CD07E
:1081B000014601222046FFF7DBF9002860D0B0F528
:1081C000E16F6CD040F21B763EE640F211763BE662
:1081D0004FF4E26638E6626B1B0403F47C1343EA57
:1081E00012434FF6FE714FF400708B42C4F85832C0
:1081F000C4F88C0203D9E16A41F01001E162013355
:108200009B02C4F88832C7E6626B40F6FC7000EA55
:10821000830343EA9270C2F3C235431CC4F8580288
:10822000A81C8340100D00F00E0084F86052C2F3C9
:10823000C26784F85E02C2F30265C2F38240092974
:10824000C4F8883284F85C7284F85D5284F85F0266
:1082500006D08B405B0A4FF40071C4E9A2319BE663
:108260004FF40073C4F88C3296E694F89032012BE8
:10827000A8D8014601222046FFF77AF90028A1D1AB
:1082800062692368012184F89012AAB120498A42C8
:1082900028BF0A46D3E9000102F058FA20622046BE
:1082A000FFF76CFAD0E540F21276CDE540F20A769F
:1082B000CAE5E26A256849E7154AEBE7D4E90C30DC
:1082C0001BBA00BAC4E90C30FAE6236B5BBA606BE8
:1082D000236340BA6063F3E60122A26226E7B4F8A2
:1082E0006A2292074FF0040148BF0822A16248BFEA
:1082F000A2621BE70222A26218E7064803F05AFABC
:10830000054803F057FA00BF40787D010800F9FFE7
:1083100080F0FA0224C700000CC7000010B5D8B1E5
:1083200001690446D9B1037F3BB10B78013B012BB6
:108330000CD901232377002010BD006800F0BCF9A0
:1083400040B921690B78013B012BF2D8206800F07D
:108350002FF9EEE7012010BD024803F02BFA024886
:1083600003F028FA50C7000068C7000010B58AB0B3
:1083700000230724CDE90333CDE90533CDE90733E5
:1083800009930294AAB10904012303918DF81130D5
:1083900002AA00236946CDE9003200F031F9059ABE
:1083A000054B1340034340F2097008BF00200AB098
:1083B00010BD8DF81120EBE70800F9FF30B58BB048
:1083C0000904002337250124039102AA6946049376
:1083D000CDE90533CDE907330093099302958DF874
:1083E0001140019200F00CF958B9059A074B13405F
:1083F0003BB912F0200F40F20C7308BF18460BB0C7
:1084000030BD40F209700BB030BD00BF0800F9FF6D
:1084100000B58BB0002302AA6946CDE90333CDE94C
:108420000533CDE90733CDE900320993029300F01B
:10843000E7F840F20973002818BF18460BB05DF842
:1084400004FB00BF30B58BB0002302AA03911025B6
:10845000012469460493CDE90533CDE90733009340
:108460000993019202958DF8114000F0C9F8059A20
:10847000044B1340034340F2097008BF00200BB0C7
:1084800030BD00BF0800F9FF704700BF08B518B144
:10849000012102F0D7FC08BD014803F08BF900BFB1
:1084A00094C700002DE9F04182B0C0B10D461646D8
:1084B0001F46044643F2DE7801E040450BD00097AA
:1084C000334600222946204602F0E2FC0028F4D17F
:1084D00002B0BDE8F081012002B0BDE8F0810148A2
:1084E00003F068F9C0C7000008B518B102F0BAFC83
:1084F000002008BD014803F05DF900BFECC7000093
:1085000008B518B102F0B8FC002008BD014803F01E
:1085100051F900BF18C800004FF47A73024903FBF9
:1085200000F000F0FFBC00BF0095BA0A10B50C4681
:108530004FF40071A06DFFF7D7FFE36D33B19A6878
:1085400022B1BDE8104019690020104710BD00BFDE
:1085500070B504460D46886D4FF48071FFF7C4FF77
:10856000A36BEA6D23F04003A36332B1936823B198
:10857000BDE8704011690120184770BD40F2A76145
:108580008A4210D040F2AA618A4208D040F2A66125
:10859000986D8A420CBF02210121FFF7A5BF986D9B
:1085A0000421FFF7A1BF986D0821FFF79DBF00BF11
:1085B00009B308B50368C1659A6A42F008029A6275
:1085C0005A6B42F040025A635A6B42F080025A637F
:1085D0009A6B42F040029A639A6B42F080029A636F
:1085E000186B10F0400005D08B6833B10120096989
:1085F0009847002008BD01207047184608BD00BFFD
:108600002DE9F04184B005460023806D03930E46AA
:108610000F21FFF775FF05F1340840F2A4670096BB
:10862000D5E90B232868414602F020FAB8420446F7
:10863000F5D0A86D03AB4FF0FF320F21FFF732FFEB
:10864000012802D0039B9F070AD52D686C6AE307B7
:108650001ED4A30724D40124204604B0BDE8F08131
:1086600032687AB158070DD41907EED4A86D03AB60
:108670004FF0FF320C21FFF715FF0128E5D0039BD7
:108680001A07E2D4002CE7D02D686C6AE307E0D526
:1086900064224FF00071284602F03EF8A307DAD5B5
:1086A000284664224FF0806102F036F8012420460B
:1086B00004B0BDE8F08100BF30B587B050B3836D22
:1086C000044653B30023CDE90133CDE903330593C9
:1086D000FFF7DAFE214602236372A372802351F86A
:1086E000080B0F4DC4E9033301F0B4FF21460D4BD5
:1086F00051F8340B059501AA01930B4D02952346C1
:1087000002F076F9A06DFFF7C1FE003818BF012016
:1087100007B030BD054803F04DF8054803F04AF8AE
:108720007D850000518500002D85000044C80000B3
:108730006CC80000026819B101290CBF0221042194
:10874000936A23F0060319439162704738B50029F4
:108750005DD0304B984206D003F50023984254D0A8
:108760002D4803F027F82D4A136843F00063136087
:108770000B794A784C799B0002F0030203F00C035A
:10878000042C43EA0203CA782BD05201CD7902F0BF
:1087900060021343002D31D043F090038360C26820
:1087A00022F00F0204F0030313438A790AB143F065
:1087B00004038A780AB143F00803C360026A0B78A5
:1087C000097A22F0030203F0030313430362436AAE
:1087D00019B143F00803436238BD23F00803436234
:1087E00038BD5201CC7902F0600213430CB143F062
:1087F00080038360C36823F00F03D6E743F01003C0
:108800008360C26822F00F02CCE7054AACE7054856
:1088100002F0D0FF00B00340C0C800003C8004401C
:10882000308004409CC80000026A12F040020346F7
:1088300004D0026A22F0400202620122596A41F029
:10884000C00159621968080635D4196A596A49067F
:10885000F8D519695AB30122196A41F04001196229
:10886000196A586A00F04000104322D1D96C30B424
:108870009C6C5A6C1D6C21441144DC6B9A6B29442E
:1088800021441144490841F40041D962D96E9C6EDB
:108890005A6E1D6E21441144DC6D9A6D29442144A9
:1088A0001144490841F4004130BC196370471A6A09
:1088B0005B6A012070471969002AD1D00022CBE7FA
:1088C000C36819B923F01003C360704743F0100365
:1088D000C3607047436A042923F0070304D001F002
:1088E00003010B4343F0040343627047012910B5B1
:1088F00011D86AB11368547903F01F030CB143F027
:10890000200312790AB143F0400340F8213010BD32
:10891000024802F04FFF024802F04CFF28C9000055
:10892000F8C80000012904D850F8210000F08000A8
:10893000704708B5014802F03DFF00BF4CC9000078
:1089400008B50E4B1B7B03F00303012B06D0022B53
:1089500002D043B1002008BD094808BD094B1A6880
:1089600042B1186808BD084B1A68002AF9D10748B7
:1089700002F020FF064802F01DFF00BF0040064045
:10898000006CDC02C0AD0120BCAD01207CC9000040
:10899000A4C9000008B5FFF7D3FF104A1378517837
:1089A000127BC3F3C20311F0300F20FA03F002F080
:1089B000030206D02AB9062B0BD0072B04D040099E
:1089C00008BD022AF7D008BD054BA3FB0030C00844
:1089D00008BD044BA3FB0030000908BD0040064061
:1089E000ABAAAAAACDCCCCCC08B5FFF7A9FF70B131
:1089F000084B1A795B7903F01F03103302F007026A
:108A00000132B0FBF2F000FB03F0400808BD024861
:108A100002F0D0FE00400640CCC90000064B9A7917
:108A2000D20702D4054B18687047054A1B7A1068B4
:108A3000C3F34203D8407047004006403000002096
:108A40002C00002008B5084B1A78120601D400202B
:108A500008BD064A116821B19B7810689B09D8406F
:108A600008BD034802F0A6FE00500640BCAD012040
:108A70000CCA0000114B10B51C68C4F38144022CD1
:108A800009D0032C03D064B10024204610BD4FF45C
:108A90007A74204610BD0A4B1A685AB11C682046E9
:108AA00010BDFFF7CFFFB0F5004F08BF4FF40044F3
:108AB000204610BD034802F07DFE00BF0070044058
:108AC000C0AD01202CCA00001349426841F24403A2
:108AD00070B4CA5041F2040602788D594378847804
:108AE000120425F440355B0002F440322A4304F0BE
:108AF000010441F2640503F00E0323438A514B51F4
:108B0000C3780A689B0403F4402322F440221343F1
:108B100070BC0B60704700BF0070044008B5104B7C
:108B20005A78910702D49A79920601D5002008BD9F
:108B30009B79DB0611D50B4B18680028F6D0084A44
:108B40000949D378D278C3F341135B0003EBD21306
:108B500031F8133000FB03F008BDFFF71BFFECE713
:108B60000040064030000020A0CA000008B5154AA9
:108B700041F20403D358C3F30143022B16D0032B55
:108B800012D0012B15D0FFF7C9FF0E4941F2640343
:108B9000CA58CB5802F00102C3F3420302FB0000A3
:108BA0000133B0FBF3F008BD0748EEE7074B186848
:108BB000EBE7074B987910F04000E6D0FFF714FF81
:108BC000E3E700BF00700440006CDC02C4AD01208C
:108BD00000400640144A9379917CC3F38103022B31
:108BE000C9B205D0032B0BD0012B03D0FFF796BFE2
:108BF000FFF7A6BE9379DB070AD40C4B18687047C1
:108C0000C1F30010C9060AD493795A060AD47047F2
:108C10000749137A0868C3F34203D8407047054BED
:108C200018687047FFF7E0BE0040064030000020A3
:108C30002C000020C4AD012010B5094B9B79DB0648
:108C400009D5084B1C68FFF7C5FFB4EBD00F94BFE4
:108C50002046002010BDFFF79DFE0446F3E700BF4D
:108C6000004006403000002008B513280FD8DFE888
:108C700000F010101B404C0E272B2F0E0A585C33AF
:108C8000370E0E0E6567344B1B781B065BD4002035
:108C900008BDFFF79FFF314A41F24403D3581B0F31
:108CA0000133B0FBF3F008BDFFF794FF2B4A41F20C
:108CB0004403D358C3F303630133B0FBF3F008BD9F
:108CC000BDE80840FFF752BFBDE80840FFF7D2BE3D
:108CD000BDE80840FFF7B6BEBDE80840FFF71EBF7D
:108CE0001F4B987910F04000D2D0BDE80840FFF744
:108CF0007BBEFFF76FFF194A41F24403D358C3F319
:108D000003530133B0FBF3F008BDFFF763FF134AD1
:108D100041F24403D358C3F303430133B0FBF3F0F0
:108D200008BDBDE80840FFF787BF0D4B187810F06D
:108D30000200ADD0BDE80840FFF770BE094808BD8D
:108D40004FF47A7008BD084B1A680AB1186808BD5C
:108D5000064802F02FFD00BF00500640007004409E
:108D600000400640006CDC02BCAD0120ECC90000F4
:108D70000D4A137B03F0030383420DD0137B00F0F5
:108D8000030003F0FC031843107340F2DC5300BFF0
:108D9000013BFCD100207047117B01F0FC010B432B
:108DA00013730020704700BF0040064008B5B0B103
:108DB00043780C4A03F0070313715179837801F06B
:108DC000E00103F01F030B435371017813790B4348
:108DD00043F04003137193795B06FCD508BD02484C
:108DE00002F0E8FC004006404CCA0000036849F667
:108DF0009702934230B42AD9164A934294BF102264
:108E00002022154B05791978144C01F0F001294303
:108E100019706178457901F0C30129430A436270F2
:108E2000C2791978807901F05F0192010143D2B2D1
:108E300019709A7015B11B781A0601D430BC7047AE
:108E4000A3799B07FAD4A3799B07F9D5F6E700220B
:108E5000D7E700BF00127A000050064000400640ED
:108E6000012838B5044601D0002934D01B4A537874
:108E700003F0FD035370137803F03B0343F08003CA
:108E80001370937903F01C03082BFAD15379134D17
:108E900003F0BF035371AB799A06FCD4BCB10F4AFF
:108EA000537943F040035371117C230101F0EF012A
:108EB00003F010030B431374937CC3F30013A3421A
:108EC000FAD1064A93799B06FCD5002038BD0846A6
:108ED000FFF76CFFE3E7024802F06CFC004006403D
:108EE00068CA0000012938B50C46154600D08AB181
:108EF000FFF73EFF29462046FFF7B2FF074A1378E7
:108F000003F03F0313709379C3F38103032BFAD16A
:108F1000002038BD024802F04DFC00BF0040064072
:108F200084CA000008B590B10C4BA0FB01014FF0C2
:108F3000FF328B4208BF82420CD3094A002303F060
:108F400032F80046A0F101000028FBD108BD054819
:108F500002F030FC044802F02DFC00BF3F420F003D
:108F600000093D00B0CA0000D4CA000008B5064B95
:108F7000984202D0054802F01DFC054A136843F0F0
:108F80000203136008BD00BF00100240FCCA0000CD
:108F90003C8004401F2938B53AD8002A3ED012F050
:108FA0001F0438D100EB411101F58053106818609F
:108FB000938841F204009BB20B52D38841F2060021
:108FC0009BB20B5241F208039068C85041F20C0367
:108FD000D068C85041F210031069C850938A41F21A
:108FE00014009BB20B52D38A41F216009BB20B5273
:108FF00041F2180341F21C009569CD500C52938B3D
:109000009BB20B52D38B41F21E029BB28B5238BDE6
:10901000044802F0CFFB044802F0CCFB034802F006
:10902000C9FB00BF34CB00009CCB00007CCB000010
:1090300070B519B3134B984202D0134802F0BAFB33
:10904000124DCA782C688B784E7844F002042C605C
:109050004FF0FF340025C5604462C46204680D7897
:10906000520024F0560142EA83030B4343EA0613FD
:1090700043EA851343F08003036070BD044802F0A7
:1090800099FB00BF00800040F0CB0000408004400E
:10909000CCCB000008B578B110F01F030FD1082227
:1090A00003608380C3808360C36003618382C38263
:1090B00083618283C38308BD024802F07BFB0248C0
:1090C00002F078FB24CC000044CC00001F2904D817
:1090D000803100EB4110FFF7DDBF08B5014802F019
:1090E00069FB00BF74CC00001F2920B513D800EB2A
:1090F000411241F21C03D55AC36A426ACB40CA40AE
:109100005B00920002F0040203F00203C5F3C010FA
:109110001343184320BD014802F04CFBBCCC0000B7
:1091200070B500284CD08368017CD97741F21C02CD
:1091300003EB4111C3688A5A044602F08005C2F36A
:10914000C01263B341F218000958C91A4B09DDB1C6
:10915000DBB2617C8B425EB21AD0617C49B25B1A91
:1091600044BF217D43FA81F3D8B26674E17C26685E
:10917000091A49B2E17416B161682046B04715B1C9
:10918000A368227C1A7770BD1F2910D9013BDFE745
:10919000E37C217D99420FD000200346E5E7056876
:1091A000002DF0D0AC464168BDE870406047237D9B
:1091B000013B03F0FF03CCE7E17C4BB20846D4E768
:1091C000014802F0F7FA00BF04CD000008B50D48D1
:1091D0000021FFF789FF420708D40A481021FFF752
:1091E00083FF430707D4BFF34F8F08BD064B1868B2
:1091F000FFF796FFF1E7044B186CFFF791FFBFF301
:109200004F8F08BD00800040C8AD012008B50D4853
:109210000121FFF769FF420708D40A481121FFF72F
:1092200063FF430707D4BFF34F8F08BD064B586851
:10923000FFF776FFF1E7044B586CFFF771FFBFF3C0
:109240004F8F08BD00800040C8AD012008B50D4813
:109250000221FFF749FF420708D40A481221FFF70D
:1092600043FF430707D4BFF34F8F08BD064B9868F1
:10927000FFF756FFF1E7044B986CFFF751FFBFF380
:109280004F8F08BD00800040C8AD012008B50D48D3
:109290000321FFF729FF420708D40A481321FFF7EB
:1092A00023FF430707D4BFF34F8F08BD064BD86891
:1092B000FFF736FFF1E7044BD86CFFF731FFBFF340
:1092C0004F8F08BD00800040C8AD012008B50D4893
:1092D0000421FFF709FF420708D40A481421FFF7C9
:1092E00003FF430707D4BFF34F8F08BD064B186930
:1092F000FFF716FFF1E7044B186DFFF711FFBFF3FF
:109300004F8F08BD00800040C8AD012008B50D4852
:109310000521FFF7E9FE420708D40A481521FFF7A7
:10932000E3FE430707D4BFF34F8F08BD064B5869D0
:10933000FFF7F6FEF1E7044B586DFFF7F1FEBFF3C0
:109340004F8F08BD00800040C8AD012008B50D4812
:109350000621FFF7C9FE420708D40A481621FFF785
:10936000C3FE430707D4BFF34F8F08BD064B986970
:10937000FFF7D6FEF1E7044B986DFFF7D1FEBFF380
:109380004F8F08BD00800040C8AD012008B50D48D2
:109390000721FFF7A9FE420708D40A481721FFF763
:1093A000A3FE430707D4BFF34F8F08BD064BD86910
:1093B000FFF7B6FEF1E7044BD86DFFF7B1FEBFF340
:1093C0004F8F08BD00800040C8AD012008B50D4892
:1093D0000821FFF789FE420708D40A481821FFF741
:1093E00083FE430707D4BFF34F8F08BD064B186AAF
:1093F000FFF796FEF1E7044B186EFFF791FEBFF3FF
:109400004F8F08BD00800040C8AD012008B50D4851
:109410000921FFF769FE420708D40A481921FFF71E
:1094200063FE430707D4BFF34F8F08BD064B586A4E
:10943000FFF776FEF1E7044B586EFFF771FEBFF3BE
:109440004F8F08BD00800040C8AD012008B50D4811
:109450000A21FFF749FE420708D40A481A21FFF7FC
:1094600043FE430707D4BFF34F8F08BD064B986AEE
:10947000FFF756FEF1E7044B986EFFF751FEBFF37E
:109480004F8F08BD00800040C8AD012008B50D48D1
:109490000B21FFF729FE420708D40A481B21FFF7DA
:1094A00023FE430707D4BFF34F8F08BD064BD86A8E
:1094B000FFF736FEF1E7044BD86EFFF731FEBFF33E
:1094C0004F8F08BD00800040C8AD012008B50D4891
:1094D0000C21FFF709FE420708D40A481C21FFF7B8
:1094E00003FE430707D4BFF34F8F08BD064B186B2D
:1094F000FFF716FEF1E7044B186FFFF711FEBFF3FD
:109500004F8F08BD00800040C8AD012008B50D4850
:109510000D21FFF7E9FD420708D40A481D21FFF796
:10952000E3FD430707D4BFF34F8F08BD064B586BCD
:10953000FFF7F6FDF1E7044B586FFFF7F1FDBFF3BE
:109540004F8F08BD00800040C8AD012008B50D4810
:109550000E21FFF7C9FD420708D40A481E21FFF774
:10956000C3FD430707D4BFF34F8F08BD064B986B6D
:10957000FFF7D6FDF1E7044B986FFFF7D1FDBFF37E
:109580004F8F08BD00800040C8AD012008B50D48D0
:109590000F21FFF7A9FD420708D40A481F21FFF752
:1095A000A3FD430707D4BFF34F8F08BD064BD86B0D
:1095B000FFF7B6FDF1E7044BD86FFFF7B1FDBFF33E
:1095C0004F8F08BD00800040C8AD01202DE9F84F45
:1095D000002900F0ED804B6813F0F00F14D0774BAA
:1095E000984214D003F58053984200F0D58003F5DB
:1095F0008053984200F0D58003F5FE23984200F096
:10960000D5806F4802F0D6F80120BDE8F88F6D4A8A
:10961000136843F0807313600B7BDFF8A0C16A4FBF
:109620006A4EDFF8B8E15B0103F0600343F0050325
:109630004365D0F858A0D1F80480446E4AF0080978
:109640000022012514E0B84200F09680B04200F0FC
:10965000938070450CBF4FF0040B4FF07F0B5B45C0
:1096600002F101020DD2DB00053305FA03F31C43BE
:109670006045D3B2E7D14FF0040B5B4502F1010224
:10968000F1D34466D0F88C3018F0800F16BF43F445
:10969000FD5343F0B40343F0140318F0700F10D0DF
:1096A00018F0100F18BF4AF0180918F0200F18BF53
:1096B00049F0200918F0400F43F4F81318BF49F09F
:1096C00040093E4C8A68C0F85890A042C0F88C30DF
:1096D0000AD03D4B984252D003F5805398424ED069
:1096E00003F5FE23984266D1D0F88C3043F0040392
:1096F000C0F88C30456E6FF0FF0645F02035FF2333
:109700004566D0F89840134034402343C0F8983061
:10971000836D8E7ED4054CBF43F0020323F0020319
:1097200092054CBF43F0010323F0010383650B78DE
:1097300003F00703D1E9044503604A789201D2B2ED
:1097400042EA4622C0F884200B7EC3654B7E036745
:10975000C5668B7B9B0104F03F02DBB2134383663B
:109760004B7BC26F1B0222F4706203F470631343DD
:10977000C3670020BDE8F88F4FF0010B6FE7D0F80A
:109780008C3043F00403C0F88C30456E6FF0030654
:1097900045F020050323B3E70A4A136843F000733A
:1097A00039E7084A136843F0806334E7084AF4E76E
:1097B000084801F0FFFF084801F0FCFF008003406B
:1097C00040CD00003C8004400090034000A00340D6
:1097D0003080044028CD00006CCD000000900B408C
:1097E0002DE9F04F83B0DDE90C57002900F0D1805E
:1097F000002F00F0D780002D00F0D180002A00F06B
:10980000CB806B4CA0420CD004F58054A04208D011
:1098100004F58054A04204D004F5FE24A04240F098
:10982000C4800468012B04F0070427FA04F70468D5
:1098300000F0A880B7FBF5F724F02004013F046096
:10984000B7F5803F80F0848002F1FF3C5FFA8CFC2A
:1098500005224FF0010802FB0C1CDFF854A1DFF8D1
:109860006C918760114407EB08020CF10A0C01921D
:10987000BE4611F8035C642D6AD8012B11F8054C23
:1098800047D9504561D04B4A904265D002F580528D
:10989000904261D002F5FE22904256D011F8022C7F
:1098A000642A55D822B10EFB02F2A9FB02625209CA
:1098B000002D47D00EFB05F5A9FB0565BEEB551F36
:1098C0004FEA551796BF019DBF18AF1800EB04155E
:1098D00011F804BCEE6826F03C0646EA8B06EE6002
:1098E0006E6926F03C0646EA8B066E61D0F864B0DD
:1098F000E40008FA04F646EA0B06032B46662A61E2
:10990000AF612BD005316145B3D1002003B0BDE874
:10991000F08F00EBC40411F8046CE26822F03C0202
:1099200042EA860242F02002E2604DB10EFB05F5EC
:10993000A9FB0552BEEB521F4FEA521598BF019D7D
:109940002561DFE72A462F46C0E704229442A5D3CB
:10995000012003B0BDE8F08F0122F7E7466E11F851
:10996000015C621C08FA02F2324342660434426E21
:1099700008FA04F415B114434466C3E722EA040468
:109980004466BFE744F020046D000460B7FBF5F7C0
:1099900056E7094801F00EFF084801F00BFF0848A0
:1099A00001F008FF074801F005FF074801F002FF3A
:1099B000008003400090034090CD0000FCCD0000EB
:1099C000D8CD0000B4CD000020CE00001F85EB51A3
:1099D00008B5C2B113784BB153787BB9012303FAB0
:1099E00001F1816043691943416108BD4369012266
:1099F00002FA01F123EA0101416108BD012303FAE2
:109A000001F14160EEE7014801F0D4FE5CCE0000B8
:109A100008B50F4B98420ED0403398420FD04033D8
:109A200098420ED0403398420DD0403398420CD02B
:109A3000084801F0BFFE084BD3F8A00008BD074B53
:109A4000FAE7074BF8E7074BF6E7074BF4E700BFE9
:109A500000F00F4080CE00000090044000A00440C1
:109A600000B0044000C0044000D0044008B50F4BD3
:109A700098420ED0403398420FD0403398420ED0D7
:109A8000403398420DD0403398420CD0084801F042
:109A900091FE084BC3F8A01008BD074BFAE7074B2F
:109AA000F8E7074BF6E7074BF4E700BF00F00F407D
:109AB00080CE00000090044000A0044000B00440AC
:109AC00000C0044000D00440C27810B5847802F091
:109AD000100304F02002134314BF034B034B1B6815
:109AE0009847BFF34F8F10BD58AE01205CAE0120E8
:109AF0004A0603D5837843F0400383708B0605D56F
:109B0000837903F0AF0343F020038371704700BFF4
:109B10004FF0000C2DE9F043E146E0464FF0FF3EE8
:109B2000174E0024142309E0774502D2BE46A14611
:109B3000E0460134402C14D036F8023F03FA0CF30F
:109B4000B2FBF3F38B42A3EB0105A1EB0307EBD3CD
:109B50007545EED26DB1A1460134402CAE46E046CB
:109B6000EAD1BCF1020F02D00CF1010CD8E74C464F
:109B7000C44644EA8C14E4B24470BDE8F08300BFEC
:109B8000FCCF000070B5002951D0002A4CD0294BE1
:109B900098420C460ED003F5805398423BD003F513
:109BA000FE2398423AD003F58053984239D0224898
:109BB00001F000FE214D402329681943296000234C
:109BC0005021FF26037043708370C670437181710A
:109BD000C371837803F07F03837083790B438371B0
:109BE0008379122143F050038371C1706168FFF7DC
:109BF0008FFF83796178227A03F07F0343EAC113F0
:109C000003F0F00302F00F02134383712378DB01AA
:109C1000DBB2837070BD094D8023CDE7084D402332
:109C2000CAE7074D8023C7E7064801F0C3FD064891
:109C300001F0C0FD00600640B4CE00003480044056
:109C40002880044010CF0000E8CE000010B4C37894
:109C5000847964068479DBB248BF43F48043E40628
:109C600048BF43F480539B0613D4837843F03003FA
:109C70008370962300BF013BFCD14900012A14BF29
:109C80000A4641F00102D2B202715DF8044B184657
:109C9000704740F24C405DF8044B704710B4C378F5
:109CA000847964068479DBB248BF43F48043E406D8
:109CB000847848BF43F48053A40601D49B061FD484
:109CC000437803F03F0444708478DBB244F014041A
:109CD0008470437000BF00BF00BF00BF00BF00BF63
:109CE000962300BF013BFCD14900012A14BF0A465C
:109CF00041F00102D2B202715DF8044B1846704780
:109D000040F24C405DF8044B704700BF70B582B024
:109D1000002900F0328104460220E0700B7FE278D7
:109D20000D4600218DF80710032B6969D2B24CD083
:109D3000052B14D09DF807100131C9B2D6068DF855
:109D4000071000F1D380D0072BD4012B4ED0023B5B
:109D5000032B00F21A81DFE803F0A598835901294B
:109D600035D09DF807100131C9B28DF80710D10622
:109D7000E9D51023E3702B685B0740F24F4214D5FE
:109D800000232B77A37803F0BF03A3702E6A002E65
:109D90003AD06B6A20462946B44602B0BDE870400E
:109DA0006047012B1FD040F24E42A3789806E7D5BA
:109DB000A178774B01F0C701A17002E0013B00F0F0
:109DC000C880E1788906DBD5F8E70029C9D19DF87C
:109DD00007100131C9B2D0068DF80710C9D4D107D8
:109DE000B3D5012BB3D140F25142DEE72B7B002BE0
:109DF00034D002222A77013BAA68DBB22B73DB0046
:109E000022FA03F3DBB2237102B070BD6B695A1EF4
:109E10006A61002BF8D06A69002A40F08B802B68B9
:109E2000590700F1A280A278594B02F0C702A27034
:109E300002E0013B00F09E80E27812F02002F8D1AF
:109E400021792B6919702B6901332B616B69012B07
:109E500000F096802B685E0792D4A6E76B7993B1E9
:109E6000A37803F0E703A3702379DBB28DF8073002
:109E70006B69012B03D1A37843F00803A37005237A
:109E80002B7702B070BD03232B776B69002B42D078
:109E90002B691B7823712B6901332B616B69013BA3
:109EA0006B61B1E72B7B002BA5D16B792BB96B696B
:109EB0008BB303222B692A77EBE70122297920460D
:109EC000FFF7ECFE042302462B7700289CD02B687A
:109ED0005E077FF56AAF40F24E4398423FF463AFAE
:109EE00040F2514398423FF47EAF49E71021012BE5
:109EF000E1707FF440AFD2073FF575AF2B7B8BB994
:109F00006B794BBB2B6803225E072A7740F24F42E6
:109F10007FF54BAF34E72B685B074FF000027FF50E
:109F200044AF2DE72B6828775B0740F24F427FF55F
:109F30003CAF25E722792B691A702B6901332B611D
:109F40006B69012B7FF460AFA37843F00803A37023
:109F50005AE74FF48A6213E72B68042258072A77DE
:109F600040F24F427FF521AF0AE7A37843F0100398
:109F7000A37065E74FF48A6262E7064801F01AFCB5
:109F8000A37843F00803A37064E7034801F012FCD0
:109F9000A086010034CF000058CF00008378084A23
:109FA00003F0C703837001E0013A05D0C37813F0D2
:109FB0002003F9D1184670474FF48A60704700BFFC
:109FC000A0860100C37881790246D8B29379490608
:109FD00048BF40F48040DB0648BF40F480507047E3
:109FE00070B4234C01E0013C38D0C5782D06FAD579
:109FF0000226C670847844F010048470551EDAB1CD
:10A0000011F8014B1A4A047101E0013A26D0C478D4
:10A01000A407FAD5C278C670D4B2D20608D51023E8
:10A02000C370E30700D5FDB940F24F4070BC7047E4
:10A03000E40717D4013DE3D25D070CD40223C370BB
:10A0400082780B4B02F0C702827001E0013B05D021
:10A05000C2789606FAD4002070BC70474FF48A602C
:10A0600070BC7047002DE7D00123C370E6E700BF46
:10A07000A086010070B483B000248DF807409DF8DD
:10A0800007602D4C0136F6B205468DF8076001E0F9
:10A09000013C33D0EE783606FAD50220E870A87875
:10A0A00000F0E700A8702879012AC0B28DF80700F7
:10A0B00039D0501E002A3CD002261F4A01E0013A46
:10A0C0001CD0EC78A407FAD560B95B071DD5AB7836
:10A0D00043F01003AB700223EB702B790B7003B0CD
:10A0E00070BC7047EE702A7901F8012B01280AD163
:10A0F000AA7842F00802AA700020DEE74FF48A60D6
:10A1000003B070BC70470138D7E7AA780A4B02F059
:10A11000C702AA70E87810F02000DCD0013BF9D12A
:10A120004FF48A60D7E7AA7842F00802AA700020AC
:10A13000C2E71046D3E700BFA0860100F8B591B38F
:10A140000C461A49884217461E460DD0184B9842B5
:10A1500023D003F5FE23984221D003F58053984283
:10A160001FD0144801F026FB00252822002120469C
:10A1700001F031FD1048114A114B124940F82540B9
:10A18000C4E908765B5711600F4903F01F000122F4
:10A190005B09824041F82320F8BD0125E5E702254F
:10A1A000E3E70325E1E7094801F004FB006006400E
:10A1B00000700640B4CE000048AE012058AE012029
:10A1C0007CD000000D9D000000E100E070CF000099
:10A1D000F8B500296AD01646002A64D00B7F0C46D9
:10A1E00013B140F24C40F8BD94460546BCE80F0060
:10A1F000274696F805E00FC79CE8030087E80300B0
:10A20000237B7269A261E3B1012372792377AB7971
:10A2100043F05003AB71AB79122143F05003AB71A3
:10A22000E9702368012A08BF4FF0000EDF0732D41F
:10A2300021799C077246284628D5FFF72FFDF8B1F3
:10A24000F8BD01232377AB7943F05003AB71AB79B1
:10A25000122243F05003AB71EA702368DA07E7D5A6
:10A26000BEF1000F1DD103232377124B01E0013B08
:10A2700014D0EA781606FAD521462846FFF746FD9F
:10A28000AB7843F04003AB700020F8BDFFF7DEFC75
:10A290000028D5D1F4E702232377E6E74FF48A605C
:10A2A000F8BD0420F8BD044801F084FA034801F029
:10A2B00081FA00BFA0860100B8CF000094CF000053
:10A2C00000B583B0002947D000228DF807209DF803
:10A2D00007300133DBB28DF80730837803F0BF031A
:10A2E00083700A7783789B062CD54B79012B10D08D
:10A2F0001B4B01E0013B2AD0C2789207FAD502231A
:10A30000C370837803F0C7038370002003B05DF847
:10A3100004FB8278124B42F00802827001E0013B9C
:10A3200015D0C2789107FAD50223C370837803F061
:10A33000C703837003790020DBB28DF8073003B0C8
:10A340005DF804FB40F24C4003B05DF804FB4FF4B1
:10A350008A6003B05DF804FB024801F02BFA00BFED
:10A36000A0860100D8CF0000024B0348D968FFF750
:10A37000ABBB00BF48AE012000700E4008B5044AD8
:10A38000044B11681B6804489847BFF34F8F08BD02
:10A3900060AE012064AE012000400C4010B531B326
:10A3A000144B984202D0144801F004FA134A13687F
:10A3B00043F400031360036823F0020303600023E7
:10A3C00000EB03140133D4F80821042B22F0070218
:10A3D000C4F80821F4D10B7823B1036823F00103FA
:10A3E000036010BD036843F00103036010BD04481F
:10A3F00001F0E0F900700340A0D000003C80044070
:10A4000080D000004B6830B4456C9C07EDB203D09F
:10A4100023F0030304334B608C6804FB03F4B5EBB7
:10A42000940F4FEA940303D29B1AAB4228BF2B46EA
:10A430006BB1C9689C1801EB820201EB8401036ACD
:10A4400042F8043B8A42FAD1204630BC7047144699
:10A45000204630BC704700BF4B6830B4456C9C0749
:10A46000C5F3074503D023F0030304334B608C6826
:10A4700004FB03F4B5EB940F4FEA940303D29B1A49
:10A48000AB4228BF2B466BB109699C1801EB8202D5
:10A4900001EB840152F8043B03628A42FAD1204660
:10A4A00030BC70471446204630BC704770B541B38D
:10A4B0004B7A0269456984690BB3032BCA600FD0DC
:10A4C000C86960B1082B1AD84FF4A37121FA03F3BD
:10A4D000DB0714D5104240F2A66008BF002070BD13
:10A4E000C369260E100E46EA03262B0E43EA042407
:10A4F00040EA0525C1E9045412028E61CA600020B9
:10A5000070BD014801F056F9D4D00000F8B500291B
:10A5100000F08880046B836B1C4014F0C00F0D4664
:10A52000064644D1444B234093B9444B1C4231D19D
:10A53000E20504D56B6913B1296A30469847630771
:10A5400004D5AB6913B1296A304698473463F8BD26
:10A550006B68002B69D014F4702F02D02B68002B8D
:10A5600056D069683046FFF7A1FFEF69002840D157
:10A570002FB12B6A40F2A96229463046B847B36B27
:10A5800023F4702323F00103B3632C4B00221C42FD
:10A590006A60CDD02B68002B4AD0AA682B685B7804
:10A5A0006BB9274B1C420AD040F2A7620FE063064A
:10A5B0001BD40B69002BB5D0296A9847B2E7A706D0
:10A5C00020D4E00628D4A107B2D540F2AA62EF69F0
:10A5D000002FADD02B6A29463046B847B16B194BD6
:10A5E00000220B40B3632A60A2E7CB68002BE3D1C3
:10A5F00098E7002FC3D02B6A40F2A6622946304666
:10A60000B847BCE729683046FFF7FCFEA860DAE7E8
:10A61000EF69002FEFD1A4E729683046FFF71CFF50
:10A62000A860D0E7084801F0C5F8084801F0C2F872
:10A63000074801F0BFF800BF01000F0032007001B1
:10A6400000007011CDFF8FEEF8D000001CD100008B
:10A6500048D1000038B500294AD08B78012B44D06E
:10A660008B68013B7F2B3DD84B68013B7F2B36D855
:10A67000214B984202D0214801F09CF8204A0C78E6
:10A68000136843F400331360C36A43F0E063C362AA
:10A69000836A456C23F44E700CB140F008004B788F
:10A6A0008A780C7989681B01120205F0FF2502F4F3
:10A6B0004072090403F030032C43134301F47F017B
:10A6C0000D4A104D2143034351649362D36A002124
:10A6D00043F00703D36255639163156338BD0A489D
:10A6E00001F068F8094801F065F8094801F062F8DE
:10A6F000084801F05FF800BF00100B4090D2000046
:10A700003080044037017F1130D20000CCD10000EE
:10A7100094D1000070D1000010B4C46A01F0E0636D
:10A720002343C362C36A194205D052B1C36A0B42C4
:10A7300002F1FF32F9D1101E18BF01205DF8044B61
:10A74000704710465DF8044B704700BFF8B500290C
:10A750005DD0002A58D0914256D3B1FBF2F6B6F53F
:10A76000805F4FD8B1FBF6F3934288BF0136102EBD
:10A77000044641D933094FF4807000E00133B0FB47
:10A78000F3F203FB02F2B2F5807FF7D1012BF5D093
:10A79000B6FBF3F202FB03F5AE4206D91D44284690
:10A7A000864202F101021D44F9D84FEAC31C012A76
:10A7B0000CF47F4C104638BF0120B1FBF0F1B1FB27
:10A7C000F3F012B1013A1201D2B2E76A27F008079A
:10A7D000E762E56A25F47F2525F47F652A4342EA8E
:10A7E0000C0242F46022E262626A1307FCD5E26A5C
:10A7F00042F00802E262F8BD32464FF0000CB1FBB5
:10A80000F6F0DEE70020F8BD024800F0D3FF024872
:10A8100000F0D0FFE8D20000C4D20000C36A43F0C9
:10A820000063C362C36A1A0105D541B1C36A1B0143
:10A8300001F1FF31F9D4081E18BF01207047084606
:10A84000704700BFF8B5D1B10D68B5F5005F1CD2F7
:10A850004C68B4F5803F15D2D1E9033742688E6861
:10A860000B4902F460421B062A4303F07C53394033
:10A8700042EA04420B4342608660C360F8BD05486B
:10A8800000F098FF044800F095FF044800F092FFA4
:10A890003700FB0030D30000BCD3000054D30000CD
:10A8A00030B50C46497A012987B037D0022910D03B
:10A8B000032945D00D1F012D3FD906292ED0072988
:10A8C00007D008292AD009290CBF4FF4D01500253C
:10A8D00001E04FF4D815217A032908BF45F440055B
:10A8E0002AB345F400150BB145F00105D3680BB14F
:10A8F00045F010059368012B03D91178D1B945F0C3
:10A9000022055268CDE90123D4E9003201A9CDE93D
:10A9100003230595FFF796FF07B030BD217A4FF46A
:10A92000D015032908BF45F44005002AD9D1CDE947
:10A930000122E9E745F02605E3E74FF40035CAE7D1
:10A940004FF41025C7E700BF2DE9F043DDE90745C7
:10A9500052B14BB15CB155B1012908D002290AD0DE
:10A9600000231846BDE8F0834E1E012EF2D80423C2
:10A970001846BDE8F08314F00301A4462FD1AE07BA
:10A9800018BF25F00305184F18BF0435A7FB05674E
:10A99000FF0BC3F35C037E1C9E4223D8DFF84C9070
:10A9A00002F1040E4FF6FC7800E01946A4EB0C030C
:10A9B000A5EB83031E04B3F5803F46F023064EF853
:10A9C000314032BF42F8316042F8319044448F4206
:10A9D00001F10103E9D1002303608265C8E74FF468
:10A9E000D563C5E70323C3E7018000802100FCFF96
:10A9F000F8B521B315462AB30C4607462422002198
:10AA000020461E4601F0E7F8D5E90012A8680F4B72
:10AA1000E160D5E903159F42C4E90420C4E90615A5
:10AA2000266202D00A4800F0C5FE0A490A4B0B4ACA
:10AA30000C601A600A4B4FF400329A60F8BD094866
:10AA400000F0B8FE084800F0B5FE00BF00100B4053
:10AA500090D2000068AE01206CAE01200DA5000070
:10AA600000E100E024D4000048D400002DE9F043C8
:10AA700083B00A9D002D62D0D5E900780446806A33
:10AA8000C0F301294D46B8F1000F39D00E46002F12
:10AA90003AD0B968B1F5803F32D2606AC00736D487
:10AAA000606A800733D47AB1D7F80CC0BCF1000FCC
:10AAB0003CD07868CDF800C000FB01F10191204640
:10AAC0002946FFF741FF38BB0023C6F804803760F2
:10AAD000B36033686BB31B4A1B4BB9F1000F0CBF5B
:10AAE000002513462363A26B1343A36320462B4622
:10AAF0003A464146FFF7D4FE002003B0BDE8F0839C
:10AB0000042003B0BDE8F083636ADB07DCD540F2C4
:10AB1000A46003B0BDE8F0830020C6F8048037606D
:10AB2000B06035682DB1084B0546DBE7D7F810C09B
:10AB3000BFE7064A2263A36B1343A363D6E7044827
:10AB400000F038FE03007F1133007F0101000F0089
:10AB50006CD4000008B5064B196831B1054B0648A6
:10AB60001B689847BFF34F8F08BD044800F022FED2
:10AB700068AE01206CAE012000100B4090D40000A4
:10AB800002460020537803F09F0343F060035370A4
:10AB9000704700BF70B5002900F0C3800B68002B20
:10ABA00000F0BC80634CA04211D004F58054A04258
:10ABB0000DD004F58054A04207D004F58054A04283
:10ABC00003D004F5FA24A0420AD1012400E00824AD
:10ABD0008D79A54200F3AB80CD79A54200F3A48026
:10ABE000B2EB031F4FEA031432BF2025B2FBF4F48B
:10ABF00065014FEA4202B2FBF3F6B2FBF6F2A6EBB6
:10AC000005054D4E38BF0124934234BFD21A9A1A1B
:10AC1000A6FB03635B0903EB4303934215D3454B48
:10AC2000984215D003F58053984267D003F58053BE
:10AC3000984267D003F58053984267D003F5FA2312
:10AC4000984267D03D4800F0B5FD40F2F53070BD48
:10AC50003B4A4FF48066136833431360C37803F0B4
:10AC6000F303C370037803F0E00343EA1423DBB279
:10AC7000E4B203704470837A05F01F0503F0E0032B
:10AC80001D4385728A7A83780C79920002F004025F
:10AC900003F0E803134314B1234343F0100383701C
:10ACA0004B7902785B0103F0200302F0DF021343CB
:10ACB00003708B79C374CB794375037C43F08803AD
:10ACC0000374437C43F0C00343740B7A1BB1437B92
:10ACD00043F0080343734B7A1BB1437B43F00103FA
:10ACE0004373C378CA7ADBB20AB143F008030A7B24
:10ACF0000AB143F00403C370002070BD104A4FF442
:10AD00000066A8E70E4A4FF48056A4E70C4A4FF4B9
:10AD10000056A0E70B4A4FF480669CE70A4800F013
:10AD200049FD0A4800F046FD094800F043FD094886
:10AD300000F040FD00A006401F85EB51BCD4000090
:10AD4000348004402880044004D50000E8D400008A
:10AD500084D500002CD5000008B5054A054B1168C4
:10AD60001B6805489847BFF34F8FBFF34F8F08BD4F
:10AD700070AE012084AE012000A0064008B5054A4F
:10AD8000054B51681B6805489847BFF34F8FBFF3C9
:10AD90004F8F08BD70AE012084AE012000B0064088
:10ADA00008B5054A054B91681B6805489847BFF3ED
:10ADB0004F8FBFF34F8F08BD70AE012084AE0120CE
:10ADC00000C0064008B5054A054BD1681B68054818
:10ADD0009847BFF34F8FBFF34F8F08BD70AE012070
:10ADE00084AE012000D0064008B5054A054B116924
:10ADF0001B6805489847BFF34F8FBFF34F8F08BDBF
:10AE000070AE012084AE012000A00E40704700BF4C
:10AE10000A4938B5D1F88820094B4CF2205542F444
:10AE200070024DF628144FF4E970C1F88820DD81D6
:10AE3000DC811880FFF7EAFF38BD00BF00ED00E0BD
:10AE40000020054008B538B1002343730173036047
:10AE500083604360184608BD014800F0ABFC00BFAA
:10AE6000DCD50000EFF3108272B68368194381606D
:10AE700082F3108800207047EFF3108272B6836867
:10AE800023EA01018160836882F310880020704703
:10AE9000F0B4049EFEB10446EFF3108772B68568E5
:10AEA0000D40356052B94DB1237B0020012B6073FA
:10AEB0000DD1A36823EA0101A16008E08D42F3D01F
:10AEC00043F2DF7243F2DE70002B18BF104687F3A7
:10AED0001088F0BC704743F2DD70F0BC704700BFD3
:10AEE00010B5134CAA2323702046FFF749FE2046D5
:10AEF000C378802BFCD10F4A0F49104841F244031C
:10AF0000D150FDF773FF0E4B0E480F4A1A600378BD
:10AF10000E4A03F0C703002103700846FDF7E2FF65
:10AF20000B48FDF7D1FD0B4B0B4A1A6010BD00BF5B
:10AF300000E00740007004400000260214D6000024
:10AF4000BCAD0120004006400024F40010D60000F3
:10AF50001CD60000340000200095BA0AFFF7C0BFDD
:10AF60002DE9F043944CDFF8D492944D944EDFF8E1
:10AF7000D082944F83B02046FDF7F8FF48469249AF
:10AF8000FEF756F8237803F0C00343F0280323703C
:10AF9000237843F080032370484600210024FEF705
:10AFA00095F88A4A48460021FDF7F4FF284688496B
:10AFB00089F81B40FDF7CAFB2B6A23F040032B6284
:10AFC00021462846FDF786FC21462846FDF778FCF9
:10AFD0002846FDF729FC2B6A7E4A43F004032B62C6
:10AFE00028462146FDF782FC30467B49FDF7AEFB43
:10AFF000336A23F04003336230460421FDF76AFCD4
:10B0000021463046FDF75CFC3046FDF70DFC734AE7
:10B0100030462146FDF76AFC71494046FEF7D6FAF4
:10B020000220FDF721FE43F6381605220190234643
:10B030006C4900964046FEF7D3FBD8F800306A49C9
:10B0400023F0180343F00803C8F800303846FEF731
:10B05000BDFA0220FDF708FE0222CDE9006023467A
:10B0600062493846FEF7BCFB3B68614923F0180390
:10B0700005F5FC2543F008033B602846FEF7A6FAD9
:10B080000220FDF7F1FD2346CDE90060594928462D
:10B090000422FEF7A5FB2B6823F0180343F00803F6
:10B0A0002B60554E4FF0804373604FF00043736048
:10B0B0000220FDF7D9FD514902465148FEF762FDD5
:10B0C0000220FDF7D1FDA5F5A42502464D492846ED
:10B0D000FEF758FD28464021FEF70AFD4FF00073A9
:10B0E00033600220FDF7C0FD474902464748FEF79E
:10B0F00049FD0220FDF7B8FD07F52D27024644491A
:10B100003846FEF73FFD4349DFF838C1C1F810C0AB
:10B11000384640278F800127A5F5403523463E4A13
:10B120008C600C730C604F613C49FFF707F82846B0
:10B130003B49FFF733F93B483B493C4A3C4BC5F898
:10B140000001C5F81011C5F82021C5F83031D5F837
:10B15000083143F00203C5F80831D5F8183143F03F
:10B160000203C5F81831D5F8283143F00203C5F8B9
:10B170002831D5F83831A02243F00203C5F8383120
:10B1800086F8314386F832234FF4803373604FF4EE
:10B19000003373604FF4802373604FF400237360B7
:10B1A0002046FDF761FD23490246234803B0BDE870
:10B1B000F043FFF7EFBC00BF0010024000B00340B7
:10B1C00000B00B4000A003403CD6000080D7000038
:10B1D00024D600003800002030D6000040000020B7
:10B1E00040D600005CD6000078D6000094D600005F
:10B1F000A0D60000BCD6000000E100E0D0D60000E0
:10B2000000600640DCD60000E8D6000000600E407A
:10B21000F4D60000B4AE0120AD1600008CAE0120C3
:10B2200000D700001FBF02008F5F01007FC3C9016C
:10B23000FF6BDC0204D7000000A006400080004045
:10B240000080034088AE0120FFF78ABEC24BC3488E
:10B250001A6842F40072F0B51A601A68C04FC14E05
:10B2600042F480621A601A6842F400621A601A6836
:10B2700042F480521A601A6897B042F400521A6081
:10B28000012401AA0521ADF80440FEF7A1FB02AAA2
:10B29000B248ADF808400E21FEF79AFB03AAAF486A
:10B2A000ADF80C400F210025FEF792FB04AAAB4835
:10B2B000ADF810501021FEF78BFB05AAA748ADF89A
:10B2C00014401121FEF784FB2946384606AAADF842
:10B2D0001840FEF77DFB2146384607AAADF81C4012
:10B2E000FEF776FB384608AA0A21ADF82050FEF793
:10B2F0006FFB384609AA0B21ADF82440FEF768FB26
:10B30000294630460AAAADF82840FEF761FB3046D0
:10B310000BAA0321ADF82C40FEF75AFB30460CAACD
:10B320000421ADF83040FEF753FB30460DAA05214D
:10B33000ADF83440FEF74CFB30460EAA06218037AC
:10B34000ADF83840FEF744FB30460FAA0721ADF8B0
:10B350003C40FEF73DFB2146384610AAADF8405070
:10B36000FEF736FB384611AA02218036ADF844407C
:10B37000FEF72EFB384612AA0621ADF84850FEF71C
:10B3800027FB304613AA1821ADF84C50FEF720FBDE
:10B39000304614AA1921ADF85040FEF719FB30468B
:10B3A00015AA1A21ADF85440FEF712FB6E496F4CF6
:10B3B0000D6B6F486F4E704B704A25F4E06545F495
:10B3C000A0650D630D6B254045F021050D634D6BA8
:10B3D00025F4E06545F4A0654D634D6B254045F0CF
:10B3E00021054D638D6B25F4E06545F480758D6313
:10B3F000CD6B25F4E06545F48075CD630D6C25F4C7
:10B40000E06545F480750D640D6C054045F003055D
:10B410000D644D6C25F4E06545F480754D644D690F
:10B4200025F4E06545F480754D614D6935404D6109
:10B430001D6825F4E06545F480751D605D6825F4A0
:10B44000E06545F480755D609D6A25F4E06545F42E
:10B4500080759D629D6A054045F003059D62DD6A29
:10B4600025F4E06545F48075DD621D6C25F4E0652A
:10B4700045F440751D645D6C25F4E06545F4407548
:10B480005D649D6C25F4E06545F440759D64DD6C5C
:10B4900025F4E06545F44075DD649D6825F4E065BC
:10B4A00045F400759D609D68254045F021059D602F
:10B4B000DD6825F4E06545F40075DD60DD68254054
:10B4C00045F02105DD60156825F4E06545F48075DB
:10B4D0001560556825F4E06545F480655560956A0A
:10B4E00025F4E06545F400759562956A254045F0C0
:10B4F00021059562D56A25F4E06545F40075D562AD
:10B50000D56A254045F02105D562956825F4E065AA
:10B5100045F480659560D56825F4E06545F480754F
:10B52000D560156925F4E06545F4807515611569E8
:10B5300005401561556925F4E06545F48075556150
:10B54000956925F4E06545F480759561956925F068
:10B55000807525F0200513E03880044000F00F408E
:10B5600040F00F4080F00F4000900440DEFFFFFEEF
:10B57000FCFFFFFEFEFFFFFE00A0044000B0044001
:10B580009561D56925F4E06545F48075D561156A46
:10B5900025F4E06545F440751562556A25F4E065CB
:10B5A00001F5405145F440755562D1F8C020694D10
:10B5B00042F04202C1F8C0200A6822F4E06242F47C
:10B5C00080620A604A6822F4E06242F480724A6053
:10B5D0004A6822F4702242F420224A604A680240FB
:10B5E00042F003024A608A6822F4E06242F4807208
:10B5F0008A60CA6822F4E06242F48062CA600A6922
:10B6000022F4E06242F480620A614A6922F4E06254
:10B6100042F480624A618A6922F4E06242F48072F4
:10B620008A618A6922F4702242F420228A618A693E
:10B6300022F0807222F0230242F003028A61CA697A
:10B6400022F4E06203F5405342F48062CA611A6852
:10B6500022F4E06242F480621A601A68024042F00A
:10B6600003021A605A6822F4E06242F480625A606F
:10B670005A68024042F003025A609A6A22F4E06279
:10B6800042F400729A629A6A224042F021029A625F
:10B69000DA6A22F4E06242F40072DA62DA6A144092
:10B6A00044F02104DC62996821F4E06141F4806196
:10B6B00099609A68324042F001029A601A6E22F450
:10B6C000E06242F480721A661A6E22F4702242F42A
:10B6D00020221A661A6E024042F003021A665A6E5F
:10B6E00022F4E06242F480725A669A6E22F4E062BA
:10B6F00042F480729A66DA6822F4E06242F4806270
:10B70000DA60DA68024042F00302DA601A6922F471
:10B71000E06242F480621A611A69024042F0030258
:10B720001A615A6922F4E06242F480625A615A69ED
:10B73000104040F0030041F20C025861AB5823F472
:10B74000E003AB5041F21002AB5823F00303AB50BF
:10B7500017B0F0BD00700440FFF778BD70B5C0B100
:10B760000D4E0E4BF3622023054633630C4B0660EF
:10B77000002014463360FDF777FA2201094B2C684C
:10B7800009497060D2B20948A065296183F8512344
:10B7900070BD074800F00EF8F0AE012054AF012054
:10B7A00000100B4000E100E0CCAE0120E0AE012033
:10B7B00014D7000010B50F4904460F4800F00EFBE7
:10B7C0000C49204600F00AFB0C49D1F88030013BBF
:10B7D000002BC1F8803008DB8B6F5A1C8A670A2265
:10B7E0001A70BDE8104000F00BB878310A2000F064
:10B7F00014FAF6E74CB0012034D70000D4AF012092
:10B8000018200149ABBE7047260002002DE9F04127
:10B81000D5685769EB0280460E46144605D5384672
:10B8200000F0B5FC45F01005A061124B2B408BB128
:10B83000A169384600F0BDFC002806DAE36843F051
:10B840008003E3604FF0FF3011E025F4003525F070
:10B850001005E56032464146384600F0B6FC20F05F
:10B860000041761AA1690E44A6610028E6D1BDE820
:10B87000F08100BF10000200F8B5304E3468002897
:10B8800051D10020F8BD2368B3F1805F39D1D4E9EC
:10B89000013252B11168B1F1805F06D151680333B2
:10B8A0000B4463609368A360F1E7AB4207DB9E45FE
:10B8B00005DB20464FF0005340F80C3BE2E76345C0
:10B8C00011D920464FF00051656040F80C1B5B1BFE
:10B8D00000EB8501A160033B4FF0805440F8254008
:10B8E000C1E90132CEE762B9A0EB830000F016F99E
:10B8F0000130C6D04FF00053C4E9003504F10C000C
:10B90000C0E72746A468002CBDD10C3000F006F932
:10B91000431CB6D04FF00053C0E90035846057B9DE
:10B9200030600C30AEE7C31C9D08002705F10A0CFF
:10B9300005F1030EE7E7B860F3E700BF8CB0012024
:10B9400010B5FFF799FF044628B90449172200F003
:10B950003CFCFFF755FF204610BD00BF49D7000053
:10B960002DE9F843C6683D4B334004460D469046EA
:10B970001BB902273846BDE8F883D0F81490484632
:10B9800000F00BFC07460028F3D1B8F1010F2CD0D2
:10B99000B8F1020F2ED0B8F1000FEAD1002DE8DB8C
:10B9A000B00404D52368E26A9A4238BFE362A16911
:10B9B000A9420EDC2368E26A934238BF134622692B
:10B9C0005818801AA84204DB206B01EB000CAC4530
:10B9D00034DC0023C4E9013346F02006A56226F4D6
:10B9E000032626F04006E660C4E7204600F038F85B
:10B9F0000544D3E7484600F0CAFBB0F1000CE2680A
:10BA000004DA42F08002E2600127B3E723681846B7
:10BA1000A3691946E36A98422CBF0918C9180B4656
:10BA200021699206A3EB010303D5A26A9342B8BF32
:10BA300013466345ACBFED186544AFE76D1AB10717
:10BA400044BF281AA060F10744BF9B1AEB1A1544A3
:10BA500048BF6360256026F02006C0E703001000A1
:10BA6000C3689A0705D10E4B21221A604FF0FF30B0
:10BA7000704703F020021B0309D512B1806A013818
:10BA800070470368826900691344181AF7E70AB11E
:10BA9000806A70470368826900691344181A704706
:10BAA00090B0012010B5174A1749002000F0F1F9B5
:10BAB0004FF480734FF480620021124800F0A4F923
:10BAC000124A1349012000F0E4F94FF480730F4843
:10BAD0004FF48062002100F097F90E4B1B68022B97
:10BAE0000EDD0D4A0A49022000F0D3F9BDE81040EE
:10BAF00009484FF480734FF48062002100F084B94C
:10BB000010BD00BFD4AF012061D7000010B00120EC
:10BB100063D7000030D700004CB0012070B50B4D4A
:10BB20002B680BB90A4B2B6003302E6820F00304FE
:10BB30003444204600F032F810B92C60304670BD15
:10BB4000044B0C221A604FF0FF36F7E788B0012053
:10BB5000B0B0012090B00120F7B5044698B103B011
:10BB6000BDE8F04000F0FFB907FB046000F0FBF90E
:10BB7000002818BF4FF0FF350134019BA342F3DCCE
:10BB8000284603B0F0BD034B034E1B6801930546E6
:10BB90003C27F2E730D70000D4AF0120044B23B19B
:10BBA000984234BF0020012070471846704700BFFC
:10BBB000B0C0012008B5FFF775FFBDE80840F4F7F5
:10BBC0007FBDB5EEC00AF1EE10FA48BFB1EE400AF3
:10BBD000704700F0A3BA00F0BBBAC368826923F0D3
:10BBE000200310B5C360836A9A4204460ED000F069
:10BBF000B4F8E36823F4405323F0100343F0100338
:10BC0000E360A36AA3612369E3622360E36823F42A
:10BC1000804323F04003E36010BDCB6823F400228F
:10BC200070B50C46CA609906054602D52046FFF756
:10BC3000D4FFD4E902365A1C10DAB0050ED4C3F191
:10BC4000FF2303F57F03FE33A360236846F4903699
:10BC50005A1CE66022601D70E8B270BD41F28A0293
:10BC60003240022A07D0002346F08006A360E66037
:10BC70004FF0FF30F1E74AF210033340B3F5004FC5
:10BC80000AD100212046FFF76BFEE368990602D532
:10BC90002046FFF7A2FFE66846F4903316F4706F73
:10BCA000E3600ED1606900F078FA00B372051ED52A
:10BCB00004F12403236123600123E36146F49233FA
:10BCC000E36013F4106F2168266926D0E36A994275
:10BCD0002CBFC6EB0101C6EB0301B9B9731CE362CB
:10BCE0002360E36923635A1EA2603570B4E74FF402
:10BCF0008070FFF725FEE26820614FF48073E361F6
:10BD000046F494331A432060E260DAE72246304674
:10BD1000FFF77CFD0028E1D0AAE74A1CEDB22260C3
:10BD20000D70E26A216891422CBFC6EB0101C6EB9F
:10BD30000201E26922635B0503D40A2D01D08A4225
:10BD400009DC0023E6622660A36022463046FFF746
:10BD50005DFD00288CD128467FE738B5016805696C
:10BD6000C36A0446C06820F40022E26000F0820248
:10BD7000022A02D04FF0FF3038BD10F48030FBD0E3
:10BD8000994238BF19468D4208D1E368E562002028
:10BD900023F480332560A060E360EDE72246491B71
:10BDA0002846FFF733FD0028EFD0E3E7A8B14FF0B6
:10BDB000805340F80C3C50F8042C72B11368B3F176
:10BDC000805F0AD150F8083C516803330B4440F8B7
:10BDD000083C936840F8043CEDE7704738B50546E9
:10BDE0000C4615F8010B70B1A368013B002BA36052
:10BDF00004DB23685A1C22601870F2E72146FFF723
:10BE00000CFF431CEDD138BD70B5C468A50708D040
:10BE1000B2F5007F11D0B2F5806F04D0B2F5807F0B
:10BE20000BD0012008E000F124010123224301612D
:10BE30000160C361C260002070BD5E1E6FF07F456F
:10BE4000AE42F3D3EDE710B5421C8307044616D18A
:10BE5000234654F8041BA1F1013020EA010010F040
:10BE6000803FF5D011F0FF0F11D011F47F4F0CD0AF
:10BE700011F47F0F14BF23460333981A04E010F81F
:10BE8000013B002BE1D1801A10BD0233F5E70133ED
:10BE9000F3E770B50D4606461046144600F02DF83F
:10BEA0002B78722B17D0772B18D0612B23D1082336
:10BEB00048F2020215F8011F2B2912D0622915D071
:10BEC0001B07E260666104D5022200212046FFF7CD
:10BED00047FD204670BD00230122EBE70423022228
:10BEE000E8E742F0030243F00203E3E742F0040212
:10BEF00043F00103DEE70024EBE7F0B5C468A107D7
:10BF000089B0054622D0220718D4D0E90467FFF78C
:10BF100023FE384600F035F9230502D53046FFF7F9
:10BF200045FFA40DA40514F1A54F07D1296A2022CD
:10BF3000684600F044F9684600F00BF83C22002106
:10BF40002846FFF748FE002009B0F0BD4FF0FF3053
:10BF5000FAE710B50446FFF776FF01462046BDE834
:10BF6000104000F020B9C36870B513F00306044612
:10BF700011D09B0611D5856AFFF72FFEE36823F4E5
:10BF80004053E3602046FFF7E8FE002206462946BC
:10BF90002046FFF7E5FC304670BD816905680D4419
:10BFA00001696D1AEAE75FF0000C30B51C0022D180
:10BFB00012006FD0914206D305460846002100F0DA
:10BFC0006FF80446284600F06BF80A462146BDE8A3
:10BFD00030401CF0404F08BF704703D549424042F3
:10BFE00061F100015FEA8C0C38BF70475B4252423E
:10BFF00063F10003704742D41C0C04BF1B040CF116
:10C00000100C13F07F4F04BF1B020CF1080C13F04F
:10C01000704F04BF1B010CF1040C13F0404F04BF20
:10C020000CF1020C5FEA83035CBF0CF1010C5B00B6
:10C03000CCF1200E22FA0EF4234302FA0CF200FA9D
:10C040000CF520FA0EF001FA0CF4204321FA0EF15F
:10C0500014461A4600F024F8A4FB0023AA1A71EB38
:10C0600003033CBF1B190138CCF1200E22FA0CF25D
:10C0700003FA0EF4224323FA0CF30021A7E7821AF5
:10C0800071EB03033CBF02460B464FF0000141F148
:10C0900000009CE700200021BDE8304000F03DB8E2
:10C0A0000423B1EB122F09D2090241EA1061000208
:10C0B000013B08BF7047B1EB122FF5D3001849417F
:10C0C00034BF9142891A4041494134BF9142891A93
:10C0D0004041494134BF9142891A4041494134BFEE
:10C0E0009142891A4041494134BF9142891A4041E5
:10C0F000494134BF9142891A4041494134BF91427C
:10C10000891A4041494134BF9142891A4041A3F103
:10C11000010313F00F0FD2D17047704740EA0103BB
:10C12000DB0703460CD40346043A22BF51F804CB84
:10C1300043F804CBB2F10402F7D2043208BF7047CF
:10C14000013A24BF11F801CB03F801CBF8D87047AE
:10C15000034613F0030F0ED101F0FF0141EA012164
:10C1600041EA0141043A24BF43F8041BB2F104023E
:10C17000F9D202F10402013A24BF03F8011BFAE7E5
:10C18000704703B469460220ABBE02B0704703B4E7
:10C1900069460C20ABBE02B0704703B46946092063
:10C1A000ABBE02B0704703B469460E20ABBE02B00E
:10C1B000704703B469460A20ABBE02B070470FB4A3
:10C1C00069460D20ABBE04B070470FB46946052028
:10C1D000ABBE04B07047FFFF000204000300011073
:10C1E000030200000302010006000400060500200F
:10C1F0000605040020212223242526FF90046853ED
:10C20000180C300C362430061006B60D100430041D
:10C21000FF7F00002B6A82785036685EF87FC77F08
:10C220003F7EFF71FF0F5B04DC46F96FEB6F7B6FA6
:10C23000FB6BFB4F9554352595746E516E5BDB7827
:10C2400002726D11580DAF24AF74AF7ED446927256
:10C250005B04685E5036BF7A7F7500129124714787
:10C26000106D1B465236FFFF0004002217FFFFFF30
:10C270000004002216FFFFFF0004223203FFFFFF2D
:10C28000000800000FFFFFFF0004223214FFFFFF31
:10C290000004002201FFFFFF00040000E1FFFFFF98
:10C2A0000004002202FFFFFF21000000815B030069
:10C2B000E1B6060041120A00A16D0D0001C910008F
:10C2C00061241400C17F170021DB1A0081361E0093
:10C2D000E191210041ED2400A148280001A42B0098
:10C2E00061FF2E00C15A320021B63500811139009C
:10C2F000E16C3C0041C83F00A1234300017F4600A0
:10C3000061DA4900C1354D002191500081EC5300A4
:10C31000E147570041A35A00A1FE5D00015A6100A8
:10C3200061B56400C1106800216C6B0081C76E00AC
:10C33000E1227200417E7500A1D9780001357C00B0
:10C3400061907F00C1EB82002147860081A28900B5
:10C35000E1FD8C0041599000A1B4930001109700B9
:10C36000616B9A00C1C69D002122A100817DA400BD
:10C37000E1D8A7004134AB00A18FAE0001EBB100C2
:10C380006146B500C1A1B80021FDBB008158BF00C6
:10C39000E1B3C200410FC600A16AC90001C6CC00CA
:10C3A0006121D000C17CD30021D8D6008133DA00CE
:10C3B000E18EDD0041EAE000A145E40001A1E700D3
:10C3C00061FCEA00C157EE0021B3F100810EF500D7
:10C3D000E169F80041C5FB00A120FF00017C0201DA
:10C3E00061D70501C1320901218E0C0181E90F01DC
:10C3F000E144130141A01601A1FB190101571D01E0
:10C4000061B22001C10D24012169270181C42A01E3
:10C41000E11F2E01417B3101A1D6340101323801E7
:10C42000618D3B01C1E83E0121444201819F4501EC
:10C43000E1FA480141564C01A1B14F01010D5301F0
:10C4400061685601C1C35901211F5D01817A6001F4
:10C45000E1D5630141316701A18C6A0101E86D01F9
:10C4600061437101C19E740121FA770181557B01FD
:10C47000E1B07E01410C8201A167850101C3880101
:10C48000611E8C01C1798F0121D592018130960105
:10C49000E18B990141E79C01A142A001019EA3010A
:10C4A00061F9A601C154AA0180F00F4000F10F40CC
:10C4B00040F00F4080F00F4000F00F4000F00F40C0
:10C4C00080F00F4000F10F4000F00F4080F00F406F
:10C4D00080F00F4000F00F40050000001900000040
:10C4E0000B00000000000000110000000F00000021
:10C4F000060000001A0000000E000000040000000A
:10C5000007000000050000009C18000064190000EE
:10C51000581B000028230000E02E00002E66736CDC
:10C520005F73642E633A363239203A206361726455
:10C5300000FFFFFF2E66736C5F73642E633A37371C
:10C5400039203A206361726400FFFFFF2E66736C2E
:10C550005F73642E633A353233203A20636172642C
:10C5600000FFFFFF2E66736C5F73642E633A3133F6
:10C570003336203A206361726400FFFF2E66736CCD
:10C580005F73642E633A31343035203A2063617230
:10C590006400FFFF2E66736C5F73642E633A31365E
:10C5A0003239203A206361726400FFFF2E66736C9B
:10C5B0005F73642E633A31363337203A20636172F9
:10C5C000640000002E66736C5F73642E633A31362C
:10C5D0003338203A20627566666572002E66736C89
:10C5E0005F73642E633A31363339203A20626C6FC0
:10C5F000636B436F756E74002E66736C5F73642E8D
:10C60000633A31363430203A2028626C6F636B43D2
:10C610006F756E74202B207374617274426C6F633B
:10C620006B29203C3D20636172642D3E626C6F6318
:10C630006B436F756E7400002E66736C5F73642EAF
:10C64000633A31343337203A20627566666572008A
:10C650002E66736C5F73642E633A31363933203A39
:10C6600020636172640000002E66736C5F73642E39
:10C67000633A31363934203A206275666665720055
:10C680002E66736C5F73642E633A31363935203A07
:10C6900020626C6F636B436F756E74002E66736CF3
:10C6A0005F73642E633A31363936203A2028626C43
:10C6B0006F636B436F756E74202B2073746172749B
:10C6C000426C6F636B29203C3D20636172642D3E98
:10C6D000626C6F636B436F756E7400002E66736CD3
:10C6E0005F73642E633A31343836203A20627566BF
:10C6F000666572002E66736C5F73642E633A313820
:10C700003037203A206361726400FFFF2E66736C3D
:10C710005F73642E633A31393130203A206361729D
:10C72000640000002E66736C5F73642E633A3139C7
:10C730003131203A20636172642D3E6973486F7312
:10C74000745265616479203D3D207472756500FF07
:10C750002E66736C5F73642E633A31393931203A37
:10C7600020636172640000002E66736C5F73642E38
:10C77000633A31393932203A20636172642D3E7553
:10C780007372506172616D2E636420213D204E559D
:10C790004C4C00FF2E66736C5F73646D6D635F6F4E
:10C7A00073612E633A3430203A206576656E7448A2
:10C7B000616E646C6520213D204E554C4C00FFFF9E
:10C7C0002E66736C5F73646D6D635F6F73612E6350
:10C7D0003A3536203A206576656E7448616E646C31
:10C7E0006520213D204E554C4C00FFFF2E66736C9A
:10C7F0005F73646D6D635F6F73612E633A383520CC
:10C800003A206576656E7448616E646C6520213DE2
:10C81000204E554C4C00FFFF2E66736C5F73646DA9
:10C820006D635F6F73612E633A313137203A206553
:10C8300076656E7448616E646C6520213D204E55AE
:10C840004C4C00FF2E66736C5F73646D6D635F68A4
:10C850006F73742E633A333439203A20686F7374DF
:10C8600020213D204E554C4C000000002E66736C7C
:10C870005F73646D6D635F686F73742E633A3335F5
:10C8800030203A20686F73742D3E686F737445765C
:10C89000656E7420213D204E554C4C002E66736C05
:10C8A0005F61646331362E633A3636203A204E5546
:10C8B0004C4C20213D20636F6E66696700000000CC
:10C8C0002E66736C5F61646331362E633A353320B4
:10C8D0003A20696E7374616E6365203C2041525248
:10C8E00041595F53495A4528735F61646331364249
:10C8F000617365732900FFFF2E66736C5F6164636B
:10C9000031362E633A343535203A206368616E6ED5
:10C91000656C47726F7570203C204144435F534300
:10C92000315F434F554E54002E66736C5F616463F4
:10C9300031362E633A343536203A204E554C4C2051
:10C94000213D20636F6E66696700FFFF2E66736C82
:10C950005F61646331362E633A343835203A2063A0
:10C9600068616E6E656C47726F7570203C20414443
:10C97000435F5343315F434F554E54002E66736CF3
:10C980005F636C6F636B2E633A323232203A203031
:10C990005520213D20675F7874616C304672657167
:10C9A000000000002E66736C5F636C6F636B2E6318
:10C9B0003A323237203A20305520213D20675F78C7
:10C9C00074616C33324672657100FFFF2E66736CC2
:10C9D0005F636C6F636B2E633A393931203A206D97
:10C9E0006367706C6C30636C6B00FFFF2E66736C5A
:10C9F0005F636C6F636B2E633A333633203A206784
:10CA00005F7874616C304672657100FF2E66736CDE
:10CA10005F636C6F636B2E633A333835203A20675F
:10CA20005F7874616C304672657100FF2E66736CBE
:10CA30005F636C6F636B2E633A343132203A206748
:10CA40005F7874616C333246726571002E66736C68
:10CA50005F636C6F636B2E633A31323737203A2055
:10CA6000636F6E66696700FF2E66736C5F636C6F41
:10CA7000636B2E633A32323130203A20636F6E6638
:10CA8000696700FF2E66736C5F636C6F636B2E6368
:10CA90003A32353031203A20636F6E66696700FFA5
:10CAA0008002DC020005B80580079508000A710BBA
:10CAB0002E66736C5F636F6D6D6F6E2E633A3234EA
:10CAC00033203A20305520213D2064656C61795F28
:10CAD000757300002E66736C5F636F6D6D6F6E2EE5
:10CAE000633A323435203A20636F756E74203C3DD2
:10CAF0002055494E5433325F4D4158002E66736CB9
:10CB00005F646D616D75782E633A3539203A20691E
:10CB10006E7374616E6365203C2041525241595FCF
:10CB200053495A4528735F646D616D75784261732E
:10CB3000657329002E66736C5F65646D612E633AC0
:10CB40003838203A206368616E6E656C203C20287E
:10CB500075696E7433325F742946534C5F464541A4
:10CB6000545552455F45444D415F4D4F44554C45EA
:10CB70005F4348414E4E454C000000002E66736CEA
:10CB80005F65646D612E633A3839203A20746364BE
:10CB900020213D204E554C4C000000002E66736C49
:10CBA0005F65646D612E633A3930203A202828751C
:10CBB000696E7433325F7429746364202620307880
:10CBC00031465529203D3D20305500FF2E66736CBF
:10CBD0005F65646D612E633A313230203A20636FB5
:10CBE0006E66696720213D204E554C4C00000000C8
:10CBF0002E66736C5F65646D612E633A3734203A3C
:10CC000020696E7374616E6365203C20415252410D
:10CC1000595F53495A4528735F65646D614261737A
:10CC2000657329002E66736C5F65646D612E633ACF
:10CC3000343233203A2074636420213D204E554C19
:10CC40004C0000002E66736C5F65646D612E633A64
:10CC5000343234203A20282875696E7433325F7478
:10CC600029746364202620307831465529203D3DC3
:10CC7000203055002E66736C5F65646D612E633ADB
:10CC8000313936203A206368616E6E656C203C2035
:10CC90002875696E7433325F742946534C5F46457C
:10CCA00041545552455F45444D415F4D4F44554CAD
:10CCB000455F4348414E4E454C00FFFF2E66736C66
:10CCC0005F65646D612E633A373137203A206368BF
:10CCD000616E6E656C203C202875696E7433325F1E
:10CCE000742946534C5F464541545552455F45446F
:10CCF0004D415F4D4F44554C455F4348414E4E4575
:10CD00004C00FFFF2E66736C5F65646D612E633AA5
:10CD100031333135203A2068616E646C6520213DE5
:10CD2000204E554C4C00FFFF2E66736C5F66746D91
:10CD30002E633A323233203A20636F6E66696700A1
:10CD40002E66736C5F66746D2E633A3830203A201D
:10CD5000696E7374616E6365203C2066746D417208
:10CD6000726179436F756E74000000002E66736CFB
:10CD70005F66746D2E633A313532203A202D3120B2
:10CD8000213D2063686E6C436F756E7400FFFFFF7A
:10CD90002E66736C5F66746D2E633A333836203AB4
:10CDA000204E554C4C20213D2063686E6C506172C2
:10CDB000616D73002E66736C5F66746D2E633A331B
:10CDC0003837203A20305520213D20737263436C60
:10CDD0006F636B5F487A00002E66736C5F66746DDC
:10CDE0002E633A333838203A20305520213D2070C8
:10CDF000776D467265715F487A0000002E66736C2D
:10CE00005F66746D2E633A333839203A20305520EE
:10CE1000213D206E756D4F6643686E6C7300000097
:10CE20002E66736C5F66746D2E633A333931203A27
:10CE3000202D3120213D2046534C5F46454154551D
:10CE400052455F46544D5F4348414E4E454C5F430B
:10CE50004F554E546E286261736529002E66736CBF
:10CE60005F6770696F2E633A313030203A204E553B
:10CE70004C4C20213D20636F6E66696700FFFFFF09
:10CE80002E66736C5F6770696F2E633A3637203A8F
:10CE900020696E7374616E6365203C20415252417B
:10CEA000595F53495A4528735F6770696F426173D0
:10CEB000657329002E66736C5F6932632E633A31A5
:10CEC0003539203A20696E7374616E6365203C20A9
:10CED00041525241595F53495A4528735F69326341
:10CEE00042617365732900FF2E66736C5F6932635C
:10CEF0002E633A353636203A204E554C4C20213D93
:10CF0000206D6173746572436F6E6669670000001F
:10CF10002E66736C5F6932632E633A353637203A7A
:10CF200020305520213D20737263436C6F636B5F2B
:10CF3000487A00FF2E66736C5F6932632E633A3164
:10CF4000363532203A204E554C4C20213D20693256
:10CF50006348616E646C65002E66736C5F69326352
:10CF60002E633A353135203A2066616C736500FFD7
:10CF70002E66736C5F6932632E633A313437342026
:10CF80003A204E554C4C20213D2068616E646C6502
:10CF900000FFFFFF2E66736C5F6932632E633A31C8
:10CFA000353132203A204E554C4C20213D206861CD
:10CFB0006E646C65000000002E66736C5F693263FE
:10CFC0002E633A31353133203A204E554C4C2021D6
:10CFD0003D207866657200FF2E66736C5F69326370
:10CFE0002E633A31353530203A204E554C4C2021B5
:10CFF0003D2068616E646C6500FFFFFF1400160041
:10D0000018001A001C001E00220028001C0020002E
:10D01000240028002C003000380044003000380084
:10D020004000480050005800680080005000600038
:10D03000700080009000A000C000F000A000C000C0
:10D04000E0000001200140018001E0014001800179
:10D05000C0010002400280020003C00380020003FE
:10D060008003000480040005000680070005000618
:10D07000000700080009000A000C000F18194A5B9D
:10D080002E66736C5F7069742E633A3730203A20D5
:10D090004E554C4C20213D20636F6E666967000041
:10D0A0002E66736C5F7069742E633A3535203A20B2
:10D0B000696E7374616E6365203C20415252415920
:10D0C0005F53495A4528735F706974426173657391
:10D0D0002900FFFF2E66736C5F736468632E633AEA
:10D0E000333331203A20636F6D6D616E6420213DD2
:10D0F000204E554C4C00FFFF2E66736C5F736468C6
:10D10000632E633A31353734203A2068616E646C9F
:10D110006520213D204E554C4C0000002E66736C5E
:10D120005F736468632E633A373031203A20686158
:10D130006E646C652D3E636F6D6D616E6420213D84
:10D14000204E554C4C0000002E66736C5F73646873
:10D15000632E633A373333203A2068616E646C651E
:10D160002D3E6461746120213D204E554C4C00FFE2
:10D170002E66736C5F736468632E633A38313020B7
:10D180003A20636F6E66696720213D204E554C4CF6
:10D19000000000002E66736C5F736468632E633A50
:10D1A000383132203A20636F6E6669672D3E646DB8
:10D1B000614D6F646520213D206B534448435F44BB
:10D1C0006D614D6F646541646D6131002E66736CF5
:10D1D0005F736468632E633A383134203A202863E1
:10D1E0006F6E6669672D3E77726974655761746505
:10D1F000726D61726B4C6576656C203E3D203155D9
:10D200004C292026262028636F6E6669672D3E779D
:10D210007269746557617465726D61726B4C657685
:10D22000656C203C3D20313238554C29000000000F
:10D230002E66736C5F736468632E633A38313520F1
:10D240003A2028636F6E6669672D3E726561645788
:10D25000617465726D61726B4C6576656C203E3DE4
:10D260002031554C292026262028636F6E66696779
:10D270002D3E7265616457617465726D61726B4CAD
:10D280006576656C203C3D20313238554C290000D4
:10D290002E66736C5F736468632E633A3232382093
:10D2A0003A20696E7374616E6365203C204152526E
:10D2B00041595F53495A4528735F736468634261FB
:10D2C000736529002E66736C5F736468632E633A1E
:10D2D000393433203A20737263436C6F636B5F4859
:10D2E0007A20213D203055002E66736C5F73646890
:10D2F000632E633A393434203A2028627573436CC4
:10D300006F636B5F487A20213D2030552920262607
:10D310002028627573436C6F636B5F487A203C3DD5
:10D3200020737263436C6F636B5F487A2900FFFF61
:10D330002E66736C5F736468632E633A31303833E2
:10D34000203A20636F6E66696720213D204E554C60
:10D350004C0000002E66736C5F736468632E633A42
:10D3600031303834203A20636F6E6669672D3E6431
:10D37000617461426C6F636B53697A65203C3D2038
:10D3800028534448435F424C4B415454525F424CF3
:10D390004B53495A455F4D41534B203E3E20534429
:10D3A00048435F424C4B415454525F424C4B5349AB
:10D3B0005A455F5348494654290000002E66736C55
:10D3C0005F736468632E633A31303835203A2063E6
:10D3D0006F6E6669672D3E64617461426C6F636B4A
:10D3E000436F756E74203C3D2028534448435F4290
:10D3F0004C4B415454525F424C4B434E545F4D4151
:10D40000534B203E3E20534448435F424C4B4154D3
:10D4100054525F424C4B434E545F53484946542943
:10D4200000FFFFFF2E66736C5F736468632E633AC0
:10D4300031343535203A2068616E646C6520213DB9
:10D44000204E554C4C0000002E66736C5F73646870
:10D45000632E633A31343536203A2063616C6C6256
:10D4600061636B20213D204E554C4C002E66736C41
:10D470005F736468632E633A31353033203A207429
:10D4800072616E7366657220213D204E554C4C00D2
:10D490002E66736C5F736468632E633A313630377F
:10D4A000203A20735F7364686348616E646C655BE7
:10D4B000305D20213D204E554C4C00FF2E66736C94
:10D4C0005F756172742E633A313435203A20696E8B
:10D4D0007374616E6365203C207561727441727271
:10D4E0006179436F756E74002E66736C5F7561723F
:10D4F000742E633A323138203A20636F6E66696762
:10D50000000000002E66736C5F756172742E633AC2
:10D51000323139203A20636F6E6669672D3E626151
:10D520007564526174655F42707300002E66736C9F
:10D530005F756172742E633A323231203A20287559
:10D54000696E74385F742946534C5F4645415455A3
:10D5500052455F554152545F4649464F5F53495AC1
:10D56000456E286261736529203E3D20636F6E66BB
:10D5700069672D3E74784669666F57617465726D90
:10D5800061726B002E66736C5F756172742E633A04
:10D59000323232203A202875696E74385F74294619
:10D5A000534C5F464541545552455F554152545F77
:10D5B0004649464F5F53495A456E28626173652953
:10D5C000203E3D20636F6E6669672D3E7278466926
:10D5D000666F57617465726D61726B002E66736C55
:10D5E0005F6F735F6162737472616374696F6E5FA2
:10D5F000626D2E633A373432203A206576656E7458
:10D6000048616E646C6500FF0700000100030100C3
:10D6100060011D000024F400080400000000000068
:10D6200000002602000301030301000001FFFFFFC9
:10D63000000301030104000100FFFFFF01010000DE
:10D640000000000080000000000000000000010059
:10D6500000000000000000000000000000020000C8
:10D6600000010200000004020000000502000000AA
:10D670000702000000FFFFFF000000008000000024
:10D680000000000000000100000000000000000099
:10D690000000000000020000000102000000FFFF87
:10D6A00000000000800000000000000000000100F9
:10D6B0000000000000000000000000000002000068
:10D6C0000003020000000402000000050200000048
:10D6D00001000000E09304007F0000000100000052
:10D6E000A08601007F00000001000000E09304001C
:10D6F0007F00000001000000A08601007F00000004
:10D7000000FFFFFF40420F00000000010000000189
:10D71000010000002E73646D6D635F636F6E666958
:10D72000672E633A3330203A206361726400FFFF52
:10D73000030000002A2A2A20617373657274206630
:10D7400061696C6564203A20002A2A2A205F4373AD
:10D7500079735F616C6C6F63206661696C65640AE4
:08D760000072007700FFFFFFDB
:10D7800010B003400000020204000000000000008E
:10D79000B4A501200000010000000000000001000D
:10D7A000FFFF0000906001205A005B005C005D00FC
:10D7B00006000000FFFFFFFF9A99993F020000005A
:10D7C000FFFFFFFFFFFFFFFFFFFFFFFF00093D001F
:10D7D0000080000000004001170000000000000071
:10D7E0001700000000000000FFFFFFFFFFFFFFFF2A
:04000003000002698E
:00000001FF
